:020000040040BA
:1040000020540020A9DF400019504000B952400060
:1040100069E0400069E0400069E040000000000005
:1040200000000000000000000000000061E340000C
:1040300069E0400000000000C1E3400025E44000CA
:1040400069E0400069E0400069E0400069E040004C
:1040500069E0400069E0400069E0400000000000C5
:1040600069E04000B50541000000000075BB40005C
:1040700089BB4000B9D7400069E0400069E04000DA
:1040800069E0400069E04000C9D74000C1904000AD
:10409000C905410069E0400069E040005D5440000E
:1040A00069E0400069E0400069E0400069E04000EC
:1040B00069E04000A94A400069E0400000000000BB
:1040C00000000000000000000000000000000000F0
:1040D00000000000000000000000000000000000E0
:1040E00000000000000000000000000000000000D0
:1040F00000000000000000000000000069E0400037
:1041000089CC400069E04000000000000000000091
:10411000000000000000000000000000000000009F
:10412000000000000000000000000000000000008F
:10413000000000000000000000000000000000007F
:10414000000000000000000000000000000000006F
:104400001C20010010B5054C237833B9044B13B1BF
:104410000448AFF300800123237010BDE80C002096
:1044200000000000345341000C4B43B10C480D49CF
:1044300010B5AFF300800C48036823B910BD0A48DB
:10444000036833B97047094B002BF7D0BDE8104023
:104450001847064B002BF5D0184700BF000000009E
:1044600034534100EC0C00203453410000000000A4
:104470000120704770470120704700207047704747
:1044800001207047014B1878704700BF0C0D0020C9
:104490007047000058B908B5054B1B78012B00D0B8
:1044A00008BD044B1B68002BFAD09847F8E770470B
:1044B000100D0020040D002008B50C4B9847C37860
:1044C0000B4A1370012B0CD101220A4B1A700022E7
:1044D000094B1A80094B9847094B1B681BB1984739
:1044E00001E0084B9847012008BD00BFBDB7400060
:1044F0000C0D0020100D00200E0D00209505410030
:10450000040D0020A105410008B5054B1B78012BC7
:1045100000D008BD0022034B1A70034B9847F8E700
:104520000C0D0020100D0020A105410010B582B037
:10453000074B00930B46024600218420054CA04700
:1045400018B9054A13680133136002B010BD00BFEB
:1045500095444000C1D34000080D0020014B186075
:10456000704700BF040D00202DE9F0474FF40046CE
:10457000BF4B5E600B20BF4CA0470C20A047BE4B3A
:104580004FF0400CC3F810C0C3F8A0C0C3F834C04B
:104590004FF0807EC3F810E0C3F8A0E0C3F834E029
:1045A000B64A01271761C2F8A0705763022414614C
:1045B000C2F8A04054631C61C3F8A0405C631F664E
:1045C000C3F890705F655F62C3F88070196F3943FC
:1045D0001967596F21F0010159675F604FF480310D
:1045E0001966C3F8901059655962C3F88010186FA6
:1045F00008431867586F20F48030586759601C6171
:10460000C3F8A0405C6304205861C3F8A00058665A
:10461000C3F8900058655862C3F88000196F21F004
:1046200004011967596F21F00401596718211966AF
:10463000C3F8901059655962C3F880101D6F25F0BA
:1046400018051D675D6F25F018055D675960082521
:104650001D66C3F890505D655D62C3F88050196FA8
:1046600021F008011967596F21F0080159675D6051
:1046700010211966C3F8901059655962C3F880106B
:10468000D3F8708028F01008C3F87080D3F87480D5
:1046900028F01008C3F8748059604FF48028C3F8DC
:1046A0001480C3F8A0804FF02009C3F81490C3F819
:1046B000A090C3F810C0C3F8A0C0C3F834C0C3F8BA
:1046C00010E0C3F8A0E0C3F834E01761C2F8A070AE
:1046D00057631461C2F8A04054634FF4007CC3F8E0
:1046E00060C0C3F890C0C3F854C0C3F824C0C3F876
:1046F00080C01C6F44EA0C041C675C6F24F40074D7
:104700005C67C3F804C04FF480641C66C3F8904033
:104710005C655C62C3F880401F6F27431F675F6F53
:1047200027F480675F675C604FF4006EC3F810E0A9
:10473000C3F8A0E0C3F834E04FF400275F61C3F88A
:10474000A0701F66C3F890705F655F62C3F88070E9
:104750001F6F27F400271F675F6F27F400275F672D
:104760004FF480175F61C3F8A0701F66C3F89070A4
:104770005F655F62C3F880701F6F27F480171F6743
:104780005F6F27F480175F674FF480575F61C3F84E
:10479000A0705F66C3F890705F655F62C3F8807059
:1047A0001F6F27F480571F675F6F27F480575F677D
:1047B0004FF400575F61C3F8A0704FF480775761E2
:1047C000C2F8A0704FF48048C3F86080C3F89080AE
:1047D000C3F85080C3F82480C3F88080D3F870A059
:1047E0002AF4804AC3F870A0D3F874A02AF4804A4F
:1047F000C3F874A0C3F81080C3F8A080C3F8308059
:104800005E61C3F8A0604FF400365E61C3F8A0603B
:104810001066C2F8900050655062C2F88000166FB2
:1048200026F004061667566F26F004065667506099
:104830001566C2F8905055655562C2F88050106FE9
:1048400020F008001067506F20F008005067556096
:104850000B4DD5F8140140F03000C5F8140151613A
:10486000C2F8A0105166C2F890105165516209E07B
:1048700050140E40F1DC4000000E0E4000100E40BF
:1048800000020E40C2F88010116F21F01001116774
:10489000516F21F010015167C2F81090C2F8A0903A
:1048A000C2F83490C2F810C0C2F8A0C0C2F830C03C
:1048B0004FF400015961C3F8A0105966C3F8901075
:1048C00059655962C3F88010196F21F40001196706
:1048D000596F21F400015967C2F860E0C2F890E016
:1048E000C2F854E0C2F824E0C2F880E0116F21F46D
:1048F00000611167516F21F400615167C2F804E053
:104900001466C2F8904054655462C2F88040116F3A
:1049100021F480611167516F21F480615167546007
:104920001F66C3F890701F655F62C3F880701A6FCE
:1049300022F480721A675A6F22F480725A671F61DC
:10494000C3F8A0701F63BDE8F08700BF08B5034B34
:1049500053F8203003B1984708BD00BF6C10002009
:1049600010B582B0036B0193002400E00134172CD2
:1049700009D8064B53F82420019B1A42F6D0204652
:10498000034B9847F2E702B010BD00BF304441002E
:104990004D49400000230360064A4260064A826097
:1049A0004FF48022C2600222027442748374C37482
:1049B000037570470000DC05808D5B00036C1943B4
:1049C0000164704710B58B7C23B34FF000434A68F5
:1049D0008C686400B2FBF4F2013A120292B2134303
:1049E0000A7C120602F0706213434A7C120702F03E
:1049F00040521343CA6813434360CB7C63B14FF00A
:104A000080730A7D52B90022134303640968054B81
:104A1000984710BD0023DAE70023F2E74FF4801235
:104A2000F2E700BFBD49400008B5036B13F0807F7B
:104A300001D0192008BD01230360064B98470023CD
:104A400004E00021044A42F823100133172BF8D95F
:104A5000002008BDC54940006C100020B1F1FF3FA7
:104A600004D0044B53F82130436270474FF0FF33BA
:104A7000436270473044410010B5084C44F821208F
:104A8000074A4FF00054C2F880411B01DBB282F8A4
:104A90001D331460034B984710BD00BF6C100020FD
:104AA00000E100E05D4A400008B50248024B98472B
:104AB00008BD00BF008003406149400042F26663C8
:104AC00003FB00F008E000BF00BF00BF00BF00BF55
:104AD00000BF00BF00BF01380028F4D170470000BC
:104AE000124B1A68126802601A6853684360936830
:104AF0008360D368C3600E4B1B68D9680161196974
:104B00004161596981619969C161D9690162196A13
:104B10004162596A81629B6AC36213690363054BF0
:104B20001B68436353698363704700BFC41300204D
:104B30006C110020781100200D4B1A6892690260F8
:104B40001B68DB6943600B4B1B681A6882605A68FC
:104B5000C2609B680361002306E05A1D064951F8B4
:104B6000231040F822100133092BF6D9704700BFFB
:104B7000C41300206C110020E01000200A2308E07C
:104B800003F180420A3A044951F8231040F82210F8
:104B90000133182BF4D97047E0100020192308E0E6
:104BA00003F18042193A064951F8231040F82210C7
:104BB00001331F2BF4D9024BD3F88030C361704707
:104BC000E0100020FEE70000284B5B6A13F0010FA5
:104BD00005D0EFF30583042B01D004207047234B4D
:104BE0005B6A13F0020F05D0EFF30583052B01D0AC
:104BF000052070471D4B5B6A13F0080F05D0EFF3DB
:104C00000583062B01D006207047184B5B6A13F012
:104C1000800F05D0EFF305830B2B01D00B207047DD
:104C2000124B5B6A13F4807F05D0EFF305830C2BE6
:104C300001D00C2070470D4B5B6A13F4806F05D0D8
:104C4000EFF305830E2B01D00E207047074B5B6AF4
:104C500013F4006F05D0EFF305830F2B03D00F2063
:104C60007047002070470020704700BF00ED00E053
:104C700000230FE0114AD2F80412A3F12000012210
:104C80008240114205D0EFF3058203F110009042FB
:104C900013D10133312B0FD81F2BEBD8074AD2F891
:104CA000001201229A401142F3D0EFF3058203F182
:104CB00010009042EDD070470020704700E100E006
:104CC00010B5EFF308831C4613F0070F00D01C1F2C
:104CD000174B5B6813F0010F01D0B7EE000A154BBC
:104CE0005B6813F4006F15D0134A22F001026FF0D5
:104CF000060E002303F1807344F8043C44F8082CAA
:104D00000E4B44F80C3C203C84F3088884F309885B
:104D1000704710BD0A4B9847034628B1094A22F054
:104D200001026FF00E0EE5E7074B98470346F5E7E3
:104D300030EF00E000ED00E0E14D4000C54B4000E9
:104D4000C94B4000C14C4000714C4000064A93687A
:104D500023F07F4323F4706343F0254343F4E0637F
:104D60009360024B1360704700140E40080000A5CA
:104D7000024B1860024B1960704700BF641100209D
:104D8000C0130020014B1870704700BF110D0020A8
:104D9000C0F30800014B1880704700BFDC100020F2
:104DA00008B5024650B9084B0849196008495960CE
:104DB000002199601046074B984708BD024B0649F1
:104DC000196006495960F5E7FC01002098020020AF
:104DD00008020020D9B04000E0000020F8000020C8
:104DE00070B564201B4B984700221B4B1A7062B6AB
:104DF00061B60120194B9847194B9847194B9847B2
:104E000007E01948194B98470028FAD0184B1B782F
:104E1000DBB9114B1B78002BFBD0154B1B7813B95A
:104E200000210D4A117010484D220270114A157868
:104E300045708370104E34682A46214604300F4B6B
:104E400098472C4434600020DEE7013B084A137089
:104E5000DFE700BFBD4A400070110020A14D4000B7
:104E6000C9B74000AD05410080130020E5B0400007
:104E700068110020D4100020D8100020611A4100D1
:104E8000F8B505464F4B4FF0FF32C3F88020C3F80A
:104E90008420C3F88021C3F8842103F540635A6855
:104EA00042F020625A605A6A22F400425A62464B2B
:104EB0009A6D5A6C22F040625A645A6C42F0006259
:104EC0005A64424C4FF4804363634FF4006363635E
:104ED0004FF48073636302203D4EB0474FF0807300
:104EE00063630420B0473B4F01237B630420B0473A
:104EF00002237B6340236363374A136823F0010373
:104F00001360364B5A6F42F480725A675A6F42F4FC
:104F100000725A67324AD2F8143143F44063C2F83F
:104F20001431002383F311882E4B1D60EA6A12F0BE
:104F3000040F26D069682C4B19602B4B1B6820335B
:104F40002A490B6012F0100F1FD148330B60284D17
:104F50002846284B9847244B1F6807F12004403D02
:104F600007F1600E2E4620686168A268E3680FC6EC
:104F7000103435467445F5D13A6E1F4BC3F8802086
:104F800006E02968184B1960D7E71B481B4B984768
:104F9000144B1B689B6813F4007F03D0134A1368FB
:104FA00004331360164B1B7813B90322154B1A8078
:104FB000154BD96A154A11609A6A154B1A60154B40
:104FC0009847F8BD00E100E000000140000E0E40EF
:104FD000BD4A400000100E4010E000E000400440D8
:104FE00000020E406C110020C41300207811002034
:104FF00020110020F1524000E0100020E552400056
:10500000110D0020DC10002000ED00E0D010002089
:1050100074110020C14C40006FF0060E70477047BD
:1050200070B58AB00446402200218048804B9847E2
:1050300023782A3B2A2B39D8DFE813F02B003800DD
:1050400038003800380038003800380038003800A0
:105050003800380038003800380038003800380090
:10506000380038003800380038003800F000ED0013
:10507000380038003800880038008E0038003800CA
:105080003800C40038003800380038003D004D00BA
:10509000790066490B462A2203F8012B654A1068FD
:1050A000C1F801009188927999809A715F48624BAA
:1050B00098470AB070BD5D4B52221A705F4A127851
:1050C0005A705F4A12885A805E4A12685A605E4A75
:1050D00012689A60EAE7554B53221A7062785A7048
:1050E0006378032BE2D8DFE803F0020A121A574C68
:1050F0002046574B98473C2304F8013CD6E7534CD5
:105100002046544B98473C2304F8013CCEE74F4CD3
:105110002046514B98473C2304F8013CC6E74B4CD2
:1051200020464E4B9847202304F8013CBEE73F4CF5
:10513000542323704A4D102128684A4B9847C2B225
:1051400062702968A01C484B9847AFE7374B47224D
:105150001A7004225A70A9E7344B49221A706278F7
:105160005A7063784BB1012B10D0022B14D0032B53
:105170001BD02E4B5E609D6098E73C4E3C4D3D4BF6
:105180003D4A92E8030018601971F2E73B4E3C4D2E
:105190003C4A384B1A60ECE73B4E3C4D354B3C4AA1
:1051A00092E8030018609980E3E73A4E68463A4B6C
:1051B0009847009D35442F4B384A92E80300186009
:1051C0001971D6E72579637905EB0325A37905EBFA
:1051D0000345E37905EB0365314B1D6013484D230F
:1051E000037063784370A378837062782946043033
:1051F0001D4B9847A378002B3FF458AF627829499C
:105200000A70013B28490B701544254B1D60012293
:10521000264B1A704AE7264B984747E7254BBB2297
:105220001A601A225A60224B98473FE780130020E9
:105230005D1C410090444100E5B04000110D00208C
:10524000DC100020D01000207411002084130020F6
:10525000E14A4000394B40007D4B40009D4B4000EF
:10526000C0130020DD1F4100611A41001000002022
:10527000E80C00208C13002098444100E80C00202A
:105280001C2400206273730020240020205400207E
:10529000A044410020540020111D4100A8444100B9
:1052A000D8100020D41000206811002070110020B8
:1052B0004D4D400090140E4072B671B6EFF303836B
:1052C000EFF30982EFF30881DFF814D02DE9FE4FE8
:1052D0006846FFF7D5FDBDE8FE4F8D4670470000DC
:1052E00080130020F1EE101AA0EC200A0160704734
:1052F000A0EC108A704700BF10B51720234CA047C0
:105300001820A047224B4FF480321A66C3F8902031
:105310005A655A62C3F88020196F11431967596F93
:1053200021F4803159675A6001225A66C3F89020EF
:105330005A655A62C3F88020196F11431967596F73
:1053400021F0010159675A60A3F5206340F212620F
:10535000DA644FF400621A600E4B0F4A5A60412221
:105360005A62052119600D4A5A644FF4F572DA65E4
:1053700000229A6519640A4B1A700A4B4FF4000216
:105380001A60702283F8172310BD00BFF1DC4000C3
:10539000000E0E40000001400406090001C4000A8E
:1053A000CC13002000E100E010B54FF40002124BD6
:1053B000C3F88020BFF34F8FBFF36F8F0F4B4FF4B5
:1053C00080321A66C3F890205A655A62C3F880206A
:1053D000196F21F480311967596F21F480315967B1
:1053E0001A601A61C3F8A0205A631720044CA04722
:1053F0001820A04710BD00BF00E100E0000E0E40E5
:1054000045DD4000642800D964200F4AD36D03FBBA
:1054100000F30E49A1FB03135B09936548B10A4BE6
:105420005A6C22F040625A645A6C42F080625A64AC
:1054300070471346526C22F040625A645A6C42F034
:1054400000625A64704700BF000001401F85EB51A5
:10545000014B1888704700BFD01300200F4B1B6A08
:1054600013F0010F06D000220D490A700D490A60A1
:105470000D490A6013F0400F0ED00122084B1A703C
:10548000064B9A69094BB3FBF2F3064A1360C3EB70
:1054900003139A00044B1A60704700BF00000140DC
:1054A000CC130020C8130020D01300201F1A0500C1
:1054B000014B1870704700BF00010020064B1B789D
:1054C00023B94FF40062054B1A6370474FF4006232
:1054D000024B5A63704700BF00010020000E0E40CF
:1054E000064B1B7823B94FF40062054B5A63704793
:1054F0004FF40062024B1A63704700BF00010020A6
:10550000000E0E402DE9F04186B00F461646984633
:10551000B8B9344B984704460025049598238DF874
:10552000043001238DF805308DF8065002238DF8E4
:10553000083005AB03938DF8075020462A4B984757
:105540000EE02A4B98470446E6E72046284B98474A
:10555000002044E09DF8153008F805300135EDB223
:10556000B54238D28DF814708DF8155000238DF89F
:105570000630322201A920461E4B9847A379DBB2A0
:10558000022B0BD020461C4B9847322201A9204603
:10559000184B9847A379DBB2022BD6D101238DF8A3
:1055A0000630322201A92046124B9847A379DBB27C
:1055B000022BCFD02046104B9847322201A920461B
:1055C0000C4B9847A379DBB2022BC3D02046084B83
:1055D0009847002003E02046054B9847012006B07D
:1055E000BDE8F081850541003D7440008D05410016
:1055F0005174400069744000197640002DE9F04173
:1056000086B00C4617469846D8B9264B98470546AB
:105610000026049698238DF8043001238DF8053078
:1056200002238DF8063003238DF8083005AB039371
:105630008DF807408DF8156028461B4B9847344677
:1056400005E01A4B98470546E2E70134E4B2BC4254
:1056500021D28DF8144018F804308DF8163032221B
:1056600001A92846124B98470646AB79DBB2022BBC
:10567000EBD028460F4B9847322201A928460C4B05
:1056800098470646AB79DBB2022BDED028460A4BA0
:105690009847002602E02846074B9847304606B058
:1056A000BDE8F081850541003D7440008D05410055
:1056B0006974400019764000517440002DE9F043B0
:1056C00087B00C4690461F46DDF83890D8B9274B76
:1056D000984705460026049698238DF80430012348
:1056E0008DF8053002238DF8063003238DF808303D
:1056F00005AB03938DF807408DF8156028461C4BC9
:105700009847344605E01B4B98470546E2E70134CD
:10571000E4B2BC4223D204EB08038DF8143019F82C
:1057200004308DF81630322201A92846124B9847D2
:105730000646AB79DBB2022BE9D028460F4B9847DF
:10574000322201A928460C4B98470646AB79DBB2BA
:10575000022BDCD028460A4B9847002602E0284658
:10576000074B9847304607B0BDE8F08385054100F8
:105770003D7440008D054100697440001976400079
:1057800051744000F8B506460D461746344BAA2220
:105790001A7011225A700222F021324CA0470128BF
:1057A00001D00020F8BD2C0AEDB22D4B1C705D70AD
:1057B0009C70DD701C715D7100229A719022DA710B
:1057C00067B182221A72264B0922C2213046254F28
:1057D000B847012806D001280BD0F8BD0222204B83
:1057E0001A72F0E71E4B0922C22130461E4EB04706
:1057F000F1E71B4B1B789C4201D00020F8BD184BF1
:105800009B789C4201D00020F8BD154B1B799C422F
:1058100001D00020F8BD124B5B789D4201D00020E2
:10582000F8BD0F4BDB789D4201D00020F8BD0C4B3A
:105830005B799D420BD10A4B9B7953B9084BDB79BD
:10584000902B08D1064B1B7A022B06D1F8BD002005
:10585000F8BD0020F8BD0020F8BD0020BDE700BF66
:10586000D4130020FD5540000555400010B500221E
:10587000054B1A7029B91121034B0122034CA04793
:1058800010BD1021F8E700BFD4130020FD554000E3
:1058900010B50022054B1A7029B92821034B0122AB
:1058A000034CA04710BD2921F8E700BFD413002006
:1058B000FD55400070B506460A4CAA2323701123FB
:1058C000637023460222F021074DA847FF2323706F
:1058D000012800D070BD23460122C0213046A847D0
:1058E000F8E700BFD4130020FD55400010B539B9CA
:1058F0000022044B1A7001223621034CA04710BD30
:105900000322F6E7D4130020FD55400038B50546C4
:105910000C4BAA221A7012225A700222F0210A4C51
:10592000A047012801D0002038BD064B0322BF212B
:105930002846064CA047012801D0002038BD014B65
:10594000987838BDD4130020FD554000055540001F
:1059500038B50D46094B0E228421094CA047012879
:1059600001D0002038BD054B186859689A68286036
:105970006960AA609B89AB810E2038BDD4130020DA
:105980000555400010B50B462C227021014CA04754
:1059900010BD00BFFD5540002DE9F04184B000234B
:1059A0008DF80F300139062945D8DFE801F00806E7
:1059B000040D0F111300214D02E0214D00E0214D97
:1059C00080460120002411E01F4DF9E71F4DF7E745
:1059D0001F4DF5E71F4DF3E70DF10F03024640465B
:1059E0001D4EB0473C44E4B20134E4B201280BD16F
:1059F00023462F5D47B1621CA95C012FECD902330D
:105A00002B44781EC0B2E9E7012804D0012809D050
:105A100004B0BDE8F081114B0222FF2140460E4C3C
:105A2000A047F3E70E4B00930D230B22F9214046CC
:105A30000C4CA047ECE70020EAE700BF044541001A
:105A4000B446410034474100B44441008845410018
:105A500034464100D8454100FD554000B044410066
:105A6000B8474100BD56400008B50721014B984793
:105A700008BD00BF9959400010B5274900238B721B
:105A8000CB720B7340F2DC528A806422CA800B8096
:105A900021F8083F0620214B98470B20204B9847C0
:105AA00080B90C201E4B984788B900221A4B5A80A7
:105AB0001C4B984701211C4B984701280CD0164BD2
:105AC000987A10BD19490B20144B9847E9E71849FB
:105AD0000C20124B9847E8E701220F4B9A72114BAA
:105AE00098470521134B9847034650B10A4AD37291
:105AF000002BE4D00B4B98470F4B9847064B588030
:105B0000DDE7084CA0470021074B9847A047032139
:105B1000084B98470346E9E734140020B17D400064
:105B2000E57D40008D054100215C400038140020D7
:105B30003A140020515E4000E15D4000014B987A2C
:105B4000704700BF3414002008B5224B9B7A8BB9F4
:105B5000214A13781F490888204921F8130001338E
:105B6000DBB213700F2B02D900221B4B1A700023DB
:105B70001A4615E01A4B98471A4B9847154B1B8944
:105B8000984203D80022134B1A80E1E7C01A114B48
:105B90001880DDE7114931F813100A440133DBB2F4
:105BA0000F2BF7D912090B4B1B7B4BB109498B8883
:105BB000C9885B1A9A420CD80022064B1A7308BD9A
:105BC00004498B88C9880B449A4202D30122014BB5
:105BD0001A7308BD34140020120D00201414002084
:105BE0008D054100715D4000014B187B704700BF7F
:105BF00034140020014B1888704700BF3414002073
:105C000008B5014B984708BD215F400008B5024B1D
:105C10009847024B984708BD8D054100295F400019
:105C200030B587B005460C4600238DF80730722248
:105C30008DF808208DF80B3001228DF809208DF8A1
:105C40000C200DF10702049202228DF80A20059320
:105C5000434B9847322202A92846424B9847002CD2
:105C600043D1012402238DF80A3080238DF80B30B4
:105C700001238DF807309C4244D08F238DF80B30E0
:105C800003238DF80A30012C43D09DF8073003F030
:105C9000F00343F005038DF8073002238DF80A3036
:105CA000012C3DD0AA238DF80B3001238DF807304D
:105CB0009C423CD007238DF80730F9238DF80B3038
:105CC000012C3BD005238DF8073080238DF80B3055
:105CD000012C3AD02846244B9847012C3CD0002276
:105CE000224B1A70204607B030BDA8238DF80B3028
:105CF00001238DF80730322202A92846194B984714
:105D00000446AFE7322202A92846164B98470446BC
:105D1000B3E7322202A92846124B98470446B4E75B
:105D2000322202A928460F4B98470446BAE732228E
:105D300002A928460B4B98470446BBE7322202A92A
:105D40002846084B98470446BCE7322202A9284659
:105D5000044B98470446BDE70122044B1A70C1E783
:105D60003D7440006974400051744000130D0020E0
:105D700030B587B004460023059301AB049372232A
:105D80008DF8083001238DF809309C238DF80B30F5
:105D900002238DF80C3003238DF80A300C4B984702
:105DA000322202A920460B4B9847054620460A4B53
:105DB0009847012D04D00020084B187007B030BD63
:105DC0009DF804009DF8053000EB032080B2F5E754
:105DD0003D7440006974400051744000130D002070
:105DE00030B587B004460023059301AB04937223BA
:105DF0008DF8083001238DF80930C0238DF80B3061
:105E000002238DF80C3003238DF80A300C4B984791
:105E1000322202A920460B4B9847054620460A4BE2
:105E20009847012D04D00020084B187007B030BDF2
:105E30009DF804009DF8053000EB032080B2F5E7E3
:105E40003D7440006974400051744000130D0020FF
:105E5000F0B587B00646002305930DF107030493C0
:105E600072238DF8083001238DF80930D9228DF87E
:105E70000B208DF80C3002238DF80A304901C9B28D
:105E800041F010018DF80710214B9847322202A9EA
:105E90003046204B98470546D7238DF80B302123F9
:105EA0008DF8073001280BD030461B4B9847DC2378
:105EB0008DF80B3003238DF80A300024274608E0C4
:105EC000322202A93046134B98470546ECE70134CD
:105ED000A4B2012D18D1BFB9092C15D819200F4B28
:105EE000984730460A4B9847322202A93046094B60
:105EF000984705463046084B98479DF8073013F001
:105F0000010FE4D00127E2E7384607B0F0BD00BF3B
:105F10003D744000697440005174400035F2400007
:105F20000048704744140020A84BDB78032B00F294
:105F30004081A64B1B793F2B00F23D81A34B5B793F
:105F4000072B00F23A81A14B9B79082B00F2378195
:105F50009E4B1B7A013BDBB2022B00F232819B4B42
:105F60005B7A032B00F22F81984B9B7A072B01D988
:105F70000020704710B586B00446002305937223B5
:105F80008DF8083001238DF809300DF107020492D5
:105F90008DF80C308E4B984780238DF80B300323FF
:105FA0008DF80A30322202A920468A4B98470128F0
:105FB00017D1864B1B78D3B19DF8073043F01003FF
:105FC0008DF8073002238DF80A30322202A92046CC
:105FD000804B9847012811D020467F4B98470020DE
:105FE00003E020467C4B9847002006B010BD9DF88A
:105FF000073023F010038DF80730E3E782238DF894
:106000000B30724B5B788DF80730322202A92046A4
:10601000704B9847012817D18D238DF80B30402302
:106020008DF80730694B9B7813B148238DF8073002
:10603000322202A92046674B9847012809D0204602
:10604000654B98470020D0E72046634B98470020D7
:10605000CBE78E238DF80B305C4AD3789B01DBB203
:10606000127902F03F0213438DF80730322202A961
:106070002046584B9847012804D02046564B984755
:106080000020B2E78F238DF80B30504A53795B0123
:10609000DBB2927902F00F0213438DF807303222FF
:1060A00002A920464B4B9847012804D020464A4B72
:1060B0009847002099E7A9238DF80B30434BDB79F3
:1060C0008DF80730322202A92046424B984701281A
:1060D0000CD1AA238DF80B303C4B1B7A022B18D025
:1060E000032B1AD0012B06D000207EE720463A4B26
:1060F0009847002079E78DF80730322202A9204620
:10610000344B984701280CD02046334B9847002049
:106110006BE702238DF80730EFE703238DF8073094
:10612000EBE7B3238DF80B30284B5B7A03F00303C6
:106130008DF80730322202A92046264B98470128C5
:1061400004D02046244B984700204EE7D9238DF8F1
:106150000B3003238DF80A30322202A920461D4B52
:106160009847012804D020461B4B984700203CE765
:106170009DF8073003F0F80343F01003134A927AB6
:1061800002F0070213438DF8073002238DF80A301E
:10619000322202A920460F4B9847012804D02046FE
:1061A0000D4B9847002020E720460B4B98470120D5
:1061B0001BE7002070470020704700207047002038
:1061C0007047002070470020704700BF4414002033
:1061D0003D744000697440005174400000FB01F0C0
:1061E000C0F3C71070470000F0B587B004460E46F4
:1061F000234B9847002304938A238DF8043001230E
:106200008DF805308DF808300DF11703039334270E
:106210008DF8077002238DF8063033788DF817302B
:10622000322201A92046174DA8478DF80770337810
:106230008DF81730322201A92046A8478DF8077043
:1062400033788DF81730322201A92046A84735232C
:106250008DF8073073788DF81730322201A9204667
:10626000A84736238DF80730B3788DF817303222DF
:1062700001A92046A8472046034B984707B0F0BD28
:106280003D7440006974400051744000F0B587B01F
:106290000446002505958A238DF8083001268DF8DF
:1062A00009608DF80C600DF107030493254B9847A6
:1062B00055238DF807308DF80B5002238DF80A30E6
:1062C000322202A92046204DA84703238DF807302B
:1062D0008DF80B60322202A92046A8478DF807608E
:1062E00004238DF80B30322202A92046A847072349
:1062F0008DF8073030238DF80B30322202A920466A
:10630000A8470F278DF8077031238DF80B30322204
:1063100002A92046A8478DF8077032268DF80B6039
:10632000324602A92046A8478DF8077033238DF81E
:106330000B30324602A92046A8472046034B984717
:1063400007B0F0BD3D7440006974400051744000D6
:10635000F0B583B007460C46802900D980240C4B49
:106360001C700C4E214630780B4DA8478DF8040068
:1063700021467078A8478DF805002146B078A847D7
:106380008DF8060001A93846044B984703B0F0BDCC
:1063900001010020140D0020DD614000E961400092
:1063A00010B5054B0C888A781C809A70034B1978BD
:1063B000034B984710BD00BF140D002001010020C1
:1063C0005163400010B586B004468DF808100023D4
:1063D0000593E7238DF80B300DF107030493012398
:1063E0008DF80C308DF8093003238DF80A303222F5
:1063F00002A90A4B9847012801D006B010BD9DF8AC
:10640000073043F001038DF8073002238DF80A307E
:10641000322202A92046014B9847EEE769744000FA
:1064200010B586B004468DF80810002305930DF1D1
:106430000703049301238DF80C308DF809300623EF
:106440008DF80B3003238DF80A30322202A9224B3B
:1064500098479DF8073063F07F038DF807300223DB
:106460008DF80A30012818D000238DF807300C234E
:106470008DF80B30012816D00D238DF80B30012834
:1064800017D00E238DF80B30012818D00F238DF86C
:106490000B30012819D006B010BD322202A92046C7
:1064A0000D4B9847E0E7322202A920460A4B984755
:1064B000E2E7322202A92046074B9847E1E7322261
:1064C00002A92046044B9847E0E7322202A9204661
:1064D000014B9847DFE700BF6974400010B586B0F4
:1064E00004468DF8081000230593E7238DF80B3040
:1064F0000DF10703049301238DF80C308DF809305A
:1065000003238DF80A30322202A90A4B984701284A
:1065100001D006B010BD9DF8073023F001038DF8BF
:10652000073002238DF80A30322202A92046014B9F
:106530009847EEE76974400070B504462022214B6D
:106540001A630A20204B98472046204B9847102179
:1065500020461F4EB047054612212046B04706464A
:10656000012D0ED0012E12D0012D16D0012E1AD0E1
:106570002046184B9847012D1BD0012E1DD02846D0
:1065800070BD10212046144B98470546EAE71221BA
:106590002046114B98470646E6E7102120460F4B50
:1065A00098470546E2E7122120460C4B98470646DD
:1065B000DEE701220A4B1A70DFE70122094B1A704D
:1065C000DDE700BF00100E4035F240003D74400092
:1065D000C56340005174400021644000DD64400008
:1065E000170D0020180D002010B1034B18787047CC
:1065F000024B1878704700BF180D0020170D0020BF
:1066000030B587B004460D4600220592A8238DF8C8
:10661000083001238DF809308DF80B200DF10702A9
:1066200004928DF80C3002238DF80A30124B9847F3
:10663000012D0ED0022D15D000238DF80730322207
:1066400002A920460D4B984720460D4B984707B0AE
:1066500030BD03238DF80730322202A92046074BB4
:106660009847F1E702238DF80730322202A920462D
:10667000024B9847E8E700BF3D7440006974400052
:106680005174400030B587B072238DF8003001237B
:106690008DF8013000238DF802308DF80330082288
:1066A0008DF8042004AA029203938DF81000C0F321
:1066B00007238DF81130C0F307438DF81230000E18
:1066C0008DF813008DF81410C1F307238DF81530E1
:1066D000C1F307438DF81630090E8DF81710084CDA
:1066E000A047084B9847A04732226946064B984777
:1066F0000546A047054B9847284607B030BD00BF68
:10670000850541003D7440006974400051744000AB
:1067100030B587B00D4672238DF8043001238DF813
:10672000053000238DF806308DF8073004228DF8EF
:10673000082005AA039204938DF81400C0F30723E0
:106740008DF81530C0F307438DF81630000E8DF824
:106750001700184CA047184B9847A047322201A9B0
:10676000164B98470446012808D0124B9847144B03
:106770009847012C0DD0204607B030BD01238DF87D
:1067800006300C4B9847322201A90C4B984704461F
:10679000EBE79DF814309DF8152003EB02239DF8DC
:1067A000162003EB02439DF8172003EB02632B60D6
:1067B000E1E700BF850541003D7440006974400079
:1067C000517440002DE9F04E82B0824689469346CE
:1067D0001BB11E46002501272FE00127012F40D0C5
:1067E000012F49D0012F4DD0012F51D04FF400037C
:1067F00001932F4B98470446012F4FD1019B13F46F
:10680000000F4BD00A9920462A4B984700284DD1BB
:1068100001A92948294B98470746EDE7EA18B25CD9
:106820004FEAC30E02FA0EF211440133DBB2A34267
:10683000F4D3012F0DD02544EDB228464D45CDD2DD
:10684000A9EB0504042C28BF0424E4B20023194654
:10685000EDE700F1201000F58070194B98470746CE
:10686000E9E74FEA0A4101F4FE0101F5000112488F
:10687000134B98470746B3E749461248104B9847D1
:106880000746AFE7594610480D4B98470746ABE718
:10689000F2210E480A4B98470746A7E71FB9052083
:1068A00002B0BDE8F08E9DF80700F9E70620F7E793
:1068B000A17A4000B97A4000100120001167400021
:1068C000856640001801200014012000FC00200013
:1068D00010B584B00A4B93E8030002908DF80C10B9
:1068E0003223009302AB002205210120054CA04772
:1068F000034610B90121044A1170184604B010BDB6
:10690000C8474100C5674000190D002070B5074D0C
:106910004FF480466E630A20054CA0472E6340F278
:106920001310A047034B984770BD00BF000E0E40E8
:1069300035F24000D168400030B583B00D463223B7
:1069400000930023024604213120074CA04704464F
:1069500010B1204603B030BD29460448044B984787
:106960000128F6D00524F4E7C56740002001200087
:106970001167400010B584B08DF80C100B0A8DF82B
:106980000D300B0C8DF80E30090E8DF80F103223E0
:10699000009303AB024604212120024CA04704B01F
:1069A00010BD00BFC567400008B5044B1B780BB194
:1069B000002008BD024B984708BD00BF190D0020FC
:1069C000D16840002DE9F04383B059B1012904D0CA
:1069D0000124204603B0BDE8F08340F65D0740F691
:1069E000050503E040F2DD7740F2857580464FF003
:1069F00000094C4601E0002CEBD1BD42E9D225F064
:106A00000306002CF7D101A93046164B98470446DF
:106A10000028F0D1019B8DF80030C3F307228DF8D8
:106A20000120C3F307428DF802201B0E8DF80330BE
:106A3000E9B2F3B2C91AC9B2C1F10403BE1B9E4246
:106A400028BF1E46042E28BF0426F6B232466944EB
:106A500008EB0900044B984735444E445FFA86F929
:106A6000C9E700BF39694000611A410028B1012817
:106A700001D000207047094800E0094800B583B004
:106A800001A9084B984728B9019B13F4006F02D065
:106A9000012000E0002003B05DF804FB4000350059
:106AA000400031003969400010B52DED028B82B0F5
:106AB000044601A93548364B98470346F8B14BB315
:106AC000002B32D0002B3BD0DFED328A002B49D097
:106AD0009FED308A73B9DDED017AB8EE677AC8EEC2
:106AE000077A9FED2D7A67EE877AFCEEE77A17EE4C
:106AF000902A6281184602B0BDEC028B10BD02A93B
:106B000051F8043D23801B0C63802448204B984798
:106B10000346D4E702A951F8043DA3801B0CE3808F
:106B20001F481B4B98470346CAE702A951F8043D8A
:106B300003F01F0323721B48154B98470346C1E718
:106B400002A951F8043DC3F3094308EE903AF8EE68
:106B5000688A9FED158A68EE888A14480C4B98471E
:106B60000346B3E702A951F8043DDBB208EE103A40
:106B7000B8EE488A28EE888ADFED077A28EE278A61
:106B80000B48034B98470346A4E700BF3008220098
:106B900039694000000000000000C84238082200A7
:106BA000540822000800200000401C46040822006F
:106BB0001408220000B583B001A941F23070094BDE
:106BC0009847034618B1184603B05DF804FB0199D5
:106BD00021F00601019141F23070034B98470346C2
:106BE000F1E700BF396940007569400030B583B0F6
:106BF00015460C4AA2FB01231B090F330093002307
:106C000002461120084CA047044610B1204603B0AC
:106C100030BD29460548064B98470128F6D0052483
:106C2000F4E700BF1F85EB51C5674000200120003D
:106C30001167400010B582B09623009313460246B8
:106C40002020024CA04702B010BD00BFC567400025
:106C5000072801D90120704710B584B08DF80C00C9
:106C600030238DF80D3041F28833009303AB0022BE
:106C700002211420014CA04704B010BDC56740009C
:106C800010F0800F11D110B584B08DF80C001023D6
:106C90008DF80D3041F28833009303AB00220221BE
:106CA0001420034CA04704B010BD0120704700BF62
:106CB000C5674000F0B583B0032832D8DFE800F0A4
:106CC0000209050747F6F07604E0184E02E0184E78
:106CD00000E0184E002401273D4604E09CB10F2C33
:106CE00011D00134E4B20F2C13D801AA0121A0194C
:106CF000114B9847B8B9002DF0D09DF80430FF2B08
:106D0000ECD00025EAE79DF80430002BE9D10027FC
:106D1000E7E717B11DB1002006E0002004E00120E4
:106D200002E0002000E0002003B0F0BDF0FF010011
:106D3000F0FF0300F07F0200ED6B400070B582B001
:106D400006460020114B984720B14FF4BE65002441
:106D500023460BE001200D4B984718B90323184632
:106D600002B070BD0A4DF2E70134E4B20E2CF6D841
:106D7000002BF9D101AA01212819064B9847034697
:106D80000028F1D19DF804203255EDE7B56C4000A4
:106D9000F0050200ED6B400030B587B01D201C4BA4
:106DA00098471C4C236C23F40013236468461A4B49
:106DB000984769462046194B9847636823F47F43F8
:106DC0006360636843F47F436360042323610823A3
:106DD000236101232361626822F08F026260104AFE
:106DE000032120460F4DA847002120460E4B98470F
:106DF000636813F0800F01D1082222600B4B4FF023
:106E000000521A60702283F81D2307B030BD00BF06
:106E1000F1DC40000080034095494000294A4000D1
:106E2000516E4000794A4000BD49400000E100E059
:106E30000222014B1A60704700800340024B188009
:106E4000024B1980704700BF02010020040100209E
:106E500010B5064C206D80B2054B9847A06DE16DD2
:106E600089B280B2034B984710BD00BF0080034039
:106E7000457F40003D6E4000014B1888704700BFC1
:106E800002010020014B1888704700BF0401002058
:106E90000D4B1B8840F68962934205D90B4A128834
:106EA0003E2A01D803207047084A128840F68961BB
:106EB0008A4203D93E2B01D804207047934201D85F
:106EC00002207047012070470201002004010020C9
:106ED00008B50120034B9847034B186000B101200F
:106EE00008BD00BFADE840005014002008B54FF0C9
:106EF000FF31024B1868024B984708BD5014002020
:106F000069EA400010B500231A4619460248006895
:106F1000024CA04710BD00BF5014002075E7400090
:106F2000154B98421BD003F5A033984219D003F5B6
:106F30008043984217D0A3F54043984215D003F5FB
:106F40008043984213D0A3F5A033984211D003F5A3
:106F50006033984201D032207047162070470820D5
:106F60007047092070470E20704713207047142087
:106F700070471520704700BF00C000404900B0FBBB
:106F8000F1F00338002302E040080133DBB2FF28B0
:106F9000FAD8020202F47F4252FA80F01B0403F492
:106FA000E0231844704700002DE9F843D0F8009022
:106FB000037ADBB2012B00F0E68009F5C0650B799E
:106FC00013B91846BDE8F88317460E460446012358
:106FD00003720023C371E1606E4B98478046B3781B
:106FE000022B08D07378012B18D033781B0403F4DC
:106FF000FE036B6050E07378012B09D033781B04DB
:1070000003F4FE0303F580736B60F378EB6043E0F9
:1070100033785B081B0403F58073F5E733785B086E
:107020001B04E6E70323A37100232372237A002BBA
:1070300000F0AB802B6A13F4807F53D113F4007FF0
:1070400078D113F0400F7AD113F0800F7CD113F078
:10705000040F4BD1394640464F4B98470028E9D0A2
:107060000723A371002323724C4BC9F800363DE07F
:107070000423A37100232372D8E70523A3710023FF
:107080002372D3E70623A37100232372CEE7394688
:107090004046414B9847E8B93379E2799B1A002B77
:1070A000C4DD2B6A13F4807FBCD113F4007FDFD1E1
:1070B00013F0400FE1D113F0800FE3D113F0040F70
:1070C000E5D0B168E379DBB25A1CD2B2E271CB5C95
:1070D0006B63DCE70723A371002323722F4BC9F8EE
:1070E0000036A3E70323A37100232372237A002B26
:1070F0004DD00223C9F800362B6A13F0010F28D1B6
:1071000013F4807F2BD113F4007F2DD113F0400FA7
:107110002FD113F0800F31D1394640461E4B98478E
:107120000028E9D00723A371002323721B4AC9F862
:10713000002646E70423A37100232372D6E7052324
:10714000A37100232372D1E70623A37100232372C6
:10715000CCE7002323720223A371012331E7032329
:10716000A371002323722CE70423A371002323724D
:1071700027E70523A3710023237222E70623A371C7
:10718000002323721DE700231BE7002319E70023D8
:1071900017E700BFA17A4000B97A400002800005DD
:1071A0002DE9F84FD0F800B0037ADBB2012B00F0E4
:1071B000CE800BF5C0670B7913B91846BDE8F88F80
:1071C00090460E460546012303720023C371E96011
:1071D000614B98478146B378032B14D07378012B09
:1071E00024D033781B0403F4FE0303F580537B6043
:1071F00096F804A0BAF1010F1ED00123CBF8003697
:107200004FF0000A64E07378012B09D033781B0437
:1072100003F4FE0303F588537B60F378FB60E7E734
:1072200033785B081B0403F58853F5E733785B0874
:107230001B0403F58053DAE70323CBF8003647E05D
:107240000323AB7100232B722B7A002B00F081807B
:107250003B6A13F0010F60D113F4807F63D113F404
:10726000007F65D113F0400F67D113F0800F69D113
:1072700041464846394B98470028E9D00723AB716F
:1072800000232B72364ACBF8002696E70423AB7115
:1072900000232B72D8E70523AB7100232B72D3E7B1
:1072A0000623AB7100232B72CEE70723AB710023BB
:1072B0002B722B4BCBF80036C6E714F0020F07D029
:1072C000B168EB79DBB25A1CD2B2EA713A6BCA549C
:1072D000EB79DBB232799342B6D23C6A14F4807F08
:1072E000AED114F4007FD1D114F0400FD3D114F0FB
:1072F000800FD5D141464846184B98470028D4D135
:10730000BAF1000FD9D13379EA799B1A012BD4D184
:1073100002233B604FF0010ACFE700232B720223C8
:10732000AB71012349E70323AB7100232B7244E7C0
:107330000423AB7100232B723FE70523AB710023BD
:107340002B723AE70623AB7100232B7235E700233B
:1073500033E7002331E700BFA17A4000B97A40004B
:10736000028000052DE9F041064688460468204663
:107370001B4B9847312801D9BDE8F0810546194BD0
:107380009847032323602423C4F800364146164857
:10739000164B9847C4F81006002333720123B371CB
:1073A0006BB2002B07DB5A0905F01F000121814059
:1073B0000F4840F82210002B0BDB03F1604303F56C
:1073C0006143202283F8002301200A4B9847306153
:1073D000D2E705F00F05084B20225A55F4E700BF0D
:1073E000216F4000F1DC40000000DC057D6F4000B3
:1073F00000E100E0ADE8400014ED00E008B50068F1
:107400000B4B9847312811D843B2002B0CDB5B099A
:1074100000F01F0101228A402033064941F8232051
:10742000BFF34F8FBFF36F8F034B984708BD00BF6B
:10743000216F400000E100E045DD400008B54FF05D
:10744000FF310069014B9847C0B208BD69EA4000AE
:1074500010B500231A4619460069024CA047C0B275
:1074600010BD00BF75E7400008B5837963B18B7824
:10747000032B0BD8DFE803F002050205044B984705
:1074800008BD044B984708BD002008BD002008BD7A
:10749000A96F4000A171400080797047F8B5064699
:1074A000036803F5C064256AC76815F0040F0BD0A4
:1074B000E26A12F0040F07D0BA78002A4DD0022AEF
:1074C0004BD0BA78032A5ED015F0020F08D0E26ADA
:1074D00012F0020F04D0BA78012A73D0032A71D0B7
:1074E00015F4807F0DD0E36A13F4807F09D040F259
:1074F0000733A362002333720323B371FB6803B124
:10750000984715F4007F0DD0E36A13F4007F09D08B
:1075100040F20733A362002333720423B371FB6884
:1075200003B1984715F0010F16D0E36A13F0010F6D
:1075300012D0BB780BB1022B09D140F20533A36204
:10754000002333720223B371FB6803B19847BB7801
:10755000012B54D0032B52D0F8BDF279D2B2397935
:107560008A4208D2B868F279D2B2511CC9B2F1711C
:10757000825C6263A5E70222C3F8002601226262F0
:107580000422A2629DE77A78012A11D03A78120487
:1075900002F4FE0202F5805262603A79012A0DD0AF
:1075A0000122C3F800260422A262022262628BE753
:1075B0003A785208120402F58052EDE70322C3F82C
:1075C0000026F0E7B868F279D2B2511CC9B2F17165
:1075D000216B8154F179C9B23A79013A91420AD0CA
:1075E000F379DBB23A7993427FF47AAF0123636295
:1075F0000223A36274E70222C3F80026F0E740F2F8
:107600000333A362002333720223B371FB68002BA0
:10761000A2D09847A0E7000070B4056805F5C066E1
:107620000379202B0BD9A3F12001CBB21A4C0121F5
:1076300099402160216521612163002211E0174CEE
:10764000F5E701339BB2B3F52F7FFAD361630023D3
:1076500001E001339BB2B3F52F7FFAD321630132EE
:10766000D2B2092A01D80023EDE761616160326975
:107670008023C5F80036002301E001339BB2B3F547
:107680002F7FFAD332612423C5F80036002303721A
:107690000123837170BC704700100E40000E0E4035
:1076A00030B591B000238DF835308DF836308DF837
:1076B00037308DF839308DF83A30ADF83E300F2341
:1076C0008DF834300223ADF83C3001248DF8384079
:1076D0000DAA0B4907A80B4DA8470DAA0A4901A8F6
:1076E000A8471023079A1360019A1360074B1C7078
:1076F000074B1C7045F6FF72064B1A8011B030BD67
:1077000000C00240D9D74000000003401C0D0020FB
:1077100034160020FE16002042B110B420B119B179
:10772000034B586099605A805DF8044B704700BF66
:107730001C0D0020154B1B783BB3144B5B8823B307
:10774000124A52680AB311498968F1B1F0B583B0A1
:10775000009201930E4D6A46694628460D4FB84780
:107760004FF480362E62094B9B6800930A4C6A46A0
:1077700069462046B847266201212846074DA8479A
:1077800001212046A84703B0F0BD70471C0D002022
:1077900000C1024015D74000000103402DD7400032
:1077A0000223034A136202F580421362704700BF4E
:1077B00000C1024010B58CB00A4B9847069A136876
:1077C00023F010031360009A136823F01003136072
:1077D0000D20054CA0471220A0470022034B1A7031
:1077E0000CB010BDA177400045DD40001C0D00200D
:1077F000064B1B783BB1054B5888054BD3F8043139
:10780000C01A80B270470020704700BF1C0D0020D6
:1078100000C00240094AD36D23F4FF4323F07F03E5
:10782000C0F30E000343D36502F58042D36D23F409
:10783000FF4323F07F031843D065704700C0024028
:10784000014B1880704700BFFE160020014B1870D6
:10785000704700BF34160020004870470017002012
:107860000048704754140020704770472DE9F843D2
:107870004F4B984705464F4B984704467FE0A0EB97
:10788000070E1FFA8EFE0EF1F00E1FFA8EFE85E037
:107890003121002308E02F21FBE747480078C0B2E0
:1078A000012831D001339BB2994259D9DA1992B2E9
:1078B000EF2A01D9F03A92B23F4800780028ECD183
:1078C0003E48B0F9000035F9126006FB00F6F613E9
:1078D0004FEA8308DFF8ECC00CF8236008F10109D7
:1078E000C6F307260CF8096034F9122000FB02F2F7
:1078F000D21308F102000CF8002008F10308C2F3CB
:1079000007220CF80820CDE735F9120034F91220CF
:10791000024402EBD272521012F5004F05DBB2F5B1
:10792000004F03DB47F6FF7200E0254A2348B0F919
:10793000000012B202FB00F2D21398005FFA82FC40
:10794000204E06F823C000F10108C2F3072206F812
:10795000082000F1020806F808C003303254A1E7FD
:10796000194BA3F800E00F44BFB2184B1F80EF2F54
:1079700001D9F03F1F8089001248154B98474FF0FE
:10798000FF310120134B9847134B98470F4B1F882B
:10799000B842FFF474AFC01B1FFA80FEBEF1300F77
:1079A0003FF676AFBEF12F0F7FF675AF302170E74F
:1079B000597840006178400034160020FE160020FF
:1079C0000080FFFF38160020FC160020280D002044
:1079D0002D45400041F74000F1774000F8B5084CD4
:1079E0004FF4804666630A20064DA8474027676328
:1079F0000A20A84727630A20A8472663F8BD00BFCE
:107A0000000E0E4035F24000F8B578B9114D4FF434
:107A100080736B630220104CA0474FF080736B6340
:107A20000420A04701220D4B5A63F8BD094E4FF4C4
:107A300080737363094F02253D632846064CA047B7
:107A400001233B630420A0474FF080733363284633
:107A5000A047F8BD000E0E4035F2400000100E4069
:107A600010B5084C4FF4804363630020064B9847E1
:107A70000220064B98470222054B5A63402363635A
:107A800010BD00BF000E0E40097A400035F24000E4
:107A900000100E400322014B1A60704730140E4054
:107AA000044B986801E0034B9868024B9B6898422E
:107AB000F9D1704730140E4010B584B001900C46D7
:107AC000064B98470390039B019A9B1AA34202D24C
:107AD000002004B010BD0120FBE700BFA17A4000E8
:107AE00030B585B01E4B1B68002B31D01D4B98471D
:107AF0004FF0FF311A4B18681B4B9847EFF3108378
:107B0000B3FA83F35B09039372B6BFF35F8F00226E
:107B1000164B1A70039D80230093154B15221421D8
:107B20001448154CA04704462DB101220F4B1A7082
:107B3000BFF35F8F62B600231A46194608480068F3
:107B40000E4DA8470E4B984744B1002005B030BDFC
:107B500001200C4B9847024B1860C7E70120F5E75E
:107B60002C0D0020ED6E400069EA40002F0300203C
:107B7000E0180020000A0E401100002075E74000C8
:107B8000056F4000ADE8400010B5074B9847002254
:107B900013210648064B98470446064B9847B4FA0B
:107BA00084F0400910BD00BFED6E4000000A0E4099
:107BB00051DA4000056F400038B5114B9847EFF39C
:107BC000108404B972B6002308E09A0002F580021E
:107BD0000C4951F82310116001339BB27F2BF4D96B
:107BE000002212210848094B9847C5B204B962B671
:107BF000074B98470DB1002038BD012038BD00BFAC
:107C0000ED6E4000E0180020000A0E4051DA4000FE
:107C1000056F400010B400240EE0400080F0070023
:107C2000C0B20133DBB2072B05D810F0800FF4D1BE
:107C30004000C0B2F5E70134944204D211F8013B90
:107C400058400023EFE75DF8044B704770B50646D7
:107C5000002501E02C44A5B2B5F5007F15D20E4BEE
:107C6000E918EA5CFF2A14D06B1C0B481B5C033339
:107C7000DCB2B242EED1621EFF20084B98472B19AE
:107C8000074A9B5C9842E5D101E04FF6FF75284614
:107C900070BD4FF6FF75FAE7E0180020157C400034
:107CA000DF18002008B5094B1B781BB1022B01D04F
:107CB000074808BD074B9847012804D10122034B10
:107CC0001A70034808BD002008BD00BF300D002019
:107CD000E0180020E17A400008B5094B1B781BB181
:107CE000022B01D0074808BD074B9847012804D153
:107CF0000122034B1A70034808BD002008BD00BFD5
:107D0000300D0020E0180020E17A4000A8B108B54D
:107D10000346B1F5007F12D28818B0F5007F01D973
:107D2000002008BD08461946064B1844064B9847E4
:107D30000222064B1A70012008BD00207047002067
:107D400008BD00BFE0180020611A4100300D00207E
:107D500008B5064B1B78022B01D0002008BD044B50
:107D600098470128FAD1034B984708BD300D0020F1
:107D7000897B4000B97B400090B110B50446026891
:107D8000094B9A4201D0002010BD9A220146FF20E3
:107D9000064B984794F89A30984203D0002010BDC3
:107DA00000207047012010BD5FE1AD5A157C4000F6
:107DB00010B50C46084B9847B0F5007F01D3002062
:107DC00010BD811C054B5A1C125C19442046044B03
:107DD0009847012010BD00BF4D7C4000E0180020F6
:107DE000611A410008B5044B9847B0F5007F01D2F5
:107DF000012008BD002008BD4D7C400008B5054BA2
:107E00009847B0F5007F02D2034BC05C08BD00204C
:107E100008BD00BF4D7C4000E1180020FF292FD095
:107E20002DE9F843D61CF6B28419B4F5007F03D9C6
:107E30004FF6FF70BDE8F88317460C460546022151
:107E4000114A1170DFF84C8000EB080900F8084077
:107E5000421C02F8087008443A46194640440B4B4D
:107E600098477C190234721E4946FF20084B9847F8
:107E700008F80400E81980B2033080B2BDE8F88346
:107E80004FF6FF70704700BF300D0020611A4100AF
:107E9000157C4000E018002010B5A8B0224B984790
:107EA0000446224B984708B928B010BD9B222146B2
:107EB00001A81F4B98474FF40072FF211D481E4B2D
:107EC000984702AB1022012100201C4CA0474FF61E
:107ED000FF73984203D026AB03220221A0474FF63E
:107EE000FF73984205D00DF19B0301220321134C2F
:107EF000A0474FF6FF73984204D027AB012204211C
:107F00000E4CA0474FF6FF73984205D00DF19D032C
:107F100001220521094CA0474FF6FF739842C3D0B8
:107F2000074B9847C0E700BFA57C4000797D400023
:107F3000611A4100E01800205D1C41001D7E4000D8
:107F4000517D4000044B1880044A1378591C11706D
:107F5000034A22F813007047E41C0020310D002072
:107F6000E41A002008B5194B1B8807EE903AF8EE8A
:107F7000677A9FED177A67EE877A164BC3ED007A22
:107F8000F7EE006A76EEE76A87EEA67ADFED126A10
:107F900067EE267A114BC3ED007A86EEA77A17EECC
:107FA000100A0F4B9847DFED0F7A07EE100A27EE05
:107FB000277ADFED0D7A77EEC77ADFED0C6A86EE71
:107FC000A77A0B4B83ED007A08BD00BFE41C0020AC
:107FD00001088039E01A002000401C46EC1C0020FB
:107FE000F50541003313954300F05745C47D7B49A7
:107FF000E81C0020BFF35F8F024B1868BFF35F8F50
:10800000704700BFE81C002068B90F4A1368B3F13D
:10801000FF3F0AD00320B3F1333F0ED013B95368AA
:1080200003B902207047094AF0E75168B1F1FF3FF8
:1080300001D00320EFE70020EDE75168B1F1333FB5
:10804000ECD10120EAE700BF00C0470000E0470094
:1080500018B101280FD0022070470B4841F6F87381
:1080600083B130B4C518C4588C4206D0083B002BED
:10807000F8D1012004E00548F0E76B6813600020A8
:1080800030BC70470120704700C0470000E0470047
:1080900070B505460020124CA04706460120A047B7
:1080A0001DB1012D12D0022070BD022803D0022E76
:1080B00007D0022070BD012E01D0012070BD00202C
:1080C00070BD012801D0002070BD70BD022E05D00A
:1080D000022801D0022070BD012070BD002070BDBB
:1080E00009804000F8B504460F461646450A094B7C
:1080F000984704F4FE7000F580031F605E602A4616
:1081000001210548054B98470446054B98472046F2
:10811000F8BD00BFED6E4000000A0E4051DA40008D
:10812000056F4000012909D002290CD1002108B5B2
:1081300038B906480A46064B984708BD4FF0333118
:10814000F5E70448F6E70120704700BF00C047008C
:10815000E580400000E0470038B518B101280DD097
:10816000022038BD0A4C0823B3F5005F0ED2E01898
:10817000E558B5F1FF3F03D00833F5E7054CF2E7CA
:10818000054B984708B1022038BD38BD012038BDE5
:1081900000C0470000E04700E580400010B568B12E
:1081A00040F2F234074B9847224607210648074B16
:1081B00098470446064B9847204610BD40F2E234EB
:1081C000F0E700BFED6E4000000A0E4051DA4000BB
:1081D000056F400070B582B000230193044668B972
:1081E0000125184E18490023B3F5006F28D251F825
:1081F0002320B2F1FF3F05D10133F5E70025134EEF
:108200001349F0E72046134B9847044610B1204627
:1082100002B070BD01AA314628460F4B984748B9B5
:10822000019A0132314628460C4B98470028EED07F
:108230000124ECE7012231462846084B9847F5E730
:108240000024E4E70120FFFF00C047000220FFFFF9
:1082500000E047009D81400051804000598140006E
:1082600070B582B005460E460846294B984701284E
:1082700006D001213046274B98470446002844D1B8
:10828000002400E00134244B1B689C4215D201AA53
:10829000224B53F824102846214B9847022833D00C
:1082A0000028EFD1019A1D4B53F8241030461D4B86
:1082B00098470028E6D0012427E028461A4B984723
:1082C000044610BB02213046124B98470446E0B9E1
:1082D00095B9164D02AA002342F8083D29463046BA
:1082E0000F4B984750B9009A0132294630460D4B42
:1082F000984750B1012408E00D4DEBE701222946D3
:108300003046084B9847F4E70124204602B070BD80
:108310000980400025814000200100200801002044
:1083200051804000598140009D8140000120FFFFA5
:108330000220FFFF10B50020104B9847044608B1FB
:10834000204610BD01200D4B984704460028F7D168
:1083500002210B4B984704460028F1D1012209491C
:10836000094B984708B10124EAE701220749064B67
:1083700098470028E4D00124E2E700BF9D81400037
:10838000258140000120FFFF598140000220FFFFAE
:1083900038B50120384B9847384B1860002869D011
:1083A0000020374DA84704460120A847012C2BD0B8
:1083B0005CB1022C46D0334B9847034618B90122D2
:1083C000314B1A700023184638BD012808D0022806
:1083D00014D100202D4B984703460028EFD0F2E738
:1083E00000202A4B984703460028ECD102210120A7
:1083F000274B984703460028E1D0E4E7214B9847F4
:1084000003460028DBD0DEE748B1022814D1002162
:108410000120204B984703460028D0D0D3E7012005
:108420001A4B984703460028CDD10221184B984794
:1084300003460028C3D0C6E7124B984703460028DE
:10844000BDD0C0E738B102280CD10E4B9847034687
:108450000028B4D0B7E701200C4B9847034600280A
:10846000ADD0B0E7012100200A4B98470346002811
:10847000A5D0A8E70123A6E7ADE84000F01C002046
:108480000980400035834000320D0020D581400036
:10849000258140006182400070B50E4B1B7813B9F6
:1084A0000324204670BD0D4604460B4E4FF0FF31AD
:1084B00030680A4B98470120094B98472A462146C5
:1084C000084B9847044600231A4619463068064D63
:1084D000A847E6E7320D0020F01C002069EA4000C2
:1084E000918040005180400075E74000F8B5194B7D
:1084F0001B7813B903242046F8BD0E4605464FF0FD
:10850000FF31154B1868154B98470020144B9847BE
:10851000074632462946134B98470446012807D0A0
:1085200000231A4619460C4800680F4DA847E2E799
:10853000B7FA87F46409214638460C4B984708B1CE
:108540000224EDE7324629462046064B984704466A
:10855000E6E700BF320D0020F01C002069EA400071
:10856000918040005981400075E7400061824000E1
:1085700008B50020094B984708B1012008BD20220A
:10858000074B5A630A20074B9847074B9847074BFE
:108590009847012801D0002008BD08BDE9654000CA
:1085A00000100E4035F240008D0541003965400055
:1085B00030B587B0174B984704468A238DF80830AA
:1085C0000025059501238DF809308DF80C300DF14B
:1085D00007030493104B98478DF80B5003238DF835
:1085E0000A30322202A920460C4B984720460C4BF9
:1085F0009847022806D0002520460A4B984728466F
:1086000007B030BD9DF80730092B01D00025F3E7F6
:108610000125F1E78D0541003D744000697440007B
:10862000997440005174400030B587B01A4B984798
:10863000044600220592A8238DF8083001238DF806
:1086400009308DF80B2001AA049202228DF80C202B
:108650008DF80A30114B9847322202A92046104B60
:10866000984720460F4B9847022806D00025204601
:108670000D4B9847284607B030BD9DF8043033B9FC
:108680009DF8053013F0F80F03D00025EFE7002523
:10869000EDE70125EBE700BF850541003D74400093
:1086A00069744000997440005174400008B5034B50
:1086B000984708B1002008BD012008BDA969400005
:1086C00030B587B0184B98470446002305937223B2
:1086D0008DF8083001238DF8093092228DF80B2097
:1086E0000DF1070204928DF80C3003238DF80A3047
:1086F0000E4B9847322202A920460D4B9847204640
:108700000C4B9847022806D0002520460A4B984774
:10871000284607B030BD9DF80730442B01D0002516
:10872000F3E70125F1E700BF8D0541003D744000EE
:1087300069744000997440005174400070B586B06F
:10874000002832D11C4B98470446002505959823F4
:108750008DF8083001268DF809608DF80A50022343
:108760008DF80C3001AB04938DF80B502046134B61
:10877000984736238DF804308DF80550322202A92F
:1087800020460F4DA8478DF80A60322202A92046E4
:10879000A84720460B4B984702280AD000252046C0
:1087A000094B9847284606B070BD084B98470446C9
:1087B000CBE73546F3E700BF850541003D74400037
:1087C0006974400099744000517440008D05410067
:1087D00038B50020064CA04705460120A047012DD2
:1087E00001D0002038BD0128FCD0002038BD00BFDA
:1087F0003D8740002DE9F0473D4BD3F858801920C4
:108800003C4B98474FF496703B4B9847002409E047
:108810003A4B98473A4B23F814000320364B9847BD
:108820000134E4B21F2CF3D9364B98478246002618
:108830003746354634463FE0314931F813100A4493
:108840000133DBB21F2BF7D94FEA5219B9F10A0FE6
:1088500017D92A4B9847631CDBB2294A22F8140027
:108860001F2B1DD81C46A9F1FA0398421AD309F10F
:10887000FA02904225D80135EDB2202D13D90126F8
:1088800011E0B8F1000F05D0194BC3F85880002053
:10889000BDE8F0870020174B98470020BDE8F0871F
:1088A0000024E0E700250320134B98474FF47A613A
:1088B0005046154B984707462FB926B900231A464C
:1088C000C0E70025EFE7B8F1000F07D0084BC3F869
:1088D000588057B936B10120BDE8F0870020054B1C
:1088E0009847F6E70020BDE8F0870020BDE8F08754
:1088F000000001400554400035F240005154400052
:10890000F41C0020A17A4000B97A4000004870476A
:10891000D0474100072070472DE9F84305460E4631
:1089200017460A469C211E4B98470446451B40B1FA
:10893000731B052B05D94378552B07D010237B706B
:1089400001E000237B702046BDE8F88390F80280A8
:10895000C37888EA0303FF2B02D011237B70F2E770
:1089600090F80490437909EB03291FFA89F9B9F1CA
:108970003A0F06D84D440635AE4205D200237B702F
:10898000E1E712237B70DEE74A46811D381D054B67
:108990009847A7F8029087F8008001237B70D2E700
:1089A00061194100611A410010B553889C1D8C4229
:1089B00019D83A2B01D9002010BD11469C23037011
:1089C00055234370137883701378DB43C370937817
:1089D000037153881B0A4371528804310630034BDC
:1089E0009847012010BD002010BD00BF611A410052
:1089F00070B582B004460378253B332B00F2198210
:108A0000DFE813F0450017021702170217023400BF
:108A1000170217021702170217021702170217028E
:108A2000170217021702170217021702170217027E
:108A30001702170217021702170217023E01170248
:108A40001702FA0017021702170217021702BA01DB
:108A500013015C0017021702170217021702170210
:108A6000170265017900CB00A600E3009C4C2A2385
:108A700023709C4DA84760809B4B98470646A847AB
:108A800002463146201D994B984702B070BD012027
:108A9000974B984780B2924B588010B945221A7074
:108AA000F3E794490120944B984718B125228C4B49
:108AB0001A70EAE745228A4B1A70E6E74388032BCF
:108AC00005D0874B00225A8045221A70DDE70379D2
:108AD0008DF8043043798DF8053083798DF80630B0
:108AE000864B984701A9864B98477D4B00225A80B8
:108AF00024221A70C9E74388012B05D0784B002245
:108B00005A8045221A70C0E703790F2B05D9744BA0
:108B100000225A8045221A70B7E77A4B9847704A6C
:108B20005523137020235380237900EB43100668EC
:108B300045688468C16856609560D46011610669B3
:108B400045698469C16956619561D46111629CE788
:108B50004388212B05D0624B00225A8045221A708F
:108B600093E701790F2905D95D4B00225A804522F0
:108B70001A708AE7202249010530634B9847012883
:108B800005D0574B00225A8045221A707DE7544B7E
:108B900000225A8024221A7077E743882BB1504B69
:108BA00000225A8045221A706FE7584B98470128D7
:108BB00005D04B4B00225A8045221A7065E7484B7E
:108BC00000225A8024221A705FE743882BB1444B5D
:108BD00000225A8045221A7057E74D4B984728B912
:108BE0003F4B00225A8024221A704EE73C4B002251
:108BF0005A8045221A7048E74388012B05D0384B2C
:108C000000225A8045221A703FE70079414B98476D
:108C100028B9334B00225A8024221A7035E7304B92
:108C200000225A8045221A702FE74388082B05D06E
:108C30002B4B00225A8045221A7026E7037942798D
:108C400003EB0223827903EB0243C079217A627A33
:108C500001EB0221A27A01EB0241E47A01AA01EBC5
:108C6000046103EB00602C4B984700287FF40DAFA4
:108C70001B4B019A5A604B221A7004225A8004E757
:108C80004388063B9BB21F2B05D9154B00225A8007
:108C900045221A70F9E64379807903EB0023E079E5
:108CA00003EB0043207A04F10902217903EB006011
:108CB0001A4B984728B90A4B00225A8024221A706E
:108CC000E3E6074B00225A8045221A70DDE643880E
:108CD00033B3034B00225A8045221A70D5E600BFF9
:108CE000341D0020158940000D894000611A4100A3
:108CF000FD7D4000381D0020B17D40008D05410004
:108D0000A1634000D97C40000D7D4000517D4000B2
:108D1000A9694000516C4000ED6B4000356C40008B
:108D20000020474B1871474B984720B1444A1379AC
:108D300043F0010313710120424B984720B1404A90
:108D4000137943F00203137102203E4B984720B180
:108D50003B4A137943F0040313710320394B9847BE
:108D600020B1374A137943F008031371344B0122C1
:108D70005A8054221A7088E64388012B05D0304B64
:108D800000225A8045221A707FE60379463B102B59
:108D900049D8DFE803F03F480948484812484836B8
:108DA0002D48481B48482400274B9847244B1871EE
:108DB0004A221A7001225A8067E6244B9847204BBA
:108DC00018714A221A7001225A805EE6204B984799
:108DD0001B4B18714A221A7001225A8055E61D4B0E
:108DE0009847174B18714A221A7001225A804CE694
:108DF000194B9847124B18714A221A7001225A8057
:108E000043E6164B98470E4B18714A221A700122FE
:108E10005A803AE6124B9847094B18714A221A7049
:108E200001225A8031E6064B45221A7000225A80F0
:108E30002BE6034B00225A8045221A7025E600BF1C
:108E4000341D0020B56C400071854000B1854000A4
:108E500029864000AD864000C1864000D187400091
:108E6000F587400000487047341D0020F0B583B0FE
:108E7000EFF31083B3FA83F35B09019372B6BFF388
:108E80005F8F0022364B1A70019E364B1B68364AA4
:108E900015682B447F2B2AD8324B1C682246334955
:108EA00033482844334B98472C442F4B1C600022F6
:108EB0002C4B1A602EB10122294B1A70BFF35F8F21
:108EC00062B62D4A284B196829482C4B9847014611
:108ED000D0B1274BC31A284842881A44951D4478BC
:108EE000012C15D044BB802B1CD900242AE01D4A3C
:108EF000136814682C441B1B03F18004204A137868
:108F000043F001031370C9E70024174B1C6019E0FC
:108F10001748154F3E68761B32464119194B984742
:108F20003E600FE0104D2C68E41A22461048154BA5
:108F300098472C60002405E00133802B05D90024DC
:108F4000094B1C60204603B0F0BD0948064D2C6853
:108F5000E41A2246C1180B4B98472C600024F1E715
:108F60002F0300207C2000208C200020D420002013
:108F70007C1F0020611A41009020002019894000C8
:108F800088200020951B410010B50DE0144B195DA1
:108F90001448154B98470134E4B2144B1B689C42AB
:108FA000F4D30022114B1A600120114B9847114B4A
:108FB00098470128F8D11048104B9847104B984714
:108FC0000246802106480F4B98470128ECD10C4BF4
:108FD000984743880633054A13600024DDE700BF45
:108FE000FC1F002000820140DBDE400084200020C6
:108FF00035F240006D8E400090200020F189400045
:10900000658E4000A989400030B583B08024224697
:1090100000211C481C4DA847224600211B48A84798
:1090200000231B4A13601B4A13601B4A13701B4A20
:1090300010215166C2F8901051655162C2F880103B
:10904000116F21F010011167516F21F0100151676C
:10905000134A4FF400211160202182F813130121DB
:10906000104A9160104A0192009322460F4910481D
:10907000104CA047012802D00F48104B984703B06E
:1090800030BD00BFD42000205D1C4100FC1F00202B
:109090007C2000208420002088200020000E0E402C
:1090A00000E100E00082014080200020D84741001C
:1090B000898F400061EF4000E0474100B513410057
:1090C000104B1B6913F0010F12D00E4B5B6913F0AC
:1090D000010F0DD00C4B1B687F2B0AD90B4A13785C
:1090E00043F001031370074B9A69094B83F87F2003
:1090F0007047054A1368591C1160024A9169044A75
:10910000D1547047008201407C200020882000203C
:10911000D4200020064A936823F07F4323F4706331
:1091200043F0254343F4E0639360024B13607047C0
:1091300000140E40080000A570B506460D46094B08
:1091400098470446002040B929462046064B9847D8
:1091500028B93046054B9847F5E7012070BD00203F
:1091600070BD00BFA17A4000B97A4000E5B0400070
:1091700010B54FF47A722B4B1A8004E04022002184
:1091800029482A4B9847274B188880B2284B984784
:10919000254C2323237014236370264B9847C0F378
:1091A0000F23A370E070244B9847C0F30F23237163
:1091B0006071224B9847C0F30F23A371E071204BDD
:1091C0009847C0F30F23237260721E4B9847C4F870
:1091D0000A001D4B1B7807EE103AB8EE477A9FED58
:1091E0001B6A27EE067ADFED1A6A37EE667A17EE0B
:1091F000103AC4F80E30174B1B7807EE903AF8EE91
:10920000677A67EE867A77EEE67A17EE903AC4F8D8
:109210001230114B98470028B0D0322120460F4B16
:109220009847ABE7C8210020782100205D1C410051
:1092300035F2400051544000F55B4000796E40002B
:10924000856E4000F57F4000F8010020B4C8363F2D
:109250006FDB4A42F9010020AF054100399140001F
:10926000F0B583B0402200219A489B4B98470BE20F
:109270009A4B98479A4B984711E2984B9847994BCD
:10928000BB221A601A225A60954B98470AE291490C
:109290000B462A2203F8012B934A1068C1F80100FB
:1092A00091889279104699809A71FEE101208F4B46
:1092B000984728B9874B45221A7002225A70F7E165
:1092C0008449252301F8013B0120894B9847EFE1B0
:1092D0000820864B984728B97E4B45221A700222F7
:1092E0005A70E8E17B49262301F8013B0820804BB6
:1092F0009847E0E109207D4B984728B9754B4522F6
:109300001A7002225A70D9E172497E2301F8013B9A
:109310000920774B9847D1E1C4F30723032B09D8E1
:10932000DFE803F0020B0406724807E0724805E02C
:10933000724803E04FF0FF3000E07148B0F1FF3FAA
:1093400010D001A96F4B984730B9624B5A221A705E
:10935000019AC3F80120B5E15E4B45221A70022242
:109360005A70AFE15B4B45221A7001225A70A9E195
:10937000C4F30723032B09D8DFE803F0020B04062C
:109380005C4807E05C4805E05C4803E04FF0FF30D4
:1093900000E05B48B0F1FF3F0ED05B4B19685B4BC0
:1093A000984718B924224B4B1A708EE1494B45223D
:1093B0001A7003225A7088E1464B45221A70012226
:1093C0005A7082E12422434B1A7081E1414B4522BD
:1093D0001A704F4A12785A707DE14E4B1B780F2B52
:1093E00005D93C4B45221A7001225A7076E14A4B4E
:1093F0009847384A5523137020235370454B1B78E8
:1094000000EB4310D0F800E047688668C168C2F8F6
:1094100002E0C2F80670C2F80A60C2F80E10D0F876
:1094200010E047698669C169C2F812E0C2F8167097
:10943000C2F81A60C2F81E1050E1264B4B221A7077
:1094400004225A706A44354B1968354B1868354BFD
:10945000984720B91F4B019AC3F8022041E100222E
:10946000314B1A603DE11B4B54221A70002058709A
:109470002E4B984720B1174A537843F0010353709D
:1094800001202A4B984720B1124A537843F0020337
:1094900053700220254B984720B10E4A537843F071
:1094A000040353700320214B9847002800F01C81CF
:1094B000084A537843F00803537015E11C4B1878A1
:1094C000072837D9802841D0024B45221A70012243
:1094D0005A700CE1D02100205D1C410009054100BB
:1094E0001591400090140E4090444100FD7D4000D5
:1094F000B17D40000110FFFF0310FFFF0410FFFFCC
:109500000210FFFF99844000C4210020ED84400038
:10951000CA210020C0210020D97C4000CC2100209D
:10952000BC210020ED6B4000D2210020B56C400032
:10953000542100207C4B984718B924227B4B1A7089
:10954000D5E07A4A452111705070D0E0784B1878F8
:1095500010F0800FB8D1774B984718B92422734B7D
:109560001A70C4E0714B452119705870BFE0724AFF
:10957000724B1968724B1868724B984718B92422BD
:109580006A4B1A70B6E0694B452119705870B1E00A
:1095900066484E2300F8013B6B4B9847002800F0CB
:1095A000AC806A4B4FF020321A605A609A60C3F860
:1095B0000B20A2E014F47F4F5C4E31464FF05E0367
:1095C00001F8023B14BF01200020614B98477070E6
:1095D000002840F095804522327091E04A22534B9A
:1095E0001A70C4F30723463B102B2DD8DFE803F095
:1095F000272C092C2C2C0E2C2C221D2C2C132C2C23
:109600001800544B9847494B58707CE0524B984790
:10961000464B587077E0514B9847444B587072E076
:109620004F4B9847414B58706DE04E4B98473F4B1E
:10963000587068E04C4B98473C4B587063E04B4B7C
:1096400098473A4B58705EE0384B45221A70012219
:109650005A7058E0464B98472422344B1A7054E015
:109660009A000232434951F82300304950500133E7
:10967000DBB20B2BF4D9404B984700284ED1402247
:1096800000212A483D4B98474FF0FF3101203C4BC9
:10969000984704460028F7D043283FF4E9AD422C10
:1096A0003FF4EBAD2A2C3FF4F2AD252C3FF4FEAD98
:1096B000262C3FF40DAE7E2C3FF41CAEE5B25A2DA5
:1096C0003FF42AAE7A2D3FF453AE242C3FF47AAE09
:1096D000452C3FF47BAE552C3FF47FAE4B2C3FF432
:1096E000ACAE542C3FF4BFAE442C3FF4E7AE412C5B
:1096F0003FF43DAF4E2C3FF44BAF5E2D3FF45AAFDD
:109700004A2D3FF46BAF3D2CA4D0732CB3D1074B43
:1097100073221A7030225A700023AAE732210348BC
:10972000184B9847ABE700BF516C4000D021002098
:10973000B8210020816C400058210020CC2100205D
:10974000BC210020356C40003D6D4000D12100203F
:109750005159400071854000B18540002986400084
:10976000AD864000C1864000D1874000F5874000AB
:1097700099A84000B4230020AF0541005D1C4100C2
:1097800041F740003991400010B500230322014603
:1097900002480068024CA04710BD00BF340D0020F5
:1097A00069F8400010B584B0002304AA42F8043DD3
:1097B00009490C680092032201462046074CA04745
:1097C000039B3BB14FF08052054B1A60BFF34F8FA4
:1097D000BFF36F8F04B010BD340D002015F94000A9
:1097E00004ED00E010B582B00F4B0193012300930C
:1097F000002380220D490E480E4CA047012802D0BC
:109800000D480E4B984700230193012200928022BD
:109810000B490C48074CA047012802D00A48074BC7
:10982000984702B010BD00BF340D00200048410031
:109830006192400061EF400010484100B5134100C3
:1098400040484100719140004C48410070B584B0DF
:10985000044603782A2B00F095802378252B00F00E
:1098600095802378262B00F0958023787E2B00F0BE
:10987000958023785A2B00F0958023787A2B00F07E
:1098800098802378532B00F0A7802378472B00F093
:10989000B0802378672B00F0BD802378462B00F042
:1098A000C4802378522B00F0C7802378502B00F01F
:1098B000D78023785E2B00F0FB802378492B00F0C3
:1098C00008812378432B00F017812378422B00F086
:1098D00017812378552B00F017812378572B00F040
:1098E0001A812378562B00F0298123784C2B00F025
:1098F000328123784D2B00F0428123784B2B00F0EE
:1099000087812378542B00F09F812378442B00F02B
:109910009F812378412B00F0B2812378592B00F0EE
:10992000D08123784E2B00F0E58123784A2B00F07C
:10993000E5812378402B00F0E78123786F2B00F03E
:10994000FC812378642B00F00A822378702B00F0CE
:10995000288223785B2B00F03D8223783D2B00F09A
:109960003F822378732B00F03F8225782C2D00F066
:109970003F822E2D00F0458223783E2B00F053824B
:1099800004B070BD2A20934B984766E72520914B81
:10999000984766E726208F4B984766E77E208D4BD9
:1099A000984766E76078000240F05A00894B984774
:1099B00063E7A378E27803EB0223227903EB024307
:1099C000627903EB0263844A13606078000240F01E
:1099D0007A00804B984754E7637833B901207F4B76
:1099E000984724207B4B98474FE700207B4B9847B4
:1099F000F7E76378A07800EB032080B210F4004F03
:109A000005D1774B98472420724B984741E747F69A
:109A1000FF70F6E76378A07800EB032000B2714B8B
:109A2000984724206B4B984737E760786E4B9847F0
:109A30002420684B984734E76278A37803EB02232D
:109A40009BB2092B05D9694A13802420614B9847A2
:109A50002BE70122664B1A7045205E4B984724E79E
:109A600063785BB1012B16D00022624B1A70012281
:109A70005F4B1A704520574B98471AE702205E4B00
:109A8000984730B904225A4B1A704520514B9847D9
:109A90000FE72420FAE70120574B984720B904220A
:109AA000534B1A70452000E024204A4B984700E7AA
:109AB00063782BB1012B07D04520464B9847FCE635
:109AC0005E20444B9847F8E64FF4AF70414B9847FF
:109AD000F3E66278A37803EB0223484A138005205B
:109AE000454B984720B90422414B1A70452000E0AD
:109AF0002420384B9847E4E64320364B9847E4E669
:109B00004220344B9847E4E662783D4B1A7055206A
:109B1000304B9847E1E661780F2908D820224901A7
:109B2000A01C384B984724202A4B9847D9E601229D
:109B30002F4B1A704520274B9847D2E608202E4B12
:109B4000984720B904222A4B1A70452000E02420AF
:109B5000204B9847C9E62C4B62781A70A2785A704D
:109B6000E2789A700720244B984720B90422204BB2
:109B70001A70452000E02420164B9847B9E6234B85
:109B800098476378003318BF01230370A3784370AC
:109B9000E378003318BF012383702379C37063799E
:109BA0000371A3794371E3798371237AC371637A73
:109BB0000372A37A4372E37A837209200E4B9847AB
:109BC00020B904220A4B1A70452000E02420014BE2
:109BD000984792E6A5974000C42100204D784000A8
:109BE000157840004178400005544000C82100200D
:109BF000CA2100207B22002095AF40009622002041
:109C0000C02100200D7D400078220020015C400032
:109C10006378A27803EB0223E27803EB0243227914
:109C200003EB02638F4A13606379A27903EB02238B
:109C3000E27903EB0243227A03EB02638A4A136060
:109C40004B208A4B98475CE65420884B98475CE64B
:109C500009228749E01C874B984748B96278864BB0
:109C60001A70A278854B1A704420804B984750E6B2
:109C70000122834B1A7045207C4B984749E6627855
:109C8000531EDBB21F2B06D901227D4B1A704520D3
:109C9000764B984741E6744B1A60A378E17803EB62
:109CA0000123217903EB0143617903EB01636D49E2
:109CB0000B60A11D7348744B984741206B4B98472C
:109CC0002BE6002604AD45F8046D704B98470095CF
:109CD0003346012204216E4DA847039B002B3FF41D
:109CE00020AE4FF080526B4B1A60BFF34F8FBFF323
:109CF0006F8F16E64E205D4B984716E6607800029F
:109D00004A305A4B984714E66078634B98475F4B4C
:109D1000984703AB00930023012204215C4DA84720
:109D2000039B002B3FF409AE4FF08052594B1A6051
:109D3000BFF34F8FBFF36F8FFFE5E21C6178A07810
:109D4000564B98470620564B984720B904224C4B57
:109D50001A70452000E02420444B9847F1E56078D4
:109D6000504B9847012803D04520404B9847ECE5DD
:109D700024203E4B9847454B984703AB0093002364
:109D800001220421424DA847039B002B3FF4DDAD87
:109D90004FF080523F4B1A60BFF34F8FBFF36F8F6E
:109DA000D3E5414B9847394B984703AB00930023C9
:109DB00001220821364DA847039B3BB14FF080524A
:109DC000344B1A60BFF34F8FBFF36F8F2420274BA4
:109DD0009847BEE5354B98472420244B9847BCE56F
:109DE0003D20224B9847BCE57320204B9847BCE5AB
:109DF00008222F49601C1F4B984700287FF4B9ADFB
:109E0000FFDE08222A49601C1A4B984700287FF47D
:109E1000B3AD284B4FF400421A60402183F80F1372
:109E2000C3F80021A8E508222149601C114B98477E
:109E300000287FF4A5AD154B984703AB0093002392
:109E400001224FF48011124CA047039B002B3FF4DA
:109E500097AD4FF080520F4B1A60BFF34F8FBFF397
:109E60006F8F8DE5BC210020CC210020A5974000FC
:109E700078484100011A410054210020B8210020F7
:109E8000CA21002058210020611A4100D1A04000C1
:109E900015F9400004ED00E035A140008DAE400012
:109EA00095AF400081A14000B5A84000C5A8400082
:109EB0008448410000E100E08388B3F59F5F0DD046
:109EC000B3F5706F25D0B3F5206F2FD0B3F5A05F39
:109ED00038D0B3F5706F41D000207047C288B2F51A
:109EE0001F6FEDD14189A1F5E752093A92B2C62A16
:109EF00045D9A1F5DD521D3A92B2C62A01D80220F9
:109F00007047A1F5B8510D3989B2C629D8D80620B5
:109F10007047C288B2F5F06FD5D14289A2F50B52D5
:109F2000053A92B2C62ACED803207047C288B2F54D
:109F3000206FCBD14289A2F6553292B2C62AC5D83B
:109F400005207047C288B2F5206FC2D14289A2F6BF
:109F5000553292B2C62ABCD805207047C388B3F5E3
:109F6000F06F01D0002070474389A3F5B8530D3B33
:109F70009BB2C62B01D804207047002070470120F7
:109F80007047000000B9704710B504460120034B2C
:109F90009847601EFFF7F6FF10BD00BF35F2400086
:109FA00038B50125044B1D7000210846034CA0471D
:109FB00000212846A04738BD390D002091584000A7
:109FC00010B50024022C09D80B4B1A780021084642
:109FD0000A4B9847012801D00134F3E70024022CF2
:109FE00009D8054B1A7800210120044B9847012815
:109FF00001D00134F3E710BD3A0D00208557400031
:10A0000038B51A4B1B786BB90024022C1FD8184B9B
:10A010001A78184B19880020174B9847012816D03A
:10A020000134F2E701210020144CA0470121084629
:10A03000A0471420124CA0470020124DA847012031
:10A04000A8471420A0470022084B1A70DCE7002420
:10A05000022C0AD8064B1A78064B19880120064BA9
:10A060009847012801D00134F2E738BD390D0020AE
:10A070003A0D00202C0100208557400091584000E7
:10A0800035F24000B5584000F8B505460E460024AC
:10A09000204601E00134A4B22746B4EB960F14D257
:10A0A00015F8241005EB84035A7801EB02219A7805
:10A0B00001EB0241DB7801EB03610028EAD107F5EF
:10A0C00040608000014B9847E4E7F8BD75694000A7
:10A0D000014B1868704700BF400D0020014B1878F5
:10A0E000704700BF3D0D002010B582B0084B0193B2
:10A0F000002300934FF4807206490748074CA0479D
:10A10000012802D00648074B984702B010BD00BF97
:10A11000400D0020904F4100CDA1400061EF400074
:10A120009C4F4100B5134100014B1878704700BFA8
:10A13000380D002001280CD038B102280DD0FF289E
:10A140000FD00A4A0A4B1A6070470A4A084B1A6035
:10A150007047094A064B1A607047084A044B1A6058
:10A160007047024A024B1A60704700BF904E410090
:10A1700028010020904A4100904841009049410048
:10A18000032817D8DFE800F002070C110A4A0B4B2E
:10A190001A60012070470A4A084B1A600120704774
:10A1A000084A064B1A6001207047074A034B1A60A1
:10A1B0000120704700207047904E41002801002088
:10A1C000904D4100904C4100904B4100F0B585B05E
:10A1D00001238DF80B307D4B009300231A467C49F8
:10A1E0007C487D4CA0477D4B186004A9502301F8A2
:10A1F000063D03207A4CA04704A9002301F8073D3F
:10A200000D20A04710B9002303930BE09DF809002F
:10A21000744B9847F7E74FF0FF3303AA0021084635
:10A22000714CA047039B13F0010FF4D040F21310C0
:10A230006E4B98476E4B98474FF480716D4B186882
:10A240006D4B984706E04FF0FF3303AA0021084604
:10A25000654CA047039B13F0020FF4D01920634B09
:10A260009847664B4FF480721A63DB6B13F4004F10
:10A2700019D0634B98470F20624B984701465F48BF
:10A28000614B98470022614B1A700DF10B010420BD
:10A29000534B984728B19DF80B3083F001038DF89C
:10A2A0000B30002403E05A4B9847E4E700241420C5
:10A2B0004E4B9847002303AA1C2118464A4DA84735
:10A2C000039B13F0080F00D0012413F0100F40F08F
:10A2D000BD80039B13F0040F32D04C4B1B78002B36
:10A2E00040F005810F20474B984701464348494BB2
:10A2F0009847474B9847484B98473D4B98473D4DAB
:10A300004FF4807128683C4B98472B68434A93422E
:10A3100000F0F980424A934200F0F580374BDB6B46
:10A3200013F4004F00F0F280354B98470F20354B67
:10A33000984701463148344B98472420394B984779
:10A34000039B13F4801F40F0E480304B1B78002BFC
:10A3500040F0E380344B9847002840F0028100220F
:10A360002A4B1A709DF80B3093B1304B1B787BB1A0
:10A370002F4B1B78002B00F024822E4B984738B9C6
:10A3800000222B4B1A702C4B9847002840F0078274
:10A39000002C8CD0264B1D78002D87D11B4B1C78B0
:10A3A000002C84D00122254B1A70254B98470B4B6B
:10A3B00018680A23009300231A460321214CA04762
:10A3C0000022214B1A702C4671E700BFA19F40006C
:10A3D000E0930400C44F4100FDFB40001022002028
:10A3E000B17D400081A14000C5F7400035F240003A
:10A3F000D16840002801002089A04000000E0E40D6
:10A40000E1544000CFD84000ABD840003D0D0020C3
:10A41000BD544000AFD840000D694000904A410053
:10A420009048410089974000DD054100240100204B
:10A430002E010020E95B4000DDA04000380D002027
:10A4400001A0400039FC4000390D00200F20934B43
:10A450009847934E01463046924B9847924B984707
:10A460004FF4804777630A20904DA847904B984758
:10A470004FF4FA70A8478F4B9847776301208E4BB3
:10A4800098471920A8474FF48073336300208B4E00
:10A49000B0470120B04700210846894EB04700214F
:10A4A0000120B04701210020864EB0470121084617
:10A4B000B0471420A8470020834EB0470120B04782
:10A4C0000127824B1F70824B98479DF80A1000238A
:10A4D000032241F480717F4EB0477F4B98470023A1
:10A4E0003A460221B0474FF0FF30A847F1E600227C
:10A4F000764B1A706A4D4FF480766E6319206B4B61
:10A5000098472E63EEE6754B984707E7664B9847EA
:10A510000CE74020724B984717E7724B984720B1E1
:10A52000714B984700287FF415AF0025674B1D70CD
:10A530006E4B1D70664B98472B4603224FF480717B
:10A54000644EB047644B98472B4601220421B04724
:10A55000534D4FF480766E631920544B98472E6309
:10A56000F8E6614B984700283FF4F9AE574B1B784B
:10A57000002B7FF4F7AE00205D4EB0475D4D287094
:10A580000120B0475C4B18702B78002B3FF4EAAEEB
:10A5900000283FF4E7AE01224C4B1A70574D284675
:10A5A000574B98472846574B98470746052816D0DB
:10A5B0000022554B1A704FF4FA703C4B984700201C
:10A5C0004B4EB0474B4D28700120B0474A4B187096
:10A5D0002B7803B138B900223C4B1A70C2E6012235
:10A5E000494B1A70E7E73A4B98479DF80A10002349
:10A5F000032241F48071374DA847374B9847002319
:10A6000001220221A84739460020404DA84739467B
:10A610000120A8470A203E4B9847D8B93D4D00215C
:10A6200028463D4B98472B78112B18D0002108461F
:10A63000234DA84700210120A8470025022D20D83E
:10A64000314B1A7800210846344B9847012818D01E
:10A650000135F3E732490A20324B9847DEE76B7841
:10A66000002BE3D1AB78002BE0D1EB78892BDDD147
:10A670002E46294600202C4DA84731460120A847E8
:10A68000D4E70025022D51D81F4B1A780021012054
:10A69000224B9847012849D00135F3E7CFD8400035
:10A6A000000E0E40AFD84000BD54400035F24000CF
:10A6B000617A4000DD794000097A4000695A400023
:10A6C0006D58400091584000B55840003D0D0020A5
:10A6D000EDAF400069F84000F9AF4000B56B4000B5
:10A6E000859F4000DD054100E9054100380D00204F
:10A6F0006D6A40003B0D00203C0D00206C220020C4
:10A70000A96A4000B99E40003A0D002099594000C6
:10A71000FD7D400014220020C5694000855740009F
:10A720002C010020B17D400085594000012100200E
:10A73000334DA84701210846A8471420314B9847BC
:10A740000020314DA8470120A8479DF80B3003B3E6
:10A750002E4B9847E8B12E4B1B78D3B12D4B1B786D
:10A760002BB101222C4B1A702C4B9847FAE500258F
:10A77000294B1D702A4B98472A4B1E682A4B984735
:10A780000A2300932B46024601213046274DA84755
:10A79000E8E50122204B1A70204B9847E2E500259E
:10A7A0001D4B1D701E4B98471E4B1E681E4B984735
:10A7B0000A2300932B460246012130461B4DA84731
:10A7C000E6E51B4B984700283FF4E2AD0122114B10
:10A7D0001A70184B984700283FF4DAAD01220E4B4F
:10A7E0001A700E4B98470F4B18680A2300930023EA
:10A7F0001A4603210D4DA84700220F4B1A70C7E5DA
:10A800009158400035F24000B55840003D5B400093
:10A81000240100202E010020380D002001A040005E
:10A82000C19F4000102200205DF0400039FC400034
:10A83000E95B4000DDA04000390D0020124A108085
:10A84000124A12787AB138B504460025022D0CD888
:10A850000F4B1A78214600200E4B984703460128DB
:10A8600003D00135F2E70120704718460025022D7C
:10A8700009D8074B1A7821460120064B9847012832
:10A8800001D00135F3E738BD2C010020380D002040
:10A890003A0D00208557400010B5044B984700231F
:10A8A00003221021024CA047012010BDD1A040007E
:10A8B00069F840000022024B1A700120704700BF67
:10A8C000240100200120014B187070472401002052
:10A8D00038B50024204609E000F47F43B3F5007F3B
:10A8E0000CD000F47F43B3F5807F0CD00028F3D167
:10A8F0004FF0FF310120134B9847EDE70020124B3A
:10A9000098470020EDE7C5B2002008E00134A4B26A
:10A9100020460D4B98470A2101200A4B984758B909
:10A92000AC42F3D308E0013CA4B22046064B984762
:10A930000A210120034B98470028D7D1AC42F2D816
:10A94000D4E700BF41F7400005544000F0B583B0A4
:10A950000224002010F0010F0AD14FF0FF31012036
:10A96000314B984700F00E03042BF3D10424F1E798
:10A970002E4B1B68ADF804301B0C8DF8063001A976
:10A9800002202B4B9847042C07D02A4B984701A94B
:10A99000294B984700252E4607E0264B9847002173
:10A9A000264B9847F1E72E460225322101201E4B07
:10A9B000984700F00E00042812D0022814D0042C6E
:10A9C000F3D1C5B1022D22D0032DEED10136F6B25E
:10A9D000182EEAD900252E46E7E703250026E4E7EE
:10A9E00000252E460424E8E7124B98478021134B9C
:10A9F00098470224E3E70F4B9847771CFFB2104BB0
:10AA0000995D0E4B9847632FCDD83E46CDE7094B55
:10AA10009847771CFFB20B4B995D084B9847632F03
:10AA2000DBD83E46C1E700BF41F74000D84F4100A8
:10AA3000B17D40008D054100A1634000516340009D
:10AA4000940100203001002008B5044B9847642091
:10AA5000034B9847034B9847F7E700BF316E400020
:10AA600035F24000657F400070B582B0944B984746
:10AA7000944B98470120944B984702A9002301F872
:10AA8000013D0520914B984728B19DF8073013B13F
:10AA900000208D4B98478E4B98478E4B98478E4A97
:10AAA0008E4B1A6001208E4B9847044690B98A4D10
:10AAB0008C4C0FCC28606960AA60EB608A4B984789
:10AAC0008A4B984702228A4B1A638A4B984705465D
:10AAD000002416E0814B196801207C4B984705E063
:10AAE0007E4B1B6800221A550134E4B20F2CF7D9B3
:10AAF000E4E70520804B98477E4B98470546013494
:10AB0000E4B20DB9132CF4D97C4B984729467C4B01
:10AB100098477C4B98477C4DA8470023012211465B
:10AB20007A4CA04701207A4B9847A847002301227E
:10AB30000221A047774B98476B4B9847764B984735
:10AB400000230122052175480068A04700252C46F6
:10AB500080E01146002341F8043B7148714B98474F
:10AB600038B9714B5968013159606D486F4B98473E
:10AB70007BE001216A486D4B984776E0114600233F
:10AB800041F8043B6A48674B984798B9694B596844
:10AB9000013159606648654B984767496748614B82
:10ABA000984760B9634B59680131596063485F4BFE
:10ABB000984768E001215E485C4B9847EDE701212A
:10ABC0005E485A4B98475EE0134600221A605A6866
:10ABD00001325A6069465A48524B984750B9594B0E
:10ABE0005968009B994201D8002514E054484F4B06
:10ABF0009847F9E7534B596851484C4B9847F3E74E
:10AC0000514A136801331360052B44D94D4B00257D
:10AC10001D605D6015604D4BA3FB0423DB0803EB57
:10AC200083035A00944238D0494B9847002840F09B
:10AC30009D80484BA3FB04235B09642202FB134362
:10AC4000002B00F096800A202B4B98470134632C90
:10AC500000D900240135B5F57A7FDCD3324A136878
:10AC6000013313603B2B3FF674AF3B4B98470028F2
:10AC7000C6D00022344B1A602E4A13680133136089
:10AC80003B2B3FF67BAF2F4A1368013313603B2BFE
:10AC90009AD80025BFE70025BDE7304B984728B973
:10ACA00047232F4A13702F4A1370BDE700202E4E02
:10ACB000B0472B4B18700120B0472A4B1870B3E7F0
:10ACC00091834000997E4000B1544000B17D400026
:10ACD000BD544000F95240009C2200207C220020FC
:10ACE000FD7D4000905041008D05410039654000D8
:10ACF000000E0E40916E400035F240008505410087
:10AD000001664000DD794000D1A0400069F84000B4
:10AD1000097A4000795A40008D624000680D002099
:10AD20000110FFFF99844000580D0020ED84400081
:10AD30000210FFFF480D00204C0D00200410FFFF03
:10AD40000310FFFF500D0020440D0020CDCCCCCCD3
:10AD50003D5B40001F85EB5129A14000DDA0400074
:10AD6000F8010020F90100200D594000024B9847DE
:10AD700069E7024B984766E7495B4000795A400013
:10AD800008B509E000210846314CA0470021012008
:10AD9000A04700222F4B1A704FF0FF3101202E4B9D
:10ADA00098472C4B1B78013B082BF2D801A252F894
:10ADB00023F000BFD9AD400085AD4000F3AD4000A9
:10ADC00003AE4000E9AD40003BAE400023AE400082
:10ADD0002FAE400035AE4000012100201C4CA047A2
:10ADE00001210846A047D4E71C4B18881C4B984704
:10ADF000CFE7002108461B4CA04700210120A047B7
:10AE0000C7E701210020174CA04701210846A047B1
:10AE10001420154B98470020144CA0470120A04750
:10AE2000B7E7134B98471349134B9847B1E7134BB8
:10AE30009847AEE7124B9847ABE7124AD01E13462D
:10AE400012F8032C817840780F4CA047A1E700BF8F
:10AE5000ED5840007B22002041F740009622002060
:10AE60003DA840009158400035F24000B5584000E0
:10AE70008D05410078220020A1634000517D4000F3
:10AE80000D5C4000AF220020FD55400010B5144677
:10AE9000044B1870597002462146981C024B984783
:10AEA00010BD00BFAC220020611A410010B582B075
:10AEB000234B01930323009300238022214922483E
:10AEC000224CA047012802D02148224B9847224B10
:10AED0000193002300938022204921481B4CA04766
:10AEE000012802D01F481B4B984700230193009371
:10AEF00080221D491D48154CA047012802D01C483E
:10AF0000144B98471B4B01930023009380221A494E
:10AF10001A480E4CA047012802D019480D4B9847FB
:10AF2000184B019300230093802217491748074CC0
:10AF3000A047012802D01648064B984702B010BD22
:10AF4000640D0020DC4F410081AD400061EF400006
:10AF5000E04F4100B51341006C0D0020FC4F410053
:10AF600069AA4000085041003050410049AA400001
:10AF700034504100680D0020505041004DA9400060
:10AF800054504100600D002070504100D1A8400095
:10AF90007450410010B584B0104B18700022039219
:10AFA00004AB43F8082D0E4A106803AA009204224D
:10AFB00001210C4CA047029B5BB9039B63B14FF08E
:10AFC0008052094B1A60BFF34F8FBFF36F8F012080
:10AFD00000E0002004B010BD0120FBE77B22002030
:10AFE000640D002015F9400004ED00E0014B1868E5
:10AFF000704700BF600D0020014B1868704700BF0C
:10B00000680D00200023044A1370044A13700120C5
:10B01000034B1870704700BF780D0020740D00209E
:10B02000710D002070470020704700000D4B5B88B9
:10B030001A0A032A01D00020704713F0FF0F0ED127
:10B04000084BDB88402B01D000207047054B064A97
:10B050009A60064A1A6140229A81012070470020B6
:10B06000704700BF102300207C0D0020A1B04000DD
:10B070000122014B1A707047710D002010B5034B6F
:10B08000034A04490448054CA04710BD2DB04000B8
:10B09000CC020020740D0020780D0020E5B14000A6
:10B0A00008B5084B9B89402B00D008BD064B1B7888
:10B0B0001BB90648064B9847F7E70448054B9847E5
:10B0C00008BD00BF10230020700D00207C0D002063
:10B0D0004D98400021504000014B1870704700BF50
:10B0E000700D0020224B1B780BB9184670472DE9D4
:10B0F000F04184B00746EFF31083B3FA83F35B09A2
:10B10000039372B6BFF35F8F00211A4B1970DDF8FD
:10B110000C80194D40222846184B98473C46403732
:10B120002E4620686168A268E3680FC61034354671
:10B13000BC42F5D1124B009340230F4A00218120DD
:10B14000104CA04780F00100094B1870B8F1000FB7
:10B1500005D00122074B1A70BFF35F8F62B6044B14
:10B160001B7883F00103184604B0BDE8F08100BFEE
:10B17000710D00202F030020BC0D00205D1C41003C
:10B1800071B04000C1D3400010B50446134B98473E
:10B19000837A212B01D0002010BD00F10902104B51
:10B1A0005B881B0A212B04D0C27B93420BD000206A
:10B1B00010BD0B4B9A60427AD9888A4228BF0A4652
:10B1C0009A81012010BD064B9C60028AD9888A4270
:10B1D00028BF0A469A81012010BD00BFBDB74000BC
:10B1E00010230020F8B5264C247865B2002D07DB2B
:10B1F000002D40DB04F06004202C22D00020F8BD9C
:10B2000014F0600603D11E4F7F78062F0BD0202E3E
:10B21000EED11B4A5278022A09D0032A0CD0012A07
:10B22000E6D19847F8BD1046164B9847F8BD144B29
:10B23000986001209881F8BD114B99600120988198
:10B24000F8BD0F4A52780A2A07D00B2A0BD0092AD8
:10B2500001D00020F8BD9847F8BD094B5B881B0A58
:10B2600003700120F8BD064BDB8833B9044B5B88C3
:10B270000B700120F8BD0020F8BD0020F8BD00BF14
:10B280001023002089B14000014B1868704700BFAF
:10B290007C220020024B1B681B68588818447047AA
:10B2A000080E002038B504460D46094B9847024663
:10B2B00020782044904207D24378042B06D0AB423A
:10B2C00005D003781844F5E7002038BD002038BDCC
:10B2D00095B2400038B5144B1B780BB3134B1B6869
:10B2E0001B681A7982421DD90D460446104A136024
:10B2F000104B984703E01A7813440D4A13600C4B27
:10B300001B6898420AD95A78042AF4D19A78944250
:10B31000F1D1DA78AA42EED1012038BD002038BD43
:10B32000002038BD002038BD040E0020080E00208B
:10B330000C0E002095B24000084BDB8863B9074B28
:10B340005B88012B01D000207047054A138823F049
:10B350000203138001207047002070471023002053
:10B36000FC0D002000207047044BDB8823B9044A01
:10B37000024B1A6101207047002070471023002003
:10B38000ADB6400038B5134B1B7803B3124B1C7994
:10B39000124B1B681B681B799C4201D3002317E0EA
:10B3A000002120460E4B9847034688B10B4B1B6883
:10B3B0005B6853F82450EB68984701462046084BD9
:10B3C0009847034620B1AB689847034600E0002346
:10B3D000184638BD040E002010230020080E00205F
:10B3E000D5B2400038B5104B1B78D3B100240F4BB9
:10B3F0001B681A681279944211D25B6853F8245082
:10B40000EB68984701462046094B9847034648B1E8
:10B41000AB689847034628B90134E4B2E7E7002354
:10B4200000E00023184638BD040E0020080E00205E
:10B43000D5B2400070B504460021114B984705462F
:10B4400008B9284670BD0F4B1B685B6853F8246031
:10B45000F368984701462046094B9847054600285F
:10B46000EFD0094B1C6805212046084B984704463D
:10B4700018B18078064B9847F5E773689847E0E77E
:10B48000D5B24000080E00200C0E0020A5B24000EE
:10B4900041D1400008B5064BDB88022B01D00020CB
:10B4A00008BD02210348044B9847012008BD00BF96
:10B4B00010230020FC0D002025D0400010B5184BB3
:10B4C0009B78032B2AD8DFE803F00502100B092034
:10B4D000144C0CE004211448144B9847002006E05B
:10B4E000134B98470446102001E00620114C08B188
:10B4F000002308E0012010BDE15C0F4A02EB43028B
:10B5000051800133DBB28342F6D3411C4900C9B2FA
:10B5100009480170054B9847012010BD002010BD5F
:10B52000102300201C0300201803002025D0400019
:10B5300089B2400028030020F402002008B5234B04
:10B540005B88DAB21B0A013B0E2B38D8DFE803F028
:10B5500008173137373737373737373737372A0014
:10B560001B4B186801781B4B9847184BDA889B894E
:10B570009A4228D2154B9A810123184608BD144BD4
:10B580001B685B7C9A4201D30023F6E7104B5B6893
:10B5900053F8320041880F4B98470C4B9B680222AE
:10B5A0005A70E2E70A4B986858B14188094B9847AE
:10B5B000DBE7094B984703460028D6D1DDE7002397
:10B5C000DBE70023D9E70123D7E700BF10230020E2
:10B5D000FC01002025D04000BDB4400008B5064B5A
:10B5E000DB88012B01D0002008BD01210348044B5A
:10B5F0009847012008BD00BF10230020040E002042
:10B6000025D0400038B5154BDB88012B02D0002433
:10B61000204638BD124B1B78F3B1104B1D79114BEE
:10B620001B681B681B799D4201D30024F0E70021B1
:10B6300028460D4B984704460028E9D0094B1B6863
:10B640005B6853F82530DB689847084B1870012178
:10B650001846074B9847DBE70024D9E71023002062
:10B66000040E0020080E0020D5B24000000E00207D
:10B6700025D0400008B5094BDB88022B01D0002003
:10B6800008BD064B1879064B9847064B18800221D7
:10B690001846054B9847012008BD00BF1023002025
:10B6A00091D14000FE0D002025D0400008B5034B8D
:10B6B000588800F07F00024B984708BD10230020F7
:10B6C000CDCF400038B505460F4B98470346C0B173
:10B6D0000E4B1C68052120460D4B9847044640B18F
:10B6E0008288C17880780B4B984703460028F1D1B7
:10B6F00007E0094B1B685B6853F825301B689847C7
:10B700000346184638BD00BFD5B240000C0E0020DD
:10B71000A5B2400031D04000080E002038B50C4BD7
:10B72000DB8893B90B4B1B780BB900230EE0084B59
:10B730001C799D782046084B9847034630B129462E
:10B740002046064B9847034600E00023184638BDC4
:10B7500010230020040E002035B44000C5B6400080
:10B7600008B5074BDB884BB9054B5B880BB1002054
:10B7700008BD034B1879034B984708BD002008BD4E
:10B7800010230020CDD24000094BDB886BB9084B59
:10B790005B880BB10020704710B5054C2079054B34
:10B7A00098472079044B984710BD0020704700BF90
:10B7B000102300203DD54000D5D14000014B186832
:10B7C000704700BF0C0E002008B5014B984708BD1C
:10B7D0006DCE400010B50B4B1B7863B1002404E024
:10B7E0002046094B98470134E4B2084B1B681B689C
:10B7F0001B799C42F4D30022024B1A700122044BA5
:10B800001A8010BD040E002035B44000080E002040
:10B81000FC0D002008B5024B9847024B984708BD25
:10B8200055CF4000D5B740001C4BDB8813B1002337
:10B830001846704710B51A4B984750B3174B9A7873
:10B84000184B1B685B7C9A4201DD002322E0164BFB
:10B850009847124B9B78154A1370EBB1114A526806
:10B8600003F10053013B02EBC303114A13600024B0
:10B870000F4B1B681B681B799C4208D20021204695
:10B880000C4B9847034628B10134E4B2F0E701239A
:10B8900000E00023184610BD0123FBE71023002021
:10B8A00009D04000FC010020D5B74000040E002064
:10B8B000080E0020C5B6400008B5344B1B7813F0C5
:10B8C000800F0ED113F01F0343D1304A5278013A52
:10B8D000082A3ED8DFE802F0343D373D313D3D3D9A
:10B8E0003A002A4AD288002A4ED013F01F0306D10C
:10B8F000264A5278062A0BD0082A0CD02AB1012BEE
:10B900000CD0022B11D0002008BD214B984708BD58
:10B91000204B984708BD204B984708BD1B4A5278DA
:10B920000A2AEED11D4B984708BD184B5B780BB126
:10B93000002008BD1A4B984708BD1A4B984708BD10
:10B94000194B984708BD194B984708BD184B9847A5
:10B9500008BD012B03D0022B08D0002008BD0B4AE4
:10B9600052780B2AF7D1134B984708BD074B5B78E9
:10B97000012B03D0032B04D0002008BD0E4B9847A9
:10B9800008BD0E4B984708BD002008BD10230020BD
:10B9900095B440003DB54000DDB5400005B640001F
:10B9A00075B6400069B3400039B3400065B340004C
:10B9B00029B840001DB7400061B7400089B740007A
:10B9C0000B4B1B7813B110B5002402E07047013413
:10B9D000E4B2084B1B681A681279944207D25B687C
:10B9E00053F824301B69002BF1D09847EFE710BDC6
:10B9F000040E0020080E002008B5184B00229A8182
:10BA00001A615A611B7813F0800F11D113F0600F87
:10BA100014D0124B1B7803F01F03012B14D00F4BD3
:10BA20001B7803F01F03022B14D00023184608BD17
:10BA30000A4AD288002AE9D10023F7E7084B984741
:10BA400003460028E5D0F1E7064B98470346002857
:10BA5000E5D0EBE7044B98470346E7E710230020C7
:10BA6000B9B8400085B34000E5B34000F8B50446DE
:10BA70000E46114B984705462046104B9847054007
:10BA800001D0002403E0F8BD0134062C11D88DB19B
:10BA900023010B4AD058B042F6D102EB0413596887
:10BAA0000D42F1D01F46DB6898477B6825EA030505
:10BAB000EAE7F8BDF8BD00BFB3D84000B7D84000F2
:10BAC000100E0020F8B5164C2768062F26D8002443
:10BAD00001E00134E4B2A446A7420AD3114E250185
:10BAE00006EB050E75598D42F3D1DEF804509542F0
:10BAF000EFD1CEF80010CEF80420CEF80830069929
:10BB0000CEF80C100137BC4505D011461A46064B3D
:10BB100098470020F8BD02490F60F6E70120F8BD04
:10BB2000800E0020100E002079D840002DE9F04151
:10BB300082B004460F4690460A4B98470546204679
:10BB4000094B984706462046084B9847CDF8008099
:10BB50003B46024631462846054CA04702B0BDE8A8
:10BB6000F08100BFBBD84000C9D84000CFD840000A
:10BB7000C5BA400008B50B210148024B984708BDE3
:10BB8000000E0E406DBA400008B50C210148024B72
:10BB9000984708BD00100E406DBA4000F8B5064643
:10BBA0000C461546224B984707464FF0FF3130466A
:10BBB000204B98473046204B9847002C0CDB6309FC
:10BBC00004F01F0101228A4020331C4941F8232040
:10BBD000BFF34F8FBFF36F8F002C08DB630904F0B6
:10BBE0001F0101228A406033144941F82320002CB0
:10BBF00017DB2D01EDB204F1604303F5614383F8D7
:10BC00000053002C08DB620904F01F04012303FA2F
:10BC100004F40A4B43F8224039463046084B984713
:10BC2000F8BD04F00F022D01EDB2064B9D54E8E77C
:10BC3000B7D84000AFD84000B3D8400000E100E0E2
:10BC4000ABD8400014ED00E082B0024610B9244B9E
:10BC50001B783BB912B1224B1B780BB3204B1A70E7
:10BC600002B070471F4B1B7803B9FEE7EFF3108358
:10BC7000B3FA83F35B09009372B6BFF35F8F0021C1
:10BC8000194B1970009817490B78013B0B7000286D
:10BC9000E0D00121144B1970BFF35F8F62B6D9E772
:10BCA000104B1B78FF2B19D0EFF31083B3FA83F3FB
:10BCB0005B09019372B6BFF35F8F00210A4B1970C5
:10BCC000019808490B7801330B700028C6D0012178
:10BCD000054B1970BFF35F8F62B6BFE7FEE700BF89
:10BCE000850E0020282300202F03002084B02A4B3B
:10BCF0009A6842F480729A609A6822F07F029A6091
:10BD00001A6B0192019A42F04F020192019A22F4B9
:10BD1000074222F080020192019A42F4004201920D
:10BD2000019A1A631C4B1B6B13F4004FFAD01A4A8A
:10BD3000136B0293029B43F04F030293029B43F465
:10BD400000430293029B136300238DF8033006E047
:10BD500000BF9DF803300133DBB28DF803309DF84E
:10BD60000330DBB2132BF3D9EFF31083B3FA83F371
:10BD70005B09039372B6BFF35F8F0022074B1A7003
:10BD8000039B0121044A116123B1044B1970BFF3D5
:10BD90005F8F62B604B07047004004402F0300205C
:10BDA000034A0023136153619381024A1370704761
:10BDB000102300208A0E002082B00522104B1A703A
:10BDC000104A136B0193019B43F04F030193019BB6
:10BDD00043F020030193019B136300238DF803308C
:10BDE00006E000BF9DF803300133DBB28DF803306D
:10BDF0009DF80330DBB2132BF3D902B0704700BFBC
:10BE00008A0E00200040044082B00322104B1A70BA
:10BE1000104A136B0193019B43F04F030193019B65
:10BE200043F010030193019B136300238DF803304B
:10BE300006E000BF9DF803300133DBB28DF803301C
:10BE40009DF80330DBB2132BF3D902B0704700BF6B
:10BE50008A0E0020004004400422014B1A707047F3
:10BE60008A0E002008B5024B1B6903B1984708BD34
:10BE70001023002030B589B06A4B1B78032B29D0E2
:10BE8000694B9C89694B1B88E41AA4B2002C43D1EE
:10BE9000674A11880B449BB21380634AD28893424D
:10BEA00003D0644B1B78002B2CD0634B9847634A1C
:10BEB000136B0393039B43F04F030393039B23F004
:10BEC00001030393039B13635C4B1B6B13F0010F84
:10BED000FAD115E0594A136B0293029B43F04F03CA
:10BEE0000293029B23F001030293029B1363534BC3
:10BEF0001B6B13F0010FFAD1514B9847514B9847E8
:10BF000009B030BD484B5B6933B1984720B100227E
:10BF1000464B1A80444B9C893F2C37D90022454B15
:10BF20001A704024404B9A68404B1B881A44EFF328
:10BF30001083B3FA83F35B09079372B6BFF35F8F85
:10BF40000021414B197007983C4B1B6B13F0020FFB
:10BF50003ED028B101223C4B1A70BFF35F8F62B60E
:10BF60000422304B1A70354A136B0493049B43F040
:10BF70004F030493049B23F001030493049B136376
:10BF80002E4B1B6B13F0010FFAD1B9E70122294B9D
:10BF90001A70C7E7157829490D650133DBB2013204
:10BFA00099B28C42F6D8214B1A8814441C80234A3B
:10BFB000136B0593059B43F04F030593059B43F0DB
:10BFC00010030593059B136300238DF8073008E0E9
:10BFD0000023E5E700BF9DF807300133DBB28DF8A1
:10BFE00007309DF80730DBB2132BF3D9134A136BDC
:10BFF0000693069B43F04F030693069B23F0010331
:10C000000693069B13630D4B1B6B13F0010FFAD1C4
:10C0100000283FF475AF01220B4B1A70BFF35F8FFE
:10C0200062B66DE78A0E002010230020860E0020E5
:10C03000880E0020840E002059BE400000400440BD
:10C0400065BE4000A1BD40002F03002010B586B0A2
:10C05000654B1B78012B1ED0022B04D0042B02D081
:10C06000624B984701E0624B9847624A136B00931A
:10C07000009B43F04F030093009B23F002030093C7
:10C08000009B13635B4B1B6B13F0020FFAD15A4BEF
:10C09000984706B010BD574B186BC0F30A40574B7A
:10C0A0009B89574A14882218934201DA181B80B2E0
:10C0B000524B9A682244002305E04E49096D1170E5
:10C0C0000133DBB2013299B28842F6D80444A4B2FB
:10C0D0004B4B1C8040281BD0484B9C815B6913B1A3
:10C0E0009847002832D0434A136B0293029B43F0D7
:10C0F0004F030293029B23F002030293029B1363FC
:10C100003C4B1B6B13F0020FFAD13E4B9847C0E734
:10C110003A4BDA883C4B1B8823449A42DCDD374B90
:10C120009B899C4227D0334A136B0593059B43F0B0
:10C130004F030593059B23F002030593059B1363AF
:10C140002C4B1B6B13F0020FFAD1A2E7274B984739
:10C15000284A136B0193019B43F04F030193019B0A
:10C1600023F002030193019B1363224B1B6B13F01B
:10C17000020FFAD18DE7214B5B6953B19847E8B1C3
:10C1800021491F4A0B88108803440B800023138029
:10C19000C9E7164B9847174A136B0393039B43F069
:10C1A0004F030393039B23F002030393039B136347
:10C1B000104B1B6B13F0020FFAD16AE70B4B984739
:10C1C0000C4A136B0493049B43F04F030493049BAA
:10C1D00023F002030493049B1363064B1B6B13F0C1
:10C1E000020FFAD155E700BF8A0E0020B9BD40000A
:10C1F00065BE400000400440A1BD40001023002067
:10C20000860E002009BE4000880E00200023042B6B
:10C2100014D810B40A499A00D418A000044608445F
:10C22000407C214400F083026FF3C7124A7401334B
:10C23000DBB2042BEED95DF8044B7047704700BFAA
:10C240008C0E002038B5437C13F0100F16D00D462D
:10C25000437C6FF30413437404687CB102F10C0354
:10C26000074951F8233013F4806F01D042F0800267
:10C270008168012D14BF00200120A04738BD00BFF8
:10C280000040044010B500240BE023460134E4B222
:10C2900003EB8303980022460121034B1844034B10
:10C2A0009847042CF1D910BD8C0E002045C24000E7
:10C2B00010B500F00F02531E03EB83039C00012115
:10C2C00002482044024B984710BD00BF8C0E00204E
:10C2D00045C2400030B482B00246441E3B4900F1E2
:10C2E0000C0551F8253051F8251013F0020302D047
:10C2F00001F0400151B9002B39D004EB84039900BF
:10C30000334B0B44597C6FF38301597404EB840362
:10C3100099002F4B0B445B7C13F00C0F32D12B494F
:10C3200000F10C0551F825300093009B43F04F03BA
:10C330000093009B23F002030093009B41F82530FB
:10C3400002F10C03214951F8233013F0020FF7D109
:10C35000002838D0032836D004EB8404A2001C4BFC
:10C3600013445A7C012161F383025A742BE004EBDD
:10C3700084039900164B0B44597C012565F3830116
:10C380005974C3E711490C3051F820300193019BD7
:10C3900043F04F030193019B23F040030193019B62
:10C3A00041F8203002F10C03084951F8233013F012
:10C3B000400FF7D104EB8404A200054B13445A7CD0
:10C3C0006FF383025A7402B030BC704700400440DF
:10C3D0008C0E0020F0B4461EB300334499002A4A64
:10C3E0000A445368D1680B449468641A128AC2F3F1
:10C3F0000902944209D31446002706EB86029500F1
:10C40000214A2A442144D1601EE00127F5E71D7826
:10C410001E4A00F1140142F821505D7842F8215083
:10C420009D7842F82150DD7842F821501D7942F87C
:10C4300021505D7942F821509D7942F82150DD79F3
:10C4400042F82150083C0833072CE0D807E01D785B
:10C4500000F114020D4941F82250013C0133002C37
:10C46000F5D1094BB1008819820010461A44527C5C
:10C47000C2F3810203440132597C62F3830159748F
:10C480003846F0BC704700BF8C0E002000400440CE
:10C4900070B582B0441E04EB84039A00364B1344FB
:10C4A0005B7CC3F3810328B1032801D0022202E0A0
:10C4B000012200E001229A4254DDA20022449500AC
:10C4C0002D4B2B44DA689B689A4205D32A4B2B44A8
:10C4D0005B7C13F0400F48D00E460546274B98472B
:10C4E000FEB1274A0C3552F825300193019B43F0E9
:10C4F0004F030193019B43F010030193019B42F80A
:10C50000253000238DF8033006E000BF9DF803308E
:10C510000133DBB28DF803309DF80330DBB2132B0F
:10C52000F3D940B104EB84039A00134B13445A7CB3
:10C530006FF386125A74A200224491000E4B0B44F2
:10C54000DA689B689A4212D30B4B0B445B7C13F066
:10C55000400F0ED1084B0B445A7C42F080025A74B3
:10C56000002000E0012002B070BD0020FBE70120A8
:10C57000F9E70120F7E700BF8C0E0020D5C340008B
:10C58000004004402DE9F84305468446471EBB00A1
:10C590003B449A002A4C1444A268E368A2EB030EC1
:10C5A000B4F81080C8F3090862681A440C302549B1
:10C5B00051F82060C6F30A4666B3B6450BD9B646B5
:10C5C0004FF0000907EB870188001D4901447344BF
:10C5D000CB6000210AE04FF00109F3E70CF11403EE
:10C5E000184850F823301370013101328E45F5D8C8
:10C5F0002846154B9847B9F1000F01D1B04507D92E
:10C6000005F10C030F4A52F8233013F0200F04D029
:10C61000BDE8F8834FF00009EAE70123AB4053611E
:10C62000074ABB00D819810008461144C968024472
:10C6300091602A4600212046044B9847E8E700BF56
:10C640008C0E002000400440D5C2400045C240008E
:10C650002DE9F0418CB00124ADE12046B34B984761
:10C660000120FAE1BB003B449900B14A0A44537CE3
:10C67000C3F38101033161F383035374537C13F0DB
:10C68000200F00F0848013F00C0F3BD0A94A04F176
:10C690000C0152F821300193019B43F04F030193A9
:10C6A000019B43F010030193019B42F821300023CA
:10C6B0008DF8013006E000BF9DF801300133DBB298
:10C6C0008DF801309DF80130DBB2132BF3D9994A74
:10C6D00006F10C0152F821300293029B43F04F0304
:10C6E0000293029B23F001030293029B42F8213044
:10C6F00006F10C038F4A52F8233013F0010FF7D1E3
:10C700000120AAE18B4A04F10C0152F82130039375
:10C71000039B43F04F030393039B23F00103039315
:10C72000039B42F8213006F10C03824A52F8233071
:10C7300013F0010FF7D1114606F10C0352F8232034
:10C740000492049A42F04F020492049A42F02002AA
:10C750000492049A41F8232000238DF8023006E069
:10C7600000BF9DF802300133DBB28DF802309DF836
:10C770000230DBB2132BF3D907EB8707BA006C4BFF
:10C7800013445A7C6FF345125A74012065E113F08B
:10C79000800F42D1BB003B449A00654B1344DA68DA
:10C7A0009B689A424CD307EB87039A00604B134473
:10C7B0005B7C13F04C0F43D1EFF31083B3FA83F398
:10C7C0005B090B9372B6BFF35F8F00225A4B1A704E
:10C7D0000B9B584A55612BB10122574B1A70BFF37E
:10C7E0005F8F62B6534A06F10C0152F8213005936F
:10C7F000059B43F04F030593059B23F0010305932D
:10C80000059B42F8213006F10C034A4A52F82330C6
:10C8100013F0010FF7D101201FE1BB003B449A0048
:10C82000434B1344597C6FF3C7115974DA689A600B
:10C83000404B5D61224600214046404B9847A9E7A6
:10C84000002C4AD0032C48D007EB87039A00384BC2
:10C8500013445B7C13F00C0F3FD0364A06F10C01F9
:10C8600052F821300693069B43F04F030693069B34
:10C8700043F010030693069B42F8213000238DF805
:10C88000033006E000BF9DF803300133DBB28DF8C2
:10C8900003309DF80330DBB2132BF3D9254A06F1A0
:10C8A0000C0152F821300793079B43F04F03079385
:10C8B000079B23F001030793079B42F8213006F101
:10C8C0000C031C4A52F8233013F0010FF7D100215A
:10C8D00020461B4B98470120BFE0002C4AD0032C78
:10C8E00048D001212046164B984758B3114A06F10B
:10C8F0000C0152F821300893089B43F04F03089332
:10C90000089B23F001030893089B42F8213006F1AD
:10C910000C03084A52F8233013F0010FF7D100211D
:10C920002046074B9847012097E000BF85C540008F
:10C930008C0E0020004004402F03002045C2400020
:10C9400091C440004749BB00D81982000A4492F8BC
:10C9500011E06FF3C71E82F811E0D2681F44BB00DC
:10C9600019448A60404B5D612246002140463F4B9E
:10C970009847BBE7012120463D4B98473A4A06F1CC
:10C980000C0152F821300993099B43F04F0309939E
:10C99000099B23F001030993099B42F8213006F11A
:10C9A0000C03314A52F8233013F0010FF7D1012064
:10C9B00053E00134E4B2052C4ED82B4B9B6926463C
:10C9C0000125A5402B42F4D0671E07EB8702930098
:10C9D000244A02EB030804F10C03234A52F82330E3
:10C9E00013F0420F7FF439AE04F10C031E4A52F8E3
:10C9F000233013F0010F7FF435AE04F10C031A4A13
:10CA000052F8233013F0080FD3D004F10C0152F880
:10CA100021300A930A9B43F04F030A930A9B23F0A9
:10CA200008030A930A9B42F8213006F10C030E4AD0
:10CA300052F8233013F0080FF7D106F10C0352F827
:10CA4000233003F4E063B3F5807F09D006F10C03D3
:10CA500052F82330012000E000200CB0BDE8F08146
:10CA60000120FAE78C0E00200040044045C240003F
:10CA700091C4400000B587B0534B1B78E3B9534BCA
:10CA80001B6BC3F30A43082B3BD0504A136B019333
:10CA9000019B43F04F030193019B23F00403019397
:10CAA000019B1363494B1B6B13F0040FFAD1484BE6
:10CAB000984707B05DF804FB464B9847464B9847AC
:10CAC000DDE7424A116D454A99540133DBB2072B29
:10CAD000F7D9434B9847B0B93C4A136B0293029B7A
:10CAE00043F04F030293029B23F004030293029B43
:10CAF0001363364B1B6B13F0040FFAD1344B98477A
:10CB0000D7E70023E3E7354B93F90030002B1EDB1A
:10CB10002E4A136B0593059B43F04F030593059B2A
:10CB200023F004030593059B1363284B1B6B13F041
:10CB3000040FFAD1294BDB88002B42D00023294A6D
:10CB40001380294A138001221F4B1A70B1E71F4A34
:10CB5000136B0393039B43F04F030393039B43F037
:10CB600080030393039B136300238DF8033006E0D7
:10CB700000BF9DF803300133DBB28DF803309DF820
:10CB80000330DBB2132BF3D9104A136B0493049BCD
:10CB900043F04F030493049B23F004030493049B8A
:10CBA00013630A4B1B6B13F0040FFAD100230D4AD9
:10CBB00013800D4A13800222034B1A700B4B9847C7
:10CBC00077E70B4B984774E78A0E0020004004403B
:10CBD000B9BD400065BE4000A1BD4000102300204B
:10CBE000F9B94000880E0020860E002075BE400076
:10CBF00009BE4000204BDB6913F0010F37D000B5B0
:10CC000083B01D4B1B6B13F0040F24D11A4B1B6B0D
:10CC100013F0010F23D1184B1B6B13F0020F22D11D
:10CC2000154B1B6B13F0080F23D0134A136B0193A2
:10CC3000019B43F04F030193019B23F008030193F1
:10CC4000019B13630C4B1B6B13F0080FFAD10120EF
:10CC500003B05DF804FB094B98470120F8E7084B47
:10CC600098470120F4E7074B98470120F0E70020A0
:10CC700070470020ECE700BF0040044075CA400048
:10CC800075BE40004DC0400010B54C4B984720B9D0
:10CC90004B4BDB6913F4807F10D03020494B984711
:10CCA000474B9B6913F4006F04D0454BDB6913F4C9
:10CCB000006F0AD1444B984770B110BD72B6BFF3F4
:10CCC0005F8F0022414B1A7010BD4FF400623C4B45
:10CCD0001A623F4B984710BD3E4B98470028ECD155
:10CCE000374B9B6913F4005F04D0354BDB6913F4B9
:10CCF000005F3DD1324B9B6913F4007F04D0304B71
:10CD0000DB6913F4007F33D12D4B9B6913F4806FE3
:10CD100004D02B4BDB6913F4806F29D1284B9B691E
:10CD200013F4807F04D0264BDB6913F4807F2FD16E
:10CD3000234BDB6913F4805FBFD0214C4FF4805349
:10CD40002362254B9847254B9847636823F00103DE
:10CD50006360636823F002036360214B9847214BB3
:10CD600098474FF4807323614FF400632361A4E775
:10CD7000134C4FF418532362636101201A4B9847F8
:10CD80004FF48073236223614FF40063236110BD6D
:10CD90000B4B4FF480721A625A614FF400521A61C1
:10CDA0004FF400721A614FF480621A6130200F4B09
:10CDB000984700200C4B984710BD00BF29DE40006B
:10CDC00000400440F1DC4000F5CB40002F03002080
:10CDD000C1B9400051C6400085C24000D5B74000EF
:10CDE000EDBC4000A1BD400049BC400045DD400015
:10CDF00010B582B0EFF31083B3FA83F35B090193AC
:10CE000072B6BFF35F8F0022144B1A70019C012091
:10CE1000134B98473020134B9847134B5A6F22F40B
:10CE200080725A675A6F42F400725A674FF48072E8
:10CE30001A614FF400521A614FF400721A614FF4F4
:10CE400080621A614FF400621A612CB10122034B17
:10CE50001A70BFF35F8F62B602B010BD2F030020BF
:10CE600049BC4000F1DC40000040044030B583B0D4
:10CE7000EFF31083B3FA83F35B09009372B6BFF349
:10CE80005F8F0024204B1C70009D204B9847302062
:10CE90001F4B98471F4B98471F4B502283F8302356
:10CEA0004FF480325A601D4B98474FF480201C4B42
:10CEB00098471C4B1C701C4B1B78FF2B22D0EFF3A8
:10CEC0001083B3FA83F35B09019372B6BFF35F8FEC
:10CED00000220D4B1A700199134A13780133137015
:10CEE00029B10122084B1A70BFF35F8F62B60F4B56
:10CEF00098472DB10122044B1A70BFF35F8F62B6C1
:10CF000003B030BDFEE700BF2F030020F5D6400080
:10CF1000F1DC4000DDD8400000E100E00DC240003F
:10CF200015DE4000850E002028230020F1CD4000B2
:10CF300008B5064B5A6F42F480725A675A6F22F452
:10CF400000725A670020024B984708BD0040044019
:10CF500049BC400010B582B0EFF31083B3FA83F3FD
:10CF60005B09009372B6BFF35F8F0022144B1A70F7
:10CF7000009C144B9847144B1B7803B9FEE7EFF362
:10CF80001083B3FA83F35B09019372B6BFF35F8F2B
:10CF900000220B4B1A7001990B4A1378013B137056
:10CFA00029B10122064B1A70BFF35F8F62B62CB114
:10CFB0000122034B1A70BFF35F8F62B602B010BD3F
:10CFC0002F03002031CF4000282300200D4B5A684A
:10CFD00022F001025A609A6822F480729A60024636
:10CFE00070B1986820F07F0002F07F0210439860D3
:10CFF0009A6842F480729A605A6842F001025A605C
:10D00000704700BF00400440054B5B6813F0010F00
:10D0100004D0034B986800F07F00704700207047F1
:10D0200000400440014B9860998170471023002014
:10D03000F0B583B045B200F00F00052873D801F0B9
:10D040000306044600F10C033B4F57F8233013F45A
:10D05000004F6BD1012E53D0031FDBB2012B54D9EB
:10D060004023934266DB461E06EB8607334B03EBF9
:10D07000870303F11007B3F810E062F3090EA3F879
:10D0800010E05B7C03F07F036FF345137B70002D92
:10D090003EDB294EB36A012282401343B362264B22
:10D0A0009B6A1A42FBD0244B9E6A26EA02029A62CD
:10D0B00000F10C0253F822300193019B43F04F031F
:10D0C0000193019B23F4074323F080030193002D78
:10D0D00023DB0A0202F4407242F40042019B134334
:10D0E000019301990C30144B43F8201004F10C0308
:10D0F000114951F8233032EA0303F7D1012013E03C
:10D10000B0B10328A8D100200EE04FF40073A8E7C7
:10D110007B786FF383037B70BBE70A0202F44072F3
:10D1200042F40442DAE7002003B0F0BD0020FBE740
:10D130000020F9E70020F7E7004004408C0E0020B3
:10D1400000F00F03052B1ED810B582B019460E4C07
:10D150000C3354F823200192019A42F04F020192BD
:10D16000019A22F400420192019A44F8232001F12D
:10D170000C03054A52F8233013F4004FF7D1034B48
:10D18000984702B010BD704700400440B1C2400053
:10D1900000F00F00431E052815D803EB83039A0007
:10D1A0000A4B13445B7C13F0200F08D10C30084B62
:10D1B00053F8203013F0280F03D0012070470120CE
:10D1C0007047002070470020704700BF8C0E002081
:10D1D0000040044010B485B044B200F00F000528B0
:10D1E00065D8421EEFF31083B3FA83F35B09039310
:10D1F00072B6BFF35F8F0021314B19700399002C79
:10D2000014DB304A00F10C0452F824300293029BE4
:10D2100043F04F030293029B43F020030293029BCF
:10D2200042F8243000238DF807302EE000F10C0383
:10D23000244C54F8233013F0100F09D102EB820371
:10D240009C00214B23445B7CC3F38103012BD8DD7D
:10D2500002EB820294001C4B23445A7C42F02002D1
:10D260005A74012303FA00F0164B186121B3012010
:10D27000134B1870BFF35F8F62B619E000BF9DF8C3
:10D2800007300133DBB28DF807309DF80730DBB291
:10D29000132BF3D9012303FA00F00A4B186169B18B
:10D2A0000120074B1870BFF35F8F62B600E00020CB
:10D2B00005B05DF8044B70470120F9E70120F7E75E
:10D2C0002F030020004004408C0E002000F00F00CF
:10D2D00005286CD830B583B00246441E04EB8403A5
:10D2E0009900354B0B44597C6FF34511597400F18B
:10D2F0000C03324951F8233013F0200F59D000F1BC
:10D300000C0551F825300093009B43F04F03009328
:10D31000009B23F020030093009B41F8253002F18D
:10D320000C03264951F8233013F0200FF7D10D4696
:10D330008B6A012181400B43AB62204B9B6A1942EF
:10D34000FBD01E4B9D6A25EA010199620C3053F80F
:10D3500020100191019941F04F010191019921F0B3
:10D3600008010191019943F8201002F10C031349BF
:10D3700051F8233013F0080FF7D104EB84039A001F
:10D380000D4B13445B7C13F0100F01D1012011E011
:10D390000949A200101983000B44587C6FF3041054
:10D3A00058741444A300CB589847012002E0002091
:10D3B0007047012003B030BD8C0E002000400440B7
:10D3C000F0B583B000F00F04052C00F2A28047B244
:10D3D000651E04F10C00554E56F8200010F4004F65
:10D3E00000F09A8005EB8500514E06EB8000407CF2
:10D3F00010F0200F40F0928004F10C004B4E56F8D4
:10D40000200010F0200F40F08B80EFF31080B0FA76
:10D4100080F04009009072B6BFF35F8F0026454848
:10D420000670DDF800E005EB8500414E06EB80005C
:10D43000407C10F0100F0AD0BEF1000F72D0012214
:10D440003C4B1A70BFF35F8F62B6002062E005EBC1
:10D450008500374E06EB8000467C46F01006467489
:10D46000BEF1000F05D0012632480670BFF35F8F72
:10D4700062B6DFF8BCE005EB850080000EEB00062D
:10D480007260B3600022F260089A4EF8002011B971
:10D490005BBB012000E00120254AA9004B1902EBEB
:10D4A00083035B7C60F386130D4402EB85026FF30C
:10D4B000C7135374EFF31083B3FA83F35B0901933B
:10D4C00072B6BFF35F8F00221A4B1A70019D0123C1
:10D4D000A340164A1361002F09DB2DB30120154B21
:10D4E0001870BFF35F8F62B614E00020D4E704F138
:10D4F0000C0352F8233013F0110FEED10121204616
:10D500000D4B98470028E8D0002120460A4B984749
:10D51000E3E7002003B0F0BD0020FBE70020F9E7BF
:10D520000020F7E70020F5E70120F3E70040044082
:10D530008C0E00202F03002091C4400070B586B0EF
:10D5400000F00F04052C00F2C98042B2EFF3108303
:10D55000B3FA83F35B09059372B6BFF35F8F0021C3
:10D560005F4B1970059B26460125A5405D494D611D
:10D570002BB101215A4B1970BFF35F8F62B6002A9D
:10D5800080F2948004F10C03564A52F8233013F0D1
:10D59000100F64D0002C49D0032C47D004F10C01AB
:10D5A00052F821300193019B43F04F030193019BFB
:10D5B00023F010030193019B42F8213006F10C0384
:10D5C000484A52F8233013F0100FF7D106F10C033C
:10D5D000444A52F8233013F0100FF7D104F10C0134
:10D5E00052F821300293029B43F04F030293029BB7
:10D5F00043F010030293029B42F8213000238DF880
:10D60000033006E000BF9DF803300133DBB28DF834
:10D6100003309DF80330DBB2132BF3D906F10C0372
:10D62000304A52F8233013F0100FF7D02D4A04F18E
:10D630000C0152F821300393039B43F04F030393F3
:10D64000039B23F010030393039B42F8213006F160
:10D650000C03244A52F8233013F0100FF7D1214A5B
:10D6600004F10C0152F821300493049B43F04F0362
:10D670000493049B23F001030493049B42F821309C
:10D6800006F10C03174A52F8233013F0010FF7D1BB
:10D69000621E02EB82029100134B0B445A7C6FF323
:10D6A00083025A740AE02046104B984706F10C0397
:10D6B0000C4A52F8233013F0420FF4D1094A936A0E
:10D6C0002B439362074B9B6A1D42FBD0054A936A2A
:10D6D00023EA050595622046054B984706B070BDC4
:10D6E0002F030020004004408C0E0020D5C24000D3
:10D6F000B1C24000064BD3F8142122F44062C3F8B3
:10D700001421D3F8202142F00102C3F820217047F0
:10D7100000020E400B4619B1096801605B68436066
:10D720001AB11368036153684361704721F0FE0129
:10D73000C905C90D0162704710B51E4B53F8204052
:10D740002268536A13F0805F11D00223C2F820319F
:10D7500023684FF0FF32DA6100232375236913F049
:10D76000010F26D0636823B32046984710BD13F0FD
:10D77000006F13D00223C2F8203123684FF00062FB
:10D78000DA61236913F0020F03D0A3680BB12046BE
:10D79000984723680122C3F8202110BD13F0007FB1
:10D7A00007D0236913F0040F03D0E3680BB12046C0
:10D7B000984710BDF00E002008B50020014B984797
:10D7C00008BD00BF39D7400008B50120014B98477C
:10D7D00008BD00BF39D7400070B505460E46144657
:10D7E000016001230B60214B99422BD00D20204B6F
:10D7F0009847204B1D6023781B0203F4FE4373609F
:10D8000063782BBB0022A3780BB142F00402E378CB
:10D810000BB142F0080223790BB142F01002637998
:10D820001B0203F47063A179090389B20B4313430C
:10D83000B3652389C3F30E03628943EA0243F365A8
:10D8400000230CE012200A4B98470A4B5D60D2E798
:10D850000222D8E705EB8302002151600133022B3D
:10D86000F8D900202861287570BD00BF0000034072
:10D87000F1DC4000F00E002012F0100F12D0C0F8C2
:10D88000B01012F0200F07D0C0F8D41012F0400FE3
:10D8900005D0C0F8C0107047C0F8D010F6E7C0F847
:10D8A000C4107047C0F8B4107047016470474164F9
:10D8B0007047C06C7047806C7047400900F50010DD
:10D8C00000F207704002704740090B30704700F0CB
:10D8D0001F00012303FA00F07047000008B5002084
:10D8E0000A4B98470A4B98470028FBD0094B9847AA
:10D8F000094A0A4BDA620A4B98470028FBD00020FD
:10D90000084B9847084B984708BD00BF6DDC4000A6
:10D9100091DC4000D5DC4000013FB80500040E401A
:10D92000E1DC4000F5DD400009DE400010B5A2B0AA
:10D930001848194B98470020184B9847184B9847A0
:10D940000028FBD0174B9847174A184B9A62184B80
:10D9500098470028FBD00020164B9847164B984755
:10D9600016480D4B9847164B1A68164B1344164A27
:10D97000934201D922B010BD2023009302AB0F22A5
:10D980000E211248124CA047BDF848101148124B06
:10D990009847EFE7000E270779E140006DDC400073
:10D9A00091DC4000B9DC4000013FB70B00040E40A1
:10D9B000C5DC400019DC400085E040000000DC05CB
:10D9C00030030020C0D3BDF980C3C901000A0E4056
:10D9D0001100002010140E4039DE400070B50D46D5
:10D9E0001446064658B14FF0FF360AE0064B186859
:10D9F000064B1B682946984701350136013C002C2F
:10DA0000F4DC304670BD00BF3823002030230020F6
:10DA100070B5013802280FD8144600258CB10A4B86
:10DA200018684E1C094B1B6809789847002806DBCC
:10DA30000135013C3146F1E74FF0FF3501E04FF091
:10DA4000FF35284670BD00BF382300203423002056
:10DA5000A1F10E03012B02D84FF0FF30704710B533
:10DA600082B0EFF31083B3FA83F35B09019372B6CC
:10DA7000BFF35F8F00240B4B1C70019C120222F03D
:10DA80007F4222F0FF02C9B2114341F0B441064B7C
:10DA900098472CB10122034B1A70BFF35F8F62B617
:10DAA00002B010BD2F030020790000204C4B1B78E2
:10DAB000FF2B31D000B583B0EFF31083B3FA83F3BB
:10DAC0005B09019372B6BFF35F8F0022454B1A705A
:10DAD0000199434A13780133137029B10122414B54
:10DAE0001A70BFF35F8F62B63F4A904215D03F4A2B
:10DAF000904220D03E4A90422BD03E4A904236D0AF
:10DB00003D4A904241D03D4A90424CD03C4A9042DE
:10DB100057D003B05DF804FBFEE71620394B984759
:10DB20000720394B984700210720384B984707209A
:10DB3000374B9847EDE71520324B98470720324B7B
:10DB4000984700210720314B98470720304B9847D2
:10DB5000DFE714202B4B984707202B4B98470021D9
:10DB600007202A4B98470720294B9847D1E71320D5
:10DB7000244B98470620244B984700210620234B2E
:10DB800098470620224B9847C3E70E201D4B984725
:10DB900006201D4B9847002106201C4B9847062065
:10DBA0001B4B9847B5E70920164B98470620164BA4
:10DBB000984700210620154B98470620144B98479C
:10DBC000A7E708200F4B984706200F4B98470021E6
:10DBD00006200E4B984706200D4B984799E700BF4B
:10DBE000282300202F030020000004400080004074
:10DBF00000C001400080014000400240000002409F
:10DC000000C00040F1DC4000E1DD400099DD400053
:10DC1000CDDD400001607047134A136B23F07003A1
:10DC2000184310634FF400630F4A926E12F0080F0E
:10DC300002D1A3B1013BF7E70B4A136B23F00303B7
:10DC400043F0020313634FF40063074A926E12F02D
:10DC5000080F02D12BB1013BF7E7002070470120EC
:10DC600070470120704700BF00040E40012803D018
:10DC7000054A064B1A607047044A936843F02543EF
:10DC800043F480139360F3E7080000A510140E40DE
:10DC9000074B5B6913F0800F06D0064B9B6E13F0A9
:10DCA000800F03D10020704700207047012070478B
:10DCB00010140E4000040E400022014B9A6270477F
:10DCC00000040E40024B986E00F00200704700BF47
:10DCD00000040E400022014BDA62704700040E403F
:10DCE000024B986E00F00400704700BF00040E4025
:10DCF00032281ED81F280CD8114B9A690123834063
:10DD0000934318D0012303FA00F00D4B1861002053
:10DD1000704720380A4BD3F80821012383409343EE
:10DD20000BD0012303FA00F0054BC3F800010020DB
:10DD3000704701207047002070470020704700BFE7
:10DD400000040E40322822D81F280ED8114B9A69A1
:10DD500001238340934301D000207047012303FA3D
:10DD600000F00C4B5861002070472038094BD3F865
:10DD7000082101238340934301D0002070470123F1
:10DD800003FA00F0034BC3F80401002070470120A0
:10DD9000704700BF00040E4041F0040100F1100282
:10DDA000094B43F822104FF40062074B996E4FF471
:10DDB00080738340194202D11AB1013AF5E700207D
:10DDC00070470120704700BF00040E404FF480737D
:10DDD00003FA00F0014B1860704700BF00040E40CA
:10DDE0004FF4807303FA00F0014B5860704700BF96
:10DDF00000040E40000200F4706040F00100014B8E
:10DE00009863704700040E408022014B1A607047EF
:10DE100000040E40C0F31200024B1A6F1043186743
:10DE2000704700BF00040E40024B187880F00100DC
:10DE3000704700BFF80E0020C36923F4F053490275
:10DE400001F4F051194341F0B44141F48071C161D2
:10DE5000704730B4B2EB011F17D3102401FB04F15B
:10DE60004B0803EBC202B2FBF1F2D3085D1E4FF682
:10DE7000FE718D4210D8082C09D0120402F4E02261
:10DE80001A430262002030BC70470824E6E741686C
:10DE900041F400214160F0E70120F4E740230360F2
:10DEA0007047882303607047102303607047242362
:10DEB000036070474FF48073036070474FF4002392
:10DEC00003607047436913F0020F04D0C1F30801E7
:10DED000C1610020704701207047436913F0020FB1
:10DEE000FBD0C1F30801C16100207047436913F002
:10DEF000010F05D08369C3F308030B60002070474E
:10DF000001207047014BC0F8E43070470041535581
:10DF100010B50446094B9847002363606362A3620F
:10DF20002046074B98472046064B98472046064B0D
:10DF300098472046054B984710BD00BF05DF4000BD
:10DF4000A3DE4000AFDE4000B5DE4000BDDE400095
:10DF500070B505460C461646104B98470022104BEC
:10DF60001A60B4B13246216828460E4B98470246E3
:10DF700088B96368A1680B4321690B43E1680B43CF
:10DF80000749086803430B6069680B436B601046E0
:10DF900070BD0122FBE70122F9E700BF11DF40005D
:10DFA000FC0E002053DE400000B583B0234B244A12
:10DFB0009A4209D0214B224A03E0116819600433C8
:10DFC000043220498B42F8D31F4B02E000221A6032
:10DFD00004331E4A9342F9D31D4A22F07F011D4BA0
:10DFE0009960EFF31083B3FA83F35B09019372B680
:10DFF000BFF35F8F0021184B1970019817490B6808
:10E0000043F470030B60BFF34F8FBFF36F8F28B1E2
:10E010000121114B1970BFF35F8F62B602F16042AC
:10E02000B2F5203F04D20B4A936843F0005393604B
:10E030000B4B98470B4B9847FEE700BF10000020A2
:10E0400034534100E80C0020E80C00201C24002080
:10E050000040400000ED00E02F03002088ED00E0CC
:10E06000651341000D03410008B50120034B98479B
:10E07000EFF30580024B9847FFDE00BF854D40005F
:10E08000914D4000344B1B6B03F00303012B20D058
:10E0900083B1022B39D0304B1B6B03F07003702B14
:10E0A00051D02D4B1A6BC2F302122C490B68D3408E
:10E0B0000B6070472A4B5B6913F0800F04D04FF45C
:10E0C0000042264B1A60E6E74FF4FA42234B1A60EF
:10E0D000E1E7214B1B6A13F0807F03D0214A1F4BDD
:10E0E0001A60D8E7204A1D4B1A601B4B1B6A03F0CD
:10E0F0007003102B05D0202BCDD11C4A174B1A6072
:10E10000C9E71B4A154B1A60C5E7154B5B6913F04D
:10E11000800F13D04FF40042104B1A600E4B1B6B54
:10E1200003F00303022BB6D10B4B9A6AC2F30C42E5
:10E130000A490B6802FB03330B60ACE74FF4FA4269
:10E14000064B1A60EAE7054A13680A49A1FB031364
:10E150005B081360704700BF00040E4030030020CE
:10E1600010140E40001BB70000127A0000366E013A
:10E170000024F400ABAAAAAA144B98420FD9144B5E
:10E18000984211D9134B984212D9134B984213D984
:10E19000124B984214D9124A124B1A6070474FF032
:10E1A0008062104B1A6070470F4A0E4B1A6070471E
:10E1B0000E4A0C4B1A6070470D4A0A4B1A607047A2
:10E1C0004FF00422074B1A60704700BFFF2C31014B
:10E1D000FF596202FF869303FFB3C404FFE0F50515
:10E1E00000050004000A0E400001000400020004C3
:10E1F000000300040A4B1B6853B1094B1B681A1833
:10E200000849914208DB1046054A106018467047DD
:10E21000054A034B1A60F0E74FF0FF30704700BF2C
:10E22000000F0020FC7F0220205400204FF0FF3020
:10E2300070474FF400534B60002070470120704737
:10E240000020704700F1080343604FF0FF32826006
:10E25000C3600361002303607047002303617047BC
:10E2600043684B609A688A609A6851609960086157
:10E27000036801330360704730B40D68B5F1FF3FA8
:10E2800002D000F1080202E0026904E01A46536875
:10E290001C68A542FAD253684B6099608A6051604D
:10E2A000086103680133036030BC7047036942684A
:10E2B000816891608268416851605A68904206D0D6
:10E2C000002202611A68013A1A6018687047826871
:10E2D0005A60F5E782B0002301934FF0500383F3B7
:10E2E0001188BFF36F8FBFF34F8F019B002BFCD0C2
:10E2F00002B0704708480068006880F308884FF053
:10E30000000080F3148862B661B6BFF34F8FBFF38D
:10E310006F8F00DF00BF000008ED00E0DFF80C00A9
:10E32000016841F4700101607047000088ED00E071
:10E330004FF0807340F8043C21F0010140F8081CC4
:10E34000054B40F80C3C40F8202C6FF0020340F8DD
:10E35000243C4438704700BFD5E240000000000074
:10E36000074B19680868B0E8F04F80F30988BFF3DD
:10E370006F8F4FF0000080F311887047AFF300807B
:10E38000040F00204FF0500383F31188BFF36F8F09
:10E39000BFF34F8F024A136801331360704700BF09
:10E3A00034030020034A1368013B13600BB983F365
:10E3B00011887047340300200000000000000000B6
:10E3C000EFF30980BFF36F8F154B1A681EF0100F23
:10E3D00008BF20ED108A20E9F04F10602DE90900F8
:10E3E0004FF0500080F31188BFF34F8FBFF36F8F52
:10E3F00000F07CFF4FF0000080F3118809BC196821
:10E400000868B0E8F04F1EF0100F08BFB0EC108A9B
:10E4100080F30988BFF36F8F704700BFAFF30080B0
:10E42000040F002008B54FF0500383F31188BFF3A9
:10E430006F8FBFF34F8F054B984718B14FF0805245
:10E44000034B1A60002383F3118808BD69F0400074
:10E4500004ED00E0054B00221A6005490A600549F9
:10E46000054A116007221A60704700BF10E000E003
:10E4700018E000E0FF7F010014E000E010B50E4B53
:10E480001A6842F470021A601A6842F070421A6008
:10E490000A4B984700240A4B1C600A4B98470A4ACB
:10E4A000136843F040431360084B9847084B984764
:10E4B000084B9847204610BD20ED00E055E4400091
:10E4C000340300201DE3400034EF00E0F5E240009B
:10E4D000EDF24000D5E2400010B50446044B9847E9
:10E4E0002046044B98470446034B9847204610BDEE
:10E4F0004DF04000DD1341005DF1400048B110B522
:10E500000446044B98472046034B9847034B9847D3
:10E5100010BD70474DF04000ED1341005DF140002B
:10E52000436A23B1036B1868C0F1050070470020EF
:10E530007047000010B50446064B9847A26BE36B8A
:10E540009A4204D00024044B9847204610BD012471
:10E55000F9E700BF85E34000A5E3400010B504469D
:10E56000054B9847A36B23B10024044B98472046E2
:10E5700010BD0124F9E700BF85E34000A5E340009A
:10E5800070B504461646856B026C5AB903681BB118
:10E5900000200135A56370BD4068174B98470023E4
:10E5A0006360F6E76EB98068144B9847226CA368E5
:10E5B0001344A3606268934219D32368A3600020C8
:10E5C000E7E7C0680D4B9847226C5242E36813445A
:10E5D000E36021688B4202D263681A44E260022E33
:10E5E00001D00020D5E725B1013D0020D1E7002072
:10E5F000CFE70020CDE700BFFDF54000611A4100E4
:10E60000026C72B110B5C3681344C3604468A3427E
:10E6100001D30368C3600C46C1682046014B98478C
:10E6200010BD7047611A410038B505461A4B98472E
:10E6300095F8454064B201E0013C64B2002C0ADD6B
:10E640006B6A43B105F12400144B98470028F3D0BE
:10E65000134B9847F0E7FF2385F84530114B984757
:10E660000D4B984795F8444064B201E0013C64B218
:10E67000002C0ADD2B6943B105F11000074B9847C8
:10E680000028F3D0064B9847F0E7FF2385F8443085
:10E69000044B984738BD00BF85E34000F1F34000CC
:10E6A000EDF44000A5E3400038B504460D46144B98
:10E6B00098472168E26B236C03FB02106060002026
:10E6C000A063A160013A02FB0313E360FF2384F817
:10E6D000443084F8453055B923691BB9094B984734
:10E6E000012038BD04F11000074B9847F6E704F10C
:10E6F0001000064DA84704F12400A847EEE700BF2C
:10E7000085E34000A5E34000F1F3400045E240000E
:10E7100038B51D46049C0B4649B12260E063236472
:10E7200001212046034B984784F84C5038BD2460A3
:10E73000F4E700BFA9E64000F0B583B005461746F0
:10E740000E4689B100FB01F05030084B9847044653
:10E7500038B100903B4600F1500231462846044D46
:10E76000A847204603B0F0BD0020EDE7D9E4400003
:10E7700011E74000F0B585B004460F4601921E46F1
:10E78000002526E0324639462046354B9847636AD5
:10E7900023B9344B9847012005B0F0BD04F12400A3
:10E7A000314B9847F5E72F4B98470020F4E702A834
:10E7B0002E4B9847012519E0002384F8443021E0CE
:10E7C000002384F8453023E02046294B9847294B05
:10E7D0009847294B9847A26BE36B9A42D2D3022EFB
:10E7E000D0D0019B002BDED0002DE0D01D4B9847F0
:10E7F000224B9847204B984794F844305BB2B3F1D2
:10E80000FF3FD9D094F845305BB2B3F1FF3FD7D08A
:10E81000144B984701A902A8194B9847C8B920463C
:10E82000184B98470028CFD0019904F11000164BDF
:10E83000984720460E4B98470E4B98470028C8D162
:10E840004FF08052114B1A60BFF34F8FBFF36F8FA1
:10E85000BFE72046064B9847064B984700209BE7AA
:10E8600081E54000A5E34000F1F3400071F4400071
:10E8700029E640005DF1400085E340004DF0400096
:10E8800089F4400035E54000A1F3400004ED00E0CC
:10E8900048B110B5002141600160C1600B460A46D5
:10E8A000014CA04710BD704775E7400010B5024607
:10E8B00000210120034B98470446034B984720460C
:10E8C00010BD00BF39E7400091E84000F8B5EFF314
:10E8D00011864FF0500484F31188BFF36F8FBFF39C
:10E8E0004F8F856BC46BA54205D3022B03D000204C
:10E8F00086F31188F8BD1746054690F8454064B286
:10E900001A460E4B9847B4F1FF3F05D0013464B26C
:10E9100085F845400120EBE76B6A0BB90120E7E77A
:10E9200005F12400064B984718B127B10120386043
:10E93000DEE70120DCE70120DAE700BF81E54000E7
:10E94000F1F34000F0B585B004460F460192002671
:10E9500032E039462046384B9847013DA56323698C
:10E9600023B9364B9847012005B0F0BD04F11000E3
:10E97000334B9847F5E7314B98470020F4E702A85E
:10E98000304B9847012621E0002384F8443029E0E9
:10E99000002384F845302BE020462B4B98472B4B27
:10E9A000984709E02046284B9847284B984720462F
:10E9B000274B984700283DD1264B9847A56B002D43
:10E9C000C7D1019B002BD6D0002ED8D01B4B984727
:10E9D000214B98471F4B984794F844305BB2B3F1F2
:10E9E000FF3FD1D094F845305BB2B3F1FF3FCFD0B9
:10E9F000124B984701A902A8184B98470028D1D17B
:10EA00002046134B98470028C6D0019904F12400F2
:10EA1000134B984720460C4B98470C4B98470028BF
:10EA2000CAD14FF080520F4B1A60BFF34F8FBFF324
:10EA30006F8FC1E7002097E701E64000A5E34000A3
:10EA4000F1F3400071F4400029E640005DF1400020
:10EA50005DE5400085E340004DF0400089F4400052
:10EA6000A1F3400004ED00E070B584B004460191CC
:10EA7000002635463EE0013BA36323683BB1236992
:10EA80004BB9444B98470126304604B070BD424B09
:10EA900098476060F3E704F11000404B9847F0E7B7
:10EAA0003C4B98470026EFE702A83D4B98470125CD
:10EAB0002AE0002384F8443032E0002384F8453013
:10EAC00034E0384B98476068374B98470646314BDF
:10EAD00098473BE02046354B9847354B984709E02F
:10EAE0002046324B9847324B98472046314B984747
:10EAF000002840D12B4B9847A36B002BBBD1019B27
:10EB0000002BCDD0002DCFD0224B98472A4B9847D1
:10EB1000244B984794F844305BB2B3F1FF3FC8D020
:10EB200094F845305BB2B3F1FF3FC6D0194B98471C
:10EB300001A902A8214B98470028D1D120461D4B9E
:10EB400098470028C6D02368002BBAD0019904F159
:10EB500024001B4B98472046144B9847144B98476A
:10EB60000028C7D14FF08052164B1A60BFF34F8F69
:10EB7000BFF36F8FBEE7002E86D00A4B9847204622
:10EB8000114B984701466068104B9847014B9847D6
:10EB9000002679E7A5E3400025F74000F1F34000A7
:10EBA00071F4400085E3400035F5400029E640005F
:10EBB0005DF140005DE540004DF0400089F440000B
:10EBC000A1F3400004ED00E021E5400085F640009F
:10EBD0000023092B0CD8074A52F833200AB101331D
:10EBE000F7E7044A42F8331002EBC303586070475A
:10EBF000704700BF3C23002070B504460D46164602
:10EC0000124B984794F844305BB2B3F1FF3F0DD0FC
:10EC100094F845305BB2B3F1FF3F0BD00C4B9847F3
:10EC2000A36B5BB120460B4B984770BD002384F863
:10EC30004430EDE7002384F84530EFE732462946BB
:10EC400004F12400044B9847ECE700BF85E3400043
:10EC5000A5E3400029E64000C5F34000F0B5036895
:10EC60004BB343685B68436000F10807BB4204D0C4
:10EC70004368D3F80CE0002609E05B684360F7E7DF
:10EC80005B68436008E02E46B6B9AE4514D04368D1
:10EC90005B6843609F42F3D04368DD6800230F2B1D
:10ECA000F2D8EA1892F83420CC5CA242ECD1002AC7
:10ECB000E9D00133F3E700263046F0BD002301E040
:10ECC000013001330278A52AFAD0C3F38F007047D0
:10ECD0000A4B1B681B684BB901234BB9074B1B68D8
:10ECE000DB68DB685A68064B1A6070470023F4E75C
:10ECF0004FF0FF32024B1A60704700BF080F002030
:10ED0000B40F00202DE9F84F81460D4617469A466C
:10ED10000A9EDDF82C800C9C9200A521206B1D4BD7
:10ED20009847236B07F18042013A03EB820727F0F3
:10ED3000070700230F2B07D8E95CE21882F834108C
:10ED4000EA5C0AB10133F5E7002384F84330042E6E
:10ED500000D90426E662E66400252565201DDFF85B
:10ED60003CB0D84704F11800D8472461C6F1050625
:10ED7000A6616462656584F8585052464946384633
:10ED8000054B98472060B8F1000F01D0C8F800404B
:10ED9000BDE8F88F5D1C410031E340005BE24000BC
:10EDA00070B5002407E004EB840293000B4818447C
:10EDB0000B4B98470134042CF5D90A4E3046084CC9
:10EDC000A047094D2846A0470848A0470848A04743
:10EDD000084B1E60084B1D6070BD00BF100F002067
:10EDE00045E24000880F00209C0F0020BC0F00204F
:10EDF000D40F0020080F00200C0F002010B504468F
:10EE00001C4B98471C4A1368013313601B4B1B684B
:10EE1000002B26D01A4B1B683BB9184B1B68DA6ACB
:10EE2000E36A9A4201D8154B1C60164A13680133F5
:10EE300013606364E36A01229A401349086802433D
:10EE40000A6003EB83039A00211D10481044104B05
:10EE50009847104B98470A4B1B680BB1074B1B6830
:10EE600010BD064B1C601368012BDED10A4B98477E
:10EE7000DBE700BF85E34000740F0020040F002093
:10EE8000D00F0020800F0020840F0020100F0020E2
:10EE900061E24000A5E34000A1ED400070B50446EA
:10EEA0000E461D4B1D681D4B186804301C4B9847BF
:10EEB00050B91A4B1B68DA6A012303FA02F21949A6
:10EEC0000B6823EA02030B60B4F1FF3F13D02C441C
:10EED000124B1B685C60A54216D8134B18680F4B89
:10EEE00019680431114B9847114B1B689C4201D2A1
:10EEF0000F4B1C6070BD002EE9D0084B196804311F
:10EF00000C480D4B984770BD0C4B1868034B1968A3
:10EF10000431064B984770BDE80F0020040F002015
:10EF2000ADE24000840F0020080F002079E240008D
:10EF3000B40F0020D40F002061E240000C0F00202D
:10EF400008B54FF08052044B1A60BFF34F8FBFF3E8
:10EF50006F8F024B9847F4E704ED00E04502410053
:10EF60002DE9F04385B006460F46154698469000B9
:10EF7000144B984700B381465C20124B98470446D7
:10EF8000B0B1C0F83090CCB10023039302940D9B34
:10EF900001930C9B009343462A46394630460A4D5E
:10EFA000A8472046094B9847012005B0BDE8F083EB
:10EFB0004846074B9847E6E70024E4E74FF0FF3068
:10EFC000F3E700BFD9E4400005ED4000FDED40004F
:10EFD000FDE4400010B582B0134B01930023009371
:10EFE000462212491248134CA047012803D0012899
:10EFF00004D002B010BD104B9847F8E74FF0500313
:10F0000083F31188BFF36F8FBFF34F8F4FF0FF3241
:10F010000A4B1A6001220A4B1A600022094B1A603F
:10F02000094B9847E5E700BFB00F0020A45041000E
:10F0300041EF400061EF4000B9FB4000B40F0020F9
:10F04000D00F0020E80F00207DE44000024A136842
:10F0500001331360704700BF7C0F0020014B18681C
:10F06000704700BFE80F002070B52F4B1B68002BC6
:10F0700052D12E4B1E6801361E604EB12C4B1B68C0
:10F080009E422FD22B4B1B68002B42D0002070BD1C
:10F09000294A1168294B186810601960284A1368BA
:10F0A00001331360274B9847E8E7012320E04FF036
:10F0B000FF321F4B1A60E5E71D4A1360E2E704F1D7
:10F0C0001800214B9847E36A01229A401F490868BB
:10F0D00002430A6003EB83039A0029461C4810444C
:10F0E0001C4B9847144B1B681B68002BDDD000237A
:10F0F000002BDCD1104B1B68DB68DC6863689E4228
:10F10000DAD3251D2846104B9847A36A002BD6D189
:10F11000D9E7114B9847B9E7064A136801331360E2
:10F120000D4B9847B2E700BF7C0F0020E80F00208E
:10F13000B40F0020780F0020080F00200C0F0020D3
:10F14000B80F0020D1EC4000ADE24000840F002059
:10F15000100F002061E240000903410070B5274B09
:10F160009847274B1A68013A1A601B68002B32D166
:10F17000244B1B68002B2ED00024234B1B6813B399
:10F18000214BDB68DC6804F11800204EB047251DD8
:10F190002846B047E36A01229A401D4908680243A5
:10F1A0000A6003EB83039A0029461A4810441A4B5D
:10F1B0009847E26A194B1B68DB6A9A42DDD3012249
:10F1C000174B1A60D9E70CB1164B9847164B1C68C1
:10F1D0003CB9134B1B68154B9847002070BD013C90
:10F1E00007D0134B98470028F9D001220C4B1A6026
:10F1F000F5E700220C4B1A60EBE700BF85E3400007
:10F200007C0F0020740F0020BC0F0020ADE24000F6
:10F21000840F0020100F002061E24000040F002046
:10F22000EC0F0020D1EC4000780F0020A5E3400057
:10F2300069F0400010B550B9002038B94FF0805245
:10F24000084B1A60BFF34F8FBFF36F8F10BD04469A
:10F25000054B984700212046044B9847044B98479C
:10F26000EBE700BF04ED00E04DF040009DEE4000F4
:10F270005DF1400070B50646154B98470524013CEA
:10F2800004EB84029300314612481844124B98470D
:10F29000054608B9002CF2D12DB15DB18DB10F4BEF
:10F2A0009847284670BD0E4B186831460A4B984760
:10F2B0000546F2E70B4B18683146074B9847054661
:10F2C000ECE731460848044B98470546E7E700BF9E
:10F2D0004DF04000100F00205DEC40005DF140005B
:10F2E000080F00200C0F0020D40F0020264B1B68B5
:10F2F000002B2FD110B50022244B1A60244B1B6821
:10F300001B6B1A68B2F1A53F28D0214B1868196809
:10F310003431204B9847204B1B68B3FA83F3DBB2A0
:10F32000C3F11F031D489A00D418A10001444C6882
:10F3300064684C601A4491000831084484421AD031
:10F3400003EB83039A00154B13445B68DA68104B98
:10F350001A6010BD01220D4B1A6070475A68B2F155
:10F36000A53FD2D19A68B2F1A53FCED1DB68B3F107
:10F37000A53FCAD1CFE7606803EB83029100074A3B
:10F380000A445060DCE700BF7C0F0020EC0F002037
:10F39000040F002009024100840F0020100F0020FC
:10F3A00010B50C46044B19681831044B98470121DD
:10F3B0002046034B984710BD040F002079E240001F
:10F3C0009DEE400038B50D461446064B19681831BD
:10F3D000054B98470CB14FF0FF3521462846034BAB
:10F3E000984738BD040F002061E240009DEE4000C8
:10F3F00038B5C368DC6804F118052846144B9847F3
:10F40000144B1B68E3B9251D2846114B9847E36A46
:10F4100001229A401049086802430A6003EB830303
:10F420009A0029460D4810440D4B9847E26A0D4B4F
:10F430001B68DB6A9A4208D901200B4B186038BD63
:10F4400029460A48064B9847F0E7002038BD00BF20
:10F45000ADE240007C0F0020840F0020100F002040
:10F4600061E24000040F0020EC0F0020BC0F0020E0
:10F47000034B1B680360034B1B684360704700BF6E
:10F48000B80F0020E80F0020F8B504460D46124BD7
:10F490009847124B19686268881A2B68B3F1FF3FCE
:10F4A00016D027680E4E3668B74201D0914211D26D
:10F4B000984206D300232B6001240A4B984720462C
:10F4C000F8BD1B1A2B602046074B98470024F4E731
:10F4D0000024F2E70124F0E785E34000E80F002074
:10F4E000B80F0020A5E3400071F440000122014B59
:10F4F0001A607047EC0F002008B5034618B1186B6E
:10F50000024B984708BD024B1B68F8E7BDEC400072
:10F51000040F0020054B1B6823B1054B1B681BB96A
:10F52000022070470120704700207047D00F002054
:10F530007C0F0020002854D038B50446C26A2A49FE
:10F540000968C96A8A4242D28169002905DB2649D5
:10F550000968C96AC1F105018161606902EB820233
:10F560009100224A0A44904207D000223AB91E4A2A
:10F570001268D26AE262012038BD0122F6E7251D39
:10F5800028461B4B984768B9E36A03EB83018A005E
:10F5900016498A5832B901229A4016490B6823EA63
:10F5A00002030B60104B1B68DB6AE362012404FA60
:10F5B00003F21049086802430A6003EB83039A00D0
:10F5C00029460A4810440C4B9847204638BDC26C67
:10F5D000054B1B68DB6A9A4201D2012038BD00202E
:10F5E00038BD0020704700BF040F0020100F00201E
:10F5F000ADE24000840F002061E24000002834D0DA
:10F6000038B50446026D013A0265C06AE16C884271
:10F610002DD00AB1002038BD251D2846154B98472E
:10F6200068B9E36A03EB83018A0013498A5832B947
:10F6300001229A4011490B6823EA02030B60E36C34
:10F64000E362C3F10502A261012404FA03F20B494B
:10F65000086802430A6003EB83039A0029460648C0
:10F660001044074B9847204638BD002070470020C3
:10F6700038BD00BFADE24000100F0020840F002015
:10F6800061E24000002843D038B50446C26C8A428B
:10F6900000D20A46E16A8A4202D0206D012800D0D9
:10F6A00038BDE262A069002802DBC2F10502A26156
:10F6B000636901EB81018800164A0244934225D018
:10F6C0000022002AECD0251D2846134B984768B924
:10F6D000E36A03EB83018A000E498A5832B901229A
:10F6E0009A400E490B6823EA02030B60E36A012289
:10F6F0009A400A49086802430A6003EB83039A00B0
:10F70000294604481044064B9847C9E70122D8E728
:10F71000704700BF100F0020ADE24000840F0020B2
:10F7200061E24000054B1B6823B1044B1A68136D5E
:10F7300001331365014B1868704700BF040F0020A8
:10F7400038B505460C461A4B98471A4B1B685B6D3B
:10F750002BB9184B1B68012283F85820ACB9164B03
:10F760009847134B9847134B1B685C6D24B1CDB978
:10F77000104B1B68621E5A650E4B1B68002283F8F3
:10F7800058200D4B9847204638BD114620460B4B5C
:10F7900098474FF080520A4B1A60BFF34F8FBFF368
:10F7A0006F8FDCE7034B1B6800225A65E4E700BF5C
:10F7B00085E34000040F0020A5E340009DEE4000DB
:10F7C00004ED00E0F8B507460D4614461E46214BF1
:10F7D0009847214B1B6893F85830DBB2022B0AD0B4
:10F7E0001D4B1A68506D20EA070050651B68012206
:10F7F00083F85820CEB9194B9847164B98471CB13F
:10F80000154B1B685B6D2360134B1B6893F85830D6
:10F81000DBB2022B16D000240F4B1B68002283F8AA
:10F8200058200E4B98472046F8BD114630460C4BE9
:10F8300098474FF080520B4B1A60BFF34F8FBFF3C6
:10F840006F8FD8E7044B1A68536D23EA0505556599
:10F850000124E1E785E34000040F0020A5E3400018
:10F860009DEE400004ED00E0F8B504460F46154655
:10F870001E46214B98470EB1636D336094F85830A3
:10F88000DBB2022284F858206A1E032A1AD8DFE865
:10F8900002F0020C1114626D174367650125012BFC
:10F8A00014D0164B98472846F8BD626D0132626548
:10F8B0000125F4E767650125F1E7022B04D06765B0
:10F8C0000125ECE70125EAE70025E8E7261D30469B
:10F8D0000B4B9847E36A01229A400A4908680243A1
:10F8E0000A6003EB83039A00314607481044074B34
:10F8F0009847074B1B68D4E785E34000A5E3400029
:10F90000ADE24000840F0020100F002061E24000B3
:10F91000040F0020F8B5EFF311854FF0500484F385
:10F920001188BFF36F8FBFF34F8F0BB1446D1C6015
:10F9300090F85830DBB2022480F85840013A032A8C
:10F940001AD8DFE802F0020C1114426D1143416530
:10F950000126012B14D085F311883046F8BD426D85
:10F96000013242650126F4E741650126F1E7022BE9
:10F9700004D041650126ECE70126EAE70026E8E726
:10F980000446164B1B68F3B9071D3846144B9847BD
:10F99000E36A01229A401349086802430A6003EBB4
:10F9A00083039A00394610481044104B9847E26A86
:10F9B0000F4B1B68DB6A9A42CDD9069B4BB10123E2
:10F9C000069A1360C7E700F118010A48074B9847E9
:10F9D000EDE70122084B1A60BDE700BF7C0F002055
:10F9E000ADE24000840F0020100F002061E24000D3
:10F9F000040F0020BC0F0020EC0F0020F8B5EFF33F
:10FA000011854FF0500383F31188BFF36F8FBFF35D
:10FA10004F8F90F85830DBB2022280F85820426DA8
:10FA200001324265012B02D085F31188F8BD0E46E4
:10FA30000446154B1B68E3B9071D3846134B98471E
:10FA4000E36A01229A401249086802430A6003EB04
:10FA500083039A0039460F4810440F4B9847E26AD7
:10FA60000E4B1B68DB6A9A42DED946B10123336034
:10FA7000DAE700F118010A48074B9847EFE701223F
:10FA8000084B1A60D0E700BF7C0F0020ADE24000B9
:10FA9000840F0020100F002061E24000040F0020BE
:10FAA000BC0F0020EC0F0020064B1A681368B3FA55
:10FAB00083F35B09036013B9D368186870470020AB
:10FAC000704700BFF00F002008B54160006191420F
:10FAD0000CD8D21A83699A4201D3012008BD011DB6
:10FAE000094B1868094B9847002008BD9A4201D27B
:10FAF000994206D2011D064B1868044B9847002016
:10FB000008BD012008BD00BFF40F002079E24000CD
:10FB1000F00F002070B5104B9847104B1B6813B1C5
:10FB20000F4B984770BD0F4D28460F4EB0470F4CF6
:10FB30002046B0470E4B1D600E4B1C6000220C216E
:10FB40000A200D4B9847054B18600028E8D00B4958
:10FB50000B4B9847E4E700BF85E3400024100020EA
:10FB6000A5E34000F80F002045E240000C10002003
:10FB7000F00F0020F40F002039E74000AC504100A6
:10FB8000D1EB40002DE9F041079C7CB19846154629
:10FB90000E460746064B98472760A661E561C4F804
:10FBA0002080069B6362201D024B9847BDE8F081D0
:10FBB00015FB40005BE2400010B582B0094B98474E
:10FBC000094B1B6863B1094B019303230093002386
:10FBD0004FF42F7206490748074CA04702B010BDEA
:10FBE0000020FBE715FB4000241000202810002017
:10FBF000B4504100F1FE400061EF40002DE9F041BA
:10FC000082B005460E46174698462C20084B98476A
:10FC1000044640B10190089B009343463A46314662
:10FC20002846044DA847204602B0BDE8F08100BF39
:10FC3000D9E4400085FB400030B585B0134C256801
:10FC40000DB31C46019102920390052913DC104B61
:10FC50009847022807D000231A4601A90B480068DC
:10FC60000C4CA0470DE00023089A01A90748006842
:10FC7000084CA04705E00023224601A92846064C6F
:10FC8000A04705B030BD0020FBE700BF24100020D6
:10FC900015F5400075E74000CDE8400070B582B032
:10FCA000154B1B681A6802B3DB681E68DC68251DEB
:10FCB0002846124B9847636A20469847E369012B10
:10FCC000EED1A36933449E4207D263602461294682
:10FCD000094B18680A4B9847E2E7002100910B4650
:10FCE00032462046074CA047DAE7074A1068024927
:10FCF0000860136002B070BDF00F0020ADE240005C
:10FD000079E2400039FC4000F40F002038B5054688
:10FD1000084B98470446084B1B68984205D30023BC
:10FD20002B60054B1C60204638BD044B98470123CF
:10FD30002B60F6E75DF04000201000209DFC4000A5
:10FD400070B582B005460E460F4B1B68DB68DC6859
:10FD5000201D0E4B9847E369012B04D0636A2046AF
:10FD6000984702B070BDA1692B463246294420460F
:10FD7000074EB0470028F1D0002100910B462A46DB
:10FD80002046044DA847E9E7F00F0020ADE240000F
:10FD9000C9FA400039FC400070B582B006460C46F6
:10FDA000174B984701A8174B9847019B23BB054663
:10FDB0000CB9B04219D22CB1134B1B681C68B4FAB1
:10FDC00084F464092246711B104B1868104B984745
:10FDD000104B984738B94FF080520F4B1A60BFF361
:10FDE0004F8FBFF36F8F02B070BD0A4B9847294603
:10FDF00030460A4B9847F6E7064B9847F3E700BFB3
:10FE00004DF040000DFD4000F40F002024100020B4
:10FE1000F9EB40005DF1400004ED00E041FD4000E1
:10FE200030B587B0002203A92A4B18682A4B98479F
:10FE300000284CD0039B002BF4DB059C636913B1B5
:10FE4000201D264B984702A8254B9847039B092B5A
:10FE5000E8D801A252F823F081FE400081FE400064
:10FE600081FE400025FE4000B5FE4000C7FE400078
:10FE700081FE400081FE400025FE4000B5FE4000AE
:10FE80000499A5690B46024629442046154DA8470A
:10FE90000028C7D0636A20469847E369012BC1D187
:10FEA000A269002100910B460498024420460E4CA2
:10FEB000A047B7E70499A1610346024601442046E2
:10FEC000084CA047AEE72046084B9847AAE707B082
:10FED00030BD00BF2410002045E94000ADE24000E5
:10FEE0000DFD4000C9FA400039FC4000FDE440002F
:10FEF00000B583B001A8044B98470199034B98477C
:10FF0000034B9847F6E700BFA9FA400099FD40006F
:10FF100021FE4000064BDB6BC3F30023054A137040
:10FF2000054BDB6BC3F34033044A1370704700BFCB
:10FF300000100E402C100020000E0E402D1000204E
:10FF400008B5054BDB6B13F4004F02D1034B984708
:10FF500008BD034B984708BD000E0E40BD5440003D
:10FF6000E154400030B583B004460D4600230193B0
:10FF70002E4B984213D02E4B9C421AD02D4B9C42B4
:10FF800021D02D4B9C4228D02C4B9C422FD02C4B67
:10FF90009C4236D02B4B9C423DD003B030BD01A9D2
:10FFA0002046294B98470028F9D19DF804302B7042
:10FFB000E1E701A92046244B98470028F9D19DF894
:10FFC00004302B70DAE701A920461F4B9847002820
:10FFD000F9D19DF804302B70D3E701A920461A4BC4
:10FFE00098470028F9D19DF804302B70CCE701A97F
:10FFF0002046154B98470028F9D19DF804302B7006
:020000040041B9
:10000000C5E701A92046104B98470028F9D19DF873
:1000100004302B70BEE701A920460B4B98470028FF
:10002000F9D19DF804302B70B7E700BF00C2004043
:1000300000020240004202400082014000C2014032
:100040000082004000020440EDDE400038B5044666
:100050000D46274B984213D0264B984218D0264B7A
:1000600098421DD0254B984222D0254B984227D04C
:10007000244B98422CD0244B984231D0002038BDDC
:1000800029462046214B98470028F9D1012038BD48
:10009000294620461D4B98470028F9D1012038BD3C
:1000A00029462046194B98470028F9D1012038BD30
:1000B00029462046154B98470028F9D1012038BD24
:1000C00029462046114B98470028F9D1012038BD18
:1000D000294620460D4B98470028F9D1012038BD0C
:1000E00029462046094B98470028F9D1012038BD00
:1000F00000C2004000020240004202400082014073
:1001000000C201400082004000020440C5DE400001
:1001100000B583B002A9002341F8043D084B1868DC
:10012000084B9847019B3BB14FF08052064B1A6039
:10013000BFF34F8FBFF36F8F03B05DF804FB00BFB9
:1001400034100020FDF9400004ED00E070B58AB0E5
:100150001D4B0FCB0AAC04E90F001C4D1C4B1D605E
:100160001C4A1D4B1A601D4A1D4B1A60069B0093CA
:10017000079B0193089B0293099B0393002404941B
:10018000184E3046184B984701213046174B984778
:10019000174A69462846174B98472846164B9847F2
:1001A0002846164B9847164E336821469868154DD9
:1001B000A847336821465868A8473368214698689D
:1001C000A8470AB070BD00BFBC504100008201408A
:1001D000382300204D0041003423002065FF4000FB
:1001E0003023002000800140ADDA400015DC4000E3
:1001F0000000DC0551DF40009DDE4000A9DE40002C
:100200003C030020491D410008B504460D460A463E
:1002100001460748074B98470220074B9847294655
:100220002046064B9847EFF30580054B9847FFDEC5
:1002300080514100B5134100854D4000714D400093
:10024000914D400070B51F4B98471F4B1B68C31A58
:10025000632B00D870BD1C4B18601C4B18681C4DDC
:10026000A8471C4C20601C481C4EB047A847606043
:100270001B48B047A847A0601A48B047A847E060AD
:100280001948B047A84720611848B047A84760619F
:100290001748B047A847A0611648B047A847E06193
:1002A0001548B047A84720621448B047A847606285
:1002B0001348B047A847A0621248B047A847E06279
:1002C000C8E700BF5DF0400030100020341000206F
:1002D000F9F44000B42300207451410075F240004D
:1002E00040484100DC4F4100FC4F4100305041008C
:1002F0005050410070504100904F4100D84741009C
:10030000A4504100B4504100704700002DE9F04373
:1003100083B04B4B98474B4A936843F0254343F4D3
:1003200080139360484B9847484B9847484B9847F1
:10033000484B9847484B9847484B98470446484B8A
:100340009847F02201462046464B9847464B98472F
:100350004648474B03602223037123234371454DD5
:100360002946454CA0474548454B03602B23037164
:100370002A2343712946A047424B9847424B98474E
:100380004248434B98474348434CA047434944485D
:10039000A04744494448A047444A45494548A047E6
:1003A00000230193042200924FF480724249434893
:1003B000434CA047012802D04248374B98473E485B
:1003C000414B9847414B1860414B9847414B9847E8
:1003D000414B9847414B9847414A00210F20414EDD
:1003E000B047414C03220B212046404DA847DFF87F
:1003F00010914A4600212820B0473D4F03220C218E
:100400003846A8472820DFF8FC80C0470146384618
:10041000384FB8474A4600210D20B04703220B2130
:100420002046A8470D20C04701462046B847324B1A
:100430009847324B9847002003B0BDE8F08300BFD7
:100440006945400010140E402DD94000957A4000B7
:10045000D16E40004D014100A17640005978400026
:10046000617840001977400035774000A0230020D4
:1004700000000240A0860100657340008C2300202C
:1004800000C00140C9B74000996D40001101410012
:100490005D454000CC504100B5134100E45041009F
:1004A000F85041009044410004514100185141006E
:1004B0002451410030514100485141006D784000C5
:1004C00061EF40005051410075F2400034100020AF
:1004D000E5974000ADAE4000E9A040000990400023
:1004E00041FF40002DBB4000000E0E409DBB400070
:1004F00000100E40ABD840001F504000D5EF400028
:1005000015FF4000CFD8400030B583B000248DF8EF
:1005100004408DF805408DF806400F4B98470F4B6F
:10052000984720460E4B98470E4D01A928460E4B82
:10053000984772B60D480E4CA0472846A0470D4B71
:1005400098470D4B98470D4B98470D4A136823F079
:100550000103136003B030BD617A40004DF04000EC
:10056000055440008C230020A1634000A0230020FC
:10057000FD734000A953400015B84000B577400016
:1005800010E000E000487047A023002000487047BA
:100590008C23002008B5014B984708BD69784000BE
:1005A00008B5014B984708BD6B78400070470120A3
:1005B0007047000008B50248024B984708BD00BFCD
:1005C000A02300209D74400008B50248024B9847C4
:1005D00008BD00BF8C2300209D744000014B18789B
:1005E000704700BF2D100020014B1878704700BFE6
:1005F0002C10002070B58AB0044600F06FF8324B22
:1006000093F900506B1C064609D02146204600F0A5
:100610008DFE20B90021204600F07EFE10B130464C
:100620000AB070BD294B08902046019300F006FBEC
:10063000CDE90401CDE902012046CDB9244B4FF0AC
:1006400060420021CDE9062300F03EFE002833D0B1
:1006500002230093684600F085F9A8B1089BC3B94E
:10066000DDE9060100F03EFB064630460AB070BDEB
:10067000184B00220021CDE9062300F025FE68B1C9
:1006800002239D420093E5D100F066FE2223036021
:10069000E4E700F061FE089B0360E1E70123022D1F
:1006A00000930BD100F058FE212303600A4800F0AC
:1006B0005BF9CDE90601D1E701230093684600F01C
:1006C00051F90028F2D1EDE738030020985141009C
:1006D000FFFFEFC70000F0FFA05041002DE9F84FE9
:1006E00030F000432DD00028014604464ADBB0F12B
:1006F000FF4F3BDAB0F5000F3CDB00268D4AC4F318
:1007000016052A4402F40002E41582F07E507F3C74
:1007100034444FF07E51284304EBD25400F036FBB2
:1007200005F10F03C3F316030F2B064631DC00213E
:1007300000F0CAFD002800F094804CB90020BDE80C
:10074000F88F00214FF04C4000F0DEFCBDE8F88F40
:10075000204600F0D1FB7849054600F021FC77499E
:100760000446284600F01CFC0146204600F010FB21
:10077000BDE8F88F4FF0984100F012FC6FF01806BA
:100780000446BBE700F002FB002100F0BDFCBDE821
:10079000F88F4FF0804100F0FBFA0146304600F040
:1007A000B3FC8046204600F0A7FB41468146404608
:1007B00000F0F6FB0146834600F0F2FB6049DFF8EB
:1007C000A0A1074600F0ECFB5E4900F0E1FA3946D3
:1007D00000F0E6FB5C4900F0DBFA394600F0E0FB94
:1007E0005A4900F0D5FA594600F0DAFB58498346D9
:1007F000384600F0D5FB574900F0CAFA394600F0F8
:10080000CFFB554900F0C4FA394600F0C9FB014658
:10081000584600F0BDFAC5F55713AA4403F52273F4
:1008200043EA0A03002B074665DD4FF07C51304652
:1008300000F0B6FB314600F0B3FB0546002C32D188
:100840002946384600F0A4FA414600F0A9FB0146CB
:10085000284600F09BFA0146304600F097FABDE8C2
:10086000F88F3E49304600F09BFB01464FF07C502C
:1008700000F08CFA31460546304600F091FB014607
:10088000284600F08DFB0546002C2ED0204600F0B7
:1008900033FB2949074600F083FB284904463846C4
:1008A00000F07EFB14E02449484600F079FB29461D
:1008B0000446384600F06CFA414600F071FB1F49CF
:1008C0000746484600F06CFB0146384600F060FAE7
:1008D0000146284600F05AFA314600F057FA014620
:1008E000204600F053FABDE8F88F0146304600F08C
:1008F0004DFABDE8F88F7CB10F49484600F050FB37
:1009000039460446304600F041FA414600F048FBC3
:100910000A4905464846C3E70146304600F036FA24
:10092000414600F03DFB0146304600F02FFABDE89D
:10093000F88F00BF20FB4A008071313FD1F7173795
:100940009788173E25333A3E2549923EABAA2A3F67
:100950004FD01C3E298E633ECDCCCC3EABAAAA3EE6
:10096000305CCFFF0020704700200149704700BF76
:100970000000F87F81F0004102E000BF83F00043F7
:1009800030B54FEA41044FEA430594EA050F08BF2A
:1009900090EA020F1FBF54EA000C55EA020C7FEAEE
:1009A000645C7FEA655C00F0E2804FEA5454D4EB6B
:1009B0005555B8BF6D420CDD2C4480EA020281EA35
:1009C000030382EA000083EA010180EA020281EA6D
:1009D0000303362D88BF30BD11F0004F4FEA0131BF
:1009E0004FF4801C4CEA113102D0404261EB4101CE
:1009F00013F0004F4FEA03334CEA133302D0524254
:100A000063EB430394EA050F00F0A780A4F101040F
:100A1000D5F1200E0DDB02FA0EFC22FA05F2801849
:100A200041F1000103FA0EF2801843FA05F359412F
:100A30000EE0A5F120050EF1200E012A03FA0EFCAE
:100A400028BF4CF0020C43FA05F3C01851EBE371D8
:100A500001F0004507D54FF0000EDCF1000C7EEBF5
:100A600000006EEB0101B1F5801F1BD3B1F5001F33
:100A70000CD349085FEA30004FEA3C0C04F1010452
:100A80004FEA445212F5800F80F09A80BCF1004F7B
:100A900008BF5FEA500C50F1000041EB045141EAFD
:100AA000050130BD5FEA4C0C404141EB010111F4FE
:100AB000801FA4F10104E9D191F0000F04BF0146A9
:100AC0000020B1FA81F308BF2033A3F10B03B3F187
:100AD00020020CDA0C3208DD02F1140CC2F10C0217
:100AE00001FA0CF021FA02F10CE002F11402D8BF75
:100AF000C2F1200C01FA02F120FA0CFCDCBF41EA41
:100B00000C019040E41AA2BF01EB0451294330BD0F
:100B10006FEA04041F3C1CDA0C340EDC04F11404EC
:100B2000C4F1200220FA04F001FA02F340EA0300C3
:100B300021FA04F345EA030130BDC4F10C04C4F109
:100B4000200220FA02F001FA04F340EA03002946E9
:100B500030BD21FA04F0294630BD94F0000F83F433
:100B6000801306BF81F480110134013D4EE77FEA16
:100B7000645C18BF7FEA655C29D094EA050F08BF62
:100B800090EA020F05D054EA000C04BF1946104643
:100B900030BD91EA030F1EBF0021002030BD5FEA87
:100BA000545C05D14000494128BF41F0004130BDAF
:100BB00014F580043CBF01F5801130BD01F0004503
:100BC00045F0FE4141F470014FF0000030BD7FEA76
:100BD000645C1ABF194610467FEA655C1CBF0B4671
:100BE000024650EA013406BF52EA033591EA030F88
:100BF00041F4002130BD00BF90F0000F04BF002180
:100C0000704730B54FF4806404F132044FF00005B2
:100C10004FF0000150E700BF90F0000F04BF00212B
:100C2000704730B54FF4806404F1320410F0004591
:100C300048BF40424FF000013EE700BF42004FEA8C
:100C4000E2014FEA31014FEA02701FBF12F07F4309
:100C500093F07F4F81F06051704792F0000F14BF06
:100C600093F07F4F704730B54FF4607401F000454A
:100C700021F0004120E700BF50EA010208BF7047A1
:100C800030B54FF000050AE050EA010208BF704796
:100C900030B511F0004502D5404261EB41014FF4FF
:100CA000806404F132045FEA915C3FF4DCAE4FF003
:100CB00003025FEADC0C18BF03325FEADC0C18BFEA
:100CC000033202EBDC02C2F1200300FA03FC20FA3B
:100CD00002F001FA03FE40EA0E0021FA02F1144488
:100CE000C1E600BF4FEA4102B2F1E04324BFB3F5D1
:100CF000001CDCF1FE5C0DD901F0004C4FEAC00293
:100D00004CEA5070B2F1004F40EB830008BF20F076
:100D10000100704711F0804F21D113F13872BCBF30
:100D200001F00040704741F480114FEA5252C2F185
:100D30001802C2F1200C10FA0CF320FA02F018BFCE
:100D400040F001004FEAC1234FEAD32303FA0CFC21
:100D500040EA0C0023FA02F34FEA4303CCE77FEAB0
:100D6000625307D150EA01331EBF4FF0FE4040F4FA
:100D70004000704701F0004040F0FE4040F40000A9
:100D8000704700BF80F0004002E000BF81F00041EA
:100D900042001FBF5FEA410392EA030F7FEA226C21
:100DA0007FEA236C6AD04FEA1262D2EB1363C1BFB1
:100DB000D218414048404140B8BF5B42192B88BF20
:100DC000704710F0004F40F4000020F07F4018BF43
:100DD000404211F0004F41F4000121F07F4118BF63
:100DE000494292EA030F3FD0A2F1010241FA03FC0B
:100DF00010EB0C00C3F1200301FA03F100F00043F3
:100E000002D5494260EB4000B0F5000F13D3B0F1BA
:100E1000807F06D340084FEA310102F10102FE2A29
:100E200051D2B1F1004F40EBC25008BF20F0010099
:100E300040EA03007047490040EB000010F4000F47
:100E4000A2F10102EDD1B0FA80FCACF1080CB2EBDA
:100E50000C0200FA0CF0AABF00EBC2505242184339
:100E6000BCBFD0401843704792F0000F81F40001DE
:100E700006BF80F400000132013BB5E74FEA4103B1
:100E80007FEA226C18BF7FEA236C21D092EA030F1D
:100E900004D092F0000F08BF0846704790EA010F97
:100EA0001CBF0020704712F07F4F04D1400028BFC4
:100EB00040F00040704712F100723CBF00F50000A6
:100EC000704700F0004343F0FE4040F400007047DC
:100ED0007FEA226216BF08467FEA23630146420288
:100EE00006BF5FEA412390EA010F40F4800070479B
:100EF0004FF0000304E000BF10F0004348BF404241
:100F00005FEA000C08BF704743F0964301464FF07C
:100F100000001CE050EA010208BF70474FF00003D8
:100F20000AE000BF50EA010208BF704711F0004319
:100F300002D5404261EB41015FEA010C02BF8446E9
:100F40000146002043F0B64308BFA3F18053A3F548
:100F50000003BCFA8CF2083AA3EBC25310DB01FA8F
:100F600002FC634400FA02FCC2F12002BCF1004F13
:100F700020FA02F243EB020008BF20F001007047A4
:100F800002F1200201FA02FCC2F1200250EA4C00F8
:100F900021FA02F243EB020008BF20EADC7070473E
:100FA0004FF0FF0C1CEAD0521EBF1CEAD15392EA4C
:100FB0000C0F93EA0C0F6FD01A4480EA010C400228
:100FC00018BF5FEA41211ED04FF0006343EA501082
:100FD00043EA5111A0FB01310CF00040B1F5000FC4
:100FE0003EBF490041EAD3715B0040EA010062F173
:100FF0007F02FD2A1DD8B3F1004F40EBC25008BF5D
:1010000020F00100704790F0000F0CF0004C08BF7A
:1010100049024CEA502040EA51207F3AC2BFD2F147
:10102000FF0340EAC250704740F400004FF0000355
:10103000013A5DDC12F1190FDCBF00F0004070478F
:10104000C2F10002410021FA02F1C2F1200200FACD
:1010500002FC5FEA310040F1000053EA4C0308BF94
:1010600020EADC70704792F0000F00F0004C02BFE5
:10107000400010F4000F013AF9D040EA0C0093F060
:10108000000F01F0004C02BF490011F4000F013BBA
:10109000F9D041EA0C018FE70CEAD15392EA0C0F28
:1010A00018BF93EA0C0F0AD030F0004C18BF31F093
:1010B000004CD8D180EA010000F00040704790F069
:1010C000000F17BF90F0004F084691F0000F91F00D
:1010D000004F14D092EA0C0F01D142020FD193EAD3
:1010E0000C0F03D14B0218BF084608D180EA01005B
:1010F00000F0004040F0FE4040F40000704740F037
:10110000FE4040F4400070474FF0FF0C1CEAD05204
:101110001EBF1CEAD15392EA0C0F93EA0C0F69D060
:10112000A2EB030280EA010C49024FEA402037D0CB
:101130004FF0805343EA111143EA10130CF00040C2
:101140008B4238BF5B0042F17D024FF4000C8B42B2
:1011500024BF5B1A40EA0C00B3EB510F24BFA3EB92
:10116000510340EA5C00B3EB910F24BFA3EB910362
:1011700040EA9C00B3EBD10F24BFA3EBD10340EABC
:10118000DC001B0118BF5FEA1C1CE0D1FD2A3FF602
:1011900050AF8B4240EBC25008BF20F001007047B7
:1011A0000CF0004C4CEA50207F32C2BFD2F1FF035A
:1011B00040EAC250704740F400004FF00003013A8B
:1011C00037E792F0000F00F0004C02BF400010F42F
:1011D000000F013AF9D040EA0C0093F0000F01F043
:1011E000004C02BF490011F4000F013BF9D041EA65
:1011F0000C0195E70CEAD15392EA0C0F08D1420298
:101200007FF47DAF93EA0C0F7FF470AF084676E76A
:1012100093EA0C0F04D14B023FF44CAF08466EE743
:1012200030F0004C18BF31F0004CCAD130F0004211
:101230007FF45CAF31F000437FF43CAF5FE700BF69
:101240004FF0FF3C06E000BF4FF0010C02E000BF92
:101250004FF0010C4DF804CD4FEA40024FEA410334
:101260007FEA226C18BF7FEA236C11D001B052EAEA
:10127000530C18BF90EA010F58BFB2EB030088BFB0
:10128000C81738BF6FEAE17018BF40F0010070471F
:101290007FEA226C02D15FEA402C05D17FEA236C01
:1012A000E4D15FEA412CE1D05DF8040B704700BF48
:1012B000844608466146FFE70FB5FFF7C9FF0028DF
:1012C00048BF10F1000F0FBD4DF808EDFFF7F4FF18
:1012D0000CBF012000205DF808FB00BF4DF808EDB1
:1012E000FFF7EAFF34BF012000205DF808FB00BFD4
:1012F0004DF808EDFFF7E0FF94BF012000205DF8F6
:1013000008FB00BF4DF808EDFFF7D2FF94BF0120A6
:1013100000205DF808FB00BF4DF808EDFFF7C8FF9F
:1013200034BF012000205DF808FB00BF4FEA4002F7
:101330004FEA41037FEA226C02D15FEA402C08D1D8
:101340007FEA236C02D15FEA412C02D14FF000000A
:1013500070474FF001007047014B1868704700BF9D
:101360003C03002070B50F4E0F4D761BB61018BF12
:10137000002405D0013455F8043B9847A642F9D122
:101380000A4E0B4D761B03F0BFFFB61018BF0024AA
:1013900006D0013455F8043B9847A642F9D170BDF8
:1013A00070BD00BF14534100145341001C53410051
:1013B000145341000FB400B5074983B004AB08686B
:1013C00053F8042B8168019300F066FE03B05DF8CA
:1013D00004EB04B0704700BF3C030020024B014601
:1013E000186800F00BB800BF3C030020024B014618
:1013F000186801F06DBF00BF3C0300202DE9F04FDD
:1014000001F10B06162E83B0054640F29E8036F0A1
:10141000070600F1BD80B14200F2BA8000F06CFC1A
:10142000B6F5FC7FC0F09382730A00F0B880042BFD
:1014300000F27981B30903F1390003F1380EC300DA
:10144000BF4F3B44A3F108015C68A14206D10CE008
:10145000002A80F2AA80E468A14206D0636823F0E3
:1014600003039A1B0F2AF3DD70463C69DFF8E4E2C0
:10147000744500F0AB81636823F003039A1B0F2AC5
:1014800000F39081002AC7F814E0C7F810E080F25A
:101490009D80B3F5007F80F06181DB0803F1010CD2
:1014A00099107A6857F83C80C4F8088001238B4073
:1014B00007EBCC0113430839E1607B6047F83C40FF
:1014C000C8F80C408210012494409C4200F28B80AA
:1014D0001C4206D120F0030064001C4200F104000D
:1014E000FAD007EBC009CC468046DCF80C309C45AE
:1014F00007D16DE1002A80F27B81DB689C4500F01A
:101500006781596821F003018A1B0F2AF2DDD3F8A5
:101510000CC0D3F8088000939C19284646F00106B9
:1015200042F001055E60C8F80CC0CCF808807C6110
:101530003C61C4F80CE0C4F808E065605A5000F063
:10154000E1FB009B03F108041EE0102920D800F005
:10155000D3FB102618230220794F3B44A3F1080245
:101560005C68944200F03D816368E168A66823F0FE
:101570000303234428465A68F16042F001028E605A
:101580005A6000F0BFFB0834204603B0BDE8F08F7E
:1015900000240C2320462B6003B0BDE8F08F4020D0
:1015A0004FF400734FF03F0E4AE72344E1685A6856
:1015B000A66842F00102F16028468E605A6000F091
:1015C000A1FB0834204603B0BDE8F08F2344284631
:1015D0005A6842F001025A6000F094FB0834204639
:1015E00003B0BDE8F08FBC68636823F00308B04522
:1015F00004D3A8EB06030F2B00F38580DFF8589186
:10160000504BD9F800201B680132334404EB080A20
:1016100000F0558103F580530F3323F47F6B2BF0DB
:101620000F0B5946284600F07DFB411C024600F096
:10163000FC80824500F2F780434B196859441960D9
:1016400000F04D81D9F8000001301BBFA2EB0A0A5F
:101650005144C9F80020196012F0070100F015810B
:10166000C1F10800C1F580510244083102EB0B09B9
:10167000C9F30B09A1EB09094946284601930092D9
:1016800000F050FB431C9DE80C0000F04381801AE1
:10169000484440F001001968BA604944BC425060B7
:1016A000196017D0B8F10F0F40F2FB806068A8F105
:1016B0000C0222F0070204EB020E00F001004FF0D2
:1016C000050C10430F2A6060CEF804C0CEF808C0A5
:1016D00000F217811D4BBC681A68914288BF1960DF
:1016E0001B4B1A689142626888BF196022F003029E
:1016F0009642A2EB060301D80F2B04DC284600F02B
:1017000001FB002440E7A21943F0010346F0010663
:1017100066602846BA60536000F0F4FA0834204648
:1017200003B0BDE8F08F142B71D9542B00F2A380C5
:10173000330B03F16F0003F16E0EC30080E600BFB0
:10174000680700206810002038100020601000207A
:101750006410002070070020700B00205A0A042A31
:101760005BD9142A00F2AE8002F15C01C9005B3241
:1017700007EB010C7958ACF1080C8C4500F088801F
:101780004A6822F00302934273D289688C45F7D1EC
:10179000DCF80C207B68E260C4F808C09460CCF8E8
:1017A0000C408FE6A11946F0010C42F00106C4F886
:1017B00004C0284679613961C1F80CE0C1F808E03D
:1017C0004E60E25000F09EFA0834DDE67B6879E670
:1017D00008F1010818F0030F0CF1080C7FF485AE36
:1017E0002DE0DC68A34208BF02303FF43EAEBBE60A
:1017F00019441C464A68DB6854F8086F42F001023D
:101800004A602846F3609E6000F07CFABCE603F173
:101810005C0003F15B0EC30012E69A0902F1390184
:10182000C9003832A4E7BC4254D0BC68626822F0D8
:1018300003025DE759F80839994540F0868010F0B9
:10184000030F00F1FF30F5D17B6823EA04037B60CE
:1018500064009C423FF6C7AE002C3FF4C4AE1C426D
:1018600040467FF43EAE64001C4200F10400FAD012
:1018700037E68C468CE7B3F5AA7F15D8F30B03F156
:10188000780003F1770EC300DAE54FF48051EDE6FE
:101890007B689210012101FA02F213437B606246D9
:1018A00079E70123536029E740F25452934222D84A
:1018B000B30C03F17D0003F17C0EC300C0E503F11E
:1018C000100BAEE6542A29D81A0B02F16F01C90099
:1018D0006E324DE7204B196859441960B2E6CAF3DD
:1018E0000B0000287FF4AEAE08EB0B03BA6843F0A0
:1018F00001035360EEE67F204FF47E734FF07E0EBF
:101900009EE504F108012846009301F0E1FC009BEC
:101910001968DFE601204FF00009BCE6B2F5AA7FA6
:1019200005D8DA0B02F17801C900773220E740F2DE
:1019300054518A4205D89A0C02F17D01C9007C32CB
:1019400016E74FF47E717E2212E77B6880E7F0088D
:1019500006F1080300E600BF381000200000000078
:1019600001F0FF01102A2BDB10F0070F08D010F850
:10197000013B013A8B422DD010F0070F42B3F6D154
:10198000F0B441EA012141EA014122F007047FF06D
:1019900000070023F0E80256083C85EA010586EAC4
:1019A000010685FA47F5A3FA87F586FA47F6A5FA00
:1019B00087F68EB9EED1F0BC01F0FF0102F007020C
:1019C00032B110F8013B013A83EA010313B1F8D1B7
:1019D0000020704701387047002D06BF3546033898
:1019E000073815F0010F07D1013015F4807F02BFD1
:1019F000013015F4C03F0130F0BC0138704700BF22
:101A0000032A70B422D940EA01039B0711D003785E
:101A10000C78A3421DD10A44013105E010F8013FC2
:101A200011F8014BA34214D19142F7D1002070BCB0
:101A300070470D680668AE420C46034601F104018A
:101A400000F1040008D1043A032AF2D8002ADED1BA
:101A5000ECE7181B70BC704721461846D7E700BF5B
:101A6000844641EA000313F003036DD1403A41D3A9
:101A700051F8043B40F8043B51F8043B40F8043B68
:101A800051F8043B40F8043B51F8043B40F8043B58
:101A900051F8043B40F8043B51F8043B40F8043B48
:101AA00051F8043B40F8043B51F8043B40F8043B38
:101AB00051F8043B40F8043B51F8043B40F8043B28
:101AC00051F8043B40F8043B51F8043B40F8043B18
:101AD00051F8043B40F8043B51F8043B40F8043B08
:101AE00051F8043B40F8043B51F8043B40F8043BF8
:101AF000403ABDD2303211D351F8043B40F8043B98
:101B000051F8043B40F8043B51F8043B40F8043BD7
:101B100051F8043B40F8043B103AEDD20C3205D3A7
:101B200051F8043B40F8043B043AF9D2043208D09F
:101B3000D2071CBF11F8013B00F8013B01D30B8811
:101B400003806046704700BF082A13D38B078DD0EF
:101B500010F003038AD0C3F10403D21ADB071CBFC1
:101B600011F8013B00F8013B80D331F8023B20F82B
:101B7000023B7BE7043AD9D3013A11F8013B00F864
:101B8000013BF9D20B7803704B7843708B788370EC
:101B9000604670478842F0B50DD98B1898420AD23A
:101BA0008418002A51D0224613F8014D02F8014D45
:101BB0009942F9D1F0BD0F2A48D941EA00039B07A9
:101BC00046D100F1100401F11003154653F8106CD2
:101BD00044F8106C53F80C6C44F80C6C53F8086C17
:101BE00044F8086C103D53F8046C44F8046C0F2D55
:101BF00003F1100304F11004E8D8A2F1100323F05C
:101C00000F0302F00F0E1033BEF1030F194403440B
:101C100021D91E1F0D467446043C55F8047B46F836
:101C2000047F032CF8D8AEF1040424F00304043438
:101C30002144234402F0030262B1013B0A4411F83B
:101C4000014B03F8014F8A42F9D1F0BD0346F3E797
:101C50000346F2E7F0BD7246EEE700BF70B48607B8
:101C600046D0541E002A41D0CAB2034602E014F105
:101C7000FF343BD303F8012B9D07F8D1032C2ED959
:101C8000CDB245EA05250F2C45EA054519D903F1E2
:101C900010022646103E0F2E42F8105C42F80C5CF3
:101CA00042F8085C42F8045C02F11002F2D8A4F198
:101CB000100222F00F0204F00F041032032C134420
:101CC0000DD91E462246043A032A46F8045BFAD888
:101CD000221F22F003020432134404F003042CB147
:101CE000C9B21C4403F8011B9C42FBD170BC704775
:101CF00014460346C2E700BF014801F083BD00BFA0
:101D000004240020014801F07FBD00BF042400200E
:101D100010B5034B0446196801F01AFE204610BDA9
:101D20003C03002038B5074C0023054608462360D5
:101D3000FCF760FA431C00D038BD2368002BFBD0B1
:101D40002B6038BD1824002000290CBF022200227D
:101D50004FF4806300F000B82DE9F043614C256832
:101D600083B004460F4690461E4615B1AB6B002B60
:101D700064D0B8F1020F06D0B8F1010F00F29F80D5
:101D8000002EC0F29C80636ED80734D521462846C9
:101D900001F020F9216B41B104F14003994202D0D6
:101DA000284601F095FA00232363B4F90C30002291
:101DB000A26162601A063AD423F44A6323F0030353
:101DC000B8F1020FA3811DD001AB6A462146284617
:101DD00001F01CFDA3891843A081002E32D1009E82
:101DE0003046FFF7FBFA074600286BD0A38943F083
:101DF0008003A38128E0A3899905C7D4A06D01F0D1
:101E000001FDC3E70025616E002604F1430243F0A3
:101E100002030120A660CE07A381226022616061D7
:101E200001D498053ED5284603B0BDE8F08321696A
:101E3000284601F04DFAB4F90C30BDE7284601F010
:101E400021F996E7002FCBD0AB6B002B33D0009B52
:101E5000B4F90C2027609E421CBF42F40062A281AC
:101E6000B8F1010F04BF42F00102A28192B212F058
:101E70000803276166610ED0D1071AD5656E7642D8
:101E8000002315F00105A661A36009D000252846AE
:101E900003B0BDE8F083A360656E15F00105F5D1D0
:101EA0009305C0D4A06D01F0AFFC284603B0BDE897
:101EB000F083A660F0E7284601F0E4F8C7E74FF0AA
:101EC000FF35B0E7DDF80090B14504D04846FFF794
:101ED00085FA074620B9B4F90C304FF0FF3592E788
:101EE0004E4683E73C030020000000000000000095
:101EF00000000000000000000000000000000000E2
:101F000090F800F06DE9024520F007016FF0000C39
:101F100010F0070491F820F040F049804FF00004E1
:101F20006FF00700D1E9002391F840F000F10800BC
:101F300082FA4CF2A4FA8CF283FA4CF3A2FA8CF3F4
:101F40004BBBD1E9022382FA4CF200F10800A4FA5B
:101F50008CF283FA4CF3A2FA8CF3E3B9D1E90423AF
:101F600082FA4CF200F10800A4FA8CF283FA4CF3E6
:101F7000A2FA8CF37BB9D1E9062301F1200182FAA0
:101F80004CF200F10800A4FA8CF283FA4CF3A2FAA6
:101F90008CF3002BC6D0002A04BF04301A4612BAB4
:101FA000B2FA82F2FDE8024500EBD2007047D1E9B7
:101FB000002304F00305C4F100004FEAC50514F046
:101FC000040F91F840F00CFA05F562EA05021CBF17
:101FD00063EA050362464FF00004A9E7B1B1037854
:101FE000B3B10144431C994214D010B41A785C1C5C
:101FF00032B1A142234606D01A785C1C002AF8D1DF
:10200000181A10BC7047081A10BC70470846704771
:1020100018467047081A70472DE9F84F4B6E9C041C
:1020200093462FD59368126853B30E46074602F1C4
:10203000080919E920045FEA9A0817D0043D002432
:1020400001E0A04510D0324655F8041F384601F093
:10205000BBF8431C04F10104F3D10023CBF8083092
:10206000CBF80430BDE8F88FDBF808302AF0030A1B
:10207000A3EB0A03CBF8083009F10809002BD8D1EB
:102080000020EAE701F00AFA0023CBF80830CBF889
:102090000430BDE8F88F00BF2DE9F04FADB01D460C
:1020A0008B4690460793069018B1836B002B00F087
:1020B000F380DBF86430BBF90C00DF0781B202D497
:1020C0008E0540F1FC808C040AD4DBF8643040F4C7
:1020D000005123F40053ABF80C10CBF8643089B2F4
:1020E000080740F1B380DBF81030002B00F0AE8021
:1020F00001F01A030A2B00F0B58000230DF17009DE
:102100000B93119310930393CDF83C90CA46CDF8EE
:1021100010B098F800304446FBB1252B02D11CE0EA
:10212000252B03D014F8013F002BF9D1A4EB0805AF
:102130009DB1109B119ACAF8008001332A44072BE5
:10214000CAF80450119210937ADD002A40F0B0844E
:10215000039B10922B44CA4603932378002B00F074
:10216000E08300204FF000038DF8373004F10108C0
:1021700062780546064603464FF0FF3408F1010831
:10218000A2F12001582900F2DE82DFE811F02102DD
:10219000DC02DC022902DC02DC02DC02DC02DC0202
:1021A000DC0289029502DC02A200BD02DC029F0172
:1021B000A401A401A401A401A401A401A401A401F7
:1021C000A401DC02DC02DC02DC02DC02DC02DC0258
:1021D000DC02DC02DC02B201DC02DC02DC02DC023A
:1021E000DC02DC02DC02DC02DC02DC029701DC0245
:1021F000DC02DC02DC02DC029B01DC02DC025302BA
:10220000DC02DC02DC02DC02DC02DC02DC02DC02DE
:10221000DC02DC025A021B02DC02DC02DC026E027F
:102220001B02DC02DC027302DC02F50182010902FE
:10223000D702DC029A02DC02A700DC02DC022E02DA
:102240000AF1080A039B2B44039386E75946069834
:1022500000F0ACFD18BBBBF80C1001F01A030A2B00
:102260007FF44BAFBBF90E30002BFFF646AFDBF827
:102270006430DB0705D48F0503D4DBF8580001F088
:10228000C3FA2B4642465946069800F04DFD03908E
:1022900003982DB0BDE8F08F00F0F4FE09E7DBF8FD
:1022A0006430D90704D4BBF80C309A0540F1AA84F5
:1022B0004FF0FF33039303982DB0BDE8F08FDBF8A8
:1022C000580001F09FFABBF90C0081B2FBE67642A0
:1022D000079243F0040398F800204FE708969E0603
:1022E00000F150840799DD060A4600F1EF83580695
:1022F00040F1EC830E8804310027012207914FF052
:1023000000018DF837100025611C00F0168123F0C4
:102310008001029156EA070140F01481002C40F040
:102320005C83002A40F0B78313F00103059300F0AB
:1023300057840DF1B00B30230BF8413D059BA342B0
:10234000B8BF234601930DB101330193029B13F0F3
:102350000203099302D0019B02330193029B13F005
:1023600084030A9340F01782089B019A9D1A002D5E
:1023700040F31182102D40F39084109B119AC44EAB
:10238000D6461027A2461946069C07E001F1020C2A
:102390000EF1080E0146103D102D11DD481C1032C3
:1023A000072811928EE8C0001090EFDD002A40F05F
:1023B000E481103D102D11464FF0010CCE46EDDCAE
:1023C00054466146F2462A4407291192CAF8006031
:1023D000CAF80450109100F3EC829DF837500AF1CE
:1023E000080A481C002D40F0DE81099B002B00F0FC
:1023F000F88102320EA902230728119210908AE870
:102400000A0040F3EA81002A40F08C830A9B802B6B
:102410004FF001001146CA4640F0E781089B019D3C
:102420005E1B002E40F3E181102E9A4D40F3508444
:10243000D4461027A246069C07E001F1020E0CF1DB
:10244000080C0146103E102E11DD481C10320728E2
:1024500011928CE8A0001090EFDD002A40F09D82E0
:10246000103E102E4FF0010E1146CC46EDDC5446C6
:10247000E2463244BEF1070F11928AE86000CDF8BF
:1024800040E000F369830AF1080A0EF10100714689
:10249000ABE1089613F0200240F08C8313F010019A
:1024A00040F01A8313F0400200F0168307980A46A2
:1024B0000146043106880791002720E7089643F07B
:1024C0001003E7E7089643F0100308E743F08003A2
:1024D00098F8002052E6A2F13001002618F8012BEE
:1024E00006EB860601EB4606A2F130010929F5D973
:1024F00046E60896002840F0088443F010039E0644
:1025000000F14C83DD0600F1F382580640F1F082C1
:10251000079DB5F900602A46F71704323046394660
:102520000792002871F10002C0F25D83611C9DF8E2
:1025300037504FF001027FF4EAAE56EA070100F08F
:102540004D820293012A00F08C82022A40F05C82C4
:102550000B98CB46330906F00F0143EA07733A099B
:102560001E461746435C0BF8013D56EA0703F1D1BE
:10257000A9EB0B030593E1E6002840F0C083990620
:1025800000F16783DA0600F1F1805B0640F1EE802E
:10259000079A136804320792BDF80C201A80B8E538
:1025A00007983D4A08960B9206687822302104303D
:1025B0008DF8392043F00203079000278DF838107A
:1025C00002229CE60896002899D08DF8375096E7AD
:1025D00098F80020002D7FF4D1AD01202025CDE515
:1025E00043F0010398F80020C8E50896002840F061
:1025F000938329490B919F0600F1E8820798DE0634
:10260000014600F170825D0640F16D82043106885A
:1026100007910027D80740F1228256EA070100F00F
:102620001E8230218DF8392043F002038DF83810D6
:10263000022264E60896002840F06B8317490B914C
:10264000D9E7079908960A688DF848204FF00000EE
:102650000A468DF837000432012001900792059058
:102660000DF1480B0293002470E643F0400398F804
:10267000002083E598F800206C2A03BF98F8012019
:1026800043F0200308F1010843F0100376E500BF92
:10269000D4514100E4514100B8514100A4514100DE
:1026A00007990E680A46002E02F10402FFF60FAEEB
:1026B000079298F8002061E598F8002001202B256A
:1026C0005CE507990896D1F800B04FF000028DF84C
:1026D00037200E1DBBF1000F00F0E582671C00F0F3
:1026E000C4822246002158460193FFF739F9019B25
:1026F000002800F0E582A0EB0B02059207960293FA
:102700009DF83750002419E698F800202A2A08F18D
:10271000010700F0E982A2F130010929B8464FF023
:1027200000043FF62DAD18F8012B04EB840401EBF7
:102730004404A2F130010929F5D921E543F0200331
:1027400098F800201AE50896002840F0DB82002A5D
:1027500000F0E78001218DF848204FF00002019140
:102760008DF8372005910DF1480B7BE7079A136828
:1027700004320792039A1A60CBE40FAA0499204608
:10278000FFF74AFC002840F039811099119A01F1B5
:10279000010CCE46FFE51099119A481C9DF8375060
:1027A000002D3FF422AE01320DF13705012107283B
:1027B00011921090CAF80050CAF8041040F3088132
:1027C000002A40F0BC81099B002B3FF41FAE0EABEA
:1027D000022208461C931D92CA4601460AF1080AC5
:1027E00001300A9B802B3FF419AE059BE41A002CA4
:1027F0002EDD102CB34D1EDDD6461026069FDDF8CB
:1028000010A006E0881C0EF1080E1946103C102C92
:1028100010DD4B1C1032072B11928EE860001093D4
:10282000F0DD002A65D1103C102C4FF0010011465C
:10283000CE46EEDCF246224407281192CAF8005038
:10284000CAF80440109000F385800AF1080A0130AC
:102850000599CAF800B00A4407281192CAF8041072
:10286000109040F38280002A40F01881029B109261
:10287000580735D5089B01995C1A002C40F3E78076
:10288000CA46102C40F3188210998F4E069FDDF82F
:1028900010B0102506E0881C0AF1080A1946103C01
:1028A000102C11DD4B1C1032072B1192CAF800605E
:1028B000CAF804501093EEDD42BB103C102C4FF0D0
:1028C00001001146CA46EDDC224407281192CAF8DD
:1028D0000060CAF80440109051DD002A40F09B814E
:1028E000039B089A01998A42ACBF9B185B1803931B
:1028F0004EE00FAA51463846FFF78EFB002840F005
:102900003F811099119A481CCE467FE70FAA59467D
:102910003846FFF781FB60B91099119A481CCA46E6
:10292000BDE7119BDDF810B0002B40F0D4810023EF
:102930001093DBF8643013F0010FBBF80C3002D1B8
:102940009A0540F1DE805B063FF5B2AC03982DB0EE
:10295000BDE8F08F002A40F00681059A1D92012300
:102960001192CDF870B01093CA460AF1080A029B82
:10297000590704D5089B01995C1A002C81DC039B44
:10298000089901988142ACBF5B181B18039372BB76
:1029900000231093CA46FFF7BCBB0FAA0499204638
:1029A000FFF73AFB50BB1099119A01F1010ECC468A
:1029B00048E5002A40F040819DF83710002900F0DA
:1029C0001B8101220DF1370110461D921C91CA4650
:1029D00001460AF1080A013007E5029B012A00F0CE
:1029E0009880022A0DD1029300260027B0E50FAA95
:1029F00004990698FFF710FB0028C9D0DDF810B045
:102A000097E7029300260027494600E05946F2085E
:102A100042EA4772F80806F00703074616463033C5
:102A200056EA070201F8013C01F1FF3BEED1029AA0
:102A3000D6077FF59DAD302B3FF49AAD0239302398
:102A40000BF8013CA9EB010305938B4676E4039B4D
:102A5000089A8A42ACBF9B185B18039398E702223E
:102A60004DE4002F08BF0A2E52D3CB4630463946DC
:102A70000A22002301F054FB30320BF8012D3046BE
:102A8000394600230A2201F04BFB06460F4656EA60
:102A90000703EBD16CE50594CB464FE40FAA0499EC
:102AA0000698FFF7B9FA0028A8D1119ACA465EE73E
:102AB0000FAA04990698FFF7AFFA00289ED1CA46DC
:102AC000FFF7C0BBE4514100D45141000431166806
:102AD00007910122002712E4079801460431066895
:102AE000079100270BE40E6804310791002791E558
:102AF00007990E680A46F71704320792304639469E
:102B00000FE5DBF8580000F07FFEBBF80C301AE749
:102B1000029B02930DF1B00B303601230BF8416D8F
:102B200005930BE40FAA04990698FFF775FA00289D
:102B30007FF464AF1099119A481CCA4651E60FAA57
:102B400004990698FFF768FA00287FF457AF1099A8
:102B5000119A481CCA4648E4002A40F0918001209E
:102B60001146CA4641E60FAA04990698FFF754FA9F
:102B700000287FF443AF1098119A0130CA4667E6E7
:102B8000D346D6E6079E073626F0070202F1080173
:102B9000D2E9006707910122FFF7B1BB079E073614
:102BA00026F00706D6E9000106F10802079206465C
:102BB0000F46B6E4079E073626F0070202F1080129
:102BC000D2E9006707910022FFF799BB079E0736FD
:102BD00026F0070101F108000790D1E9006719E527
:102BE000CB46FFF7ABBB2D25764267EB47078DF849
:102BF00037500122FFF788BB099BB3B9114601206A
:102C0000CA46F2E5DBF8580000F0FEFD4FF0FF3356
:102C10000393FFF750BB0FAA04990698FFF7FCF93E
:102C200000287FF4EBAE119AA9E60EAB02221C93AA
:102C30001D920120CA46D0E50FAA04990698FFF715
:102C4000EBF900287FF4DAAE1099119A481CCA46B5
:102C5000A4E5079A03991368CD170846043229465C
:102C60000792C3E90001FFF754BA5846079602934A
:102C7000FFF746F9002405909DF83750FFF75EBB3B
:102C80000FAA04990698FFF7C7F900287FF4B6AE9B
:102C90001099119A481CCA46A7E51099119A204E1E
:102CA0000131FFF790BB062C28BF06240594079638
:102CB0000194DFF870B0D5E41098194E013003E6A6
:102CC00005949DF83750079602930446FFF736BBEC
:102CD0008646FFF7CEBB06980FAA5946FFF79CF928
:102CE00000283FF424AE24E6079998F801200C68E8
:102CF000043144EAE474B8460791FFF73FBA8DF80F
:102D000037503CE48DF8375021E58DF83750FFF708
:102D1000F4BB8DF8375091E48DF8375069E400BF6B
:102D2000D4514100CC5141002DE9F0410C46ADF5A4
:102D30008D6D8989666EE589199621F00201064636
:102D4000E069ADF80C1017464FF48061626AADF887
:102D50000E5098461AAD0023079016A809920693C4
:102D6000009504950291059100F048FD43463A46CE
:102D700069463046FFF790F9051E07DB3046694685
:102D800000F028F9002818BF4FF0FF35BDF80C30CF
:102D90005B0603D5A38943F04003A381169800F096
:102DA0002FFD28460DF58D6DBDE8F08138B5304B0F
:102DB0001B6805460C4613B19A6B002A38D0B4F94B
:102DC0000C2093B218070CD52069A8B113F00102AA
:102DD0001ED0636900225B42A361A260F0B10020B3
:102DE00038BDD9063CD5580726D4206942F00803DF
:102DF000A3819BB20028E9D103F42072B2F5007FD1
:102E0000E4D02846214600F02FFDA3892069DDE7A4
:102E1000990758BF6269A2600028E0D1B4F90C306C
:102E20001A06DDD543F04003A3814FF0FF3038BDD3
:102E3000184600F027F9C2E7216B51B104F14003B5
:102E4000994204D0284600F043FAB4F90C2000233C
:102E5000236300232069636022F024022060C5E719
:102E600042F0400209232B604FF0FF30A28138BDB1
:102E70003C030020024B13B1024800F005B8704734
:102E800000000000F5304100002301461A461846B4
:102E900001F01EB8B1F90C309AB22DE9F0410D469F
:102EA000110780463AD46A6843F40063002AAB8174
:102EB0006FDDAC6A002C49D000229BB2D8F80060CC
:102EC000C8F8002013F4805267D02A6D5F0705D53B
:102ED00069682B6B521A0BB1EB6BD21A0023E969AC
:102EE0004046A047441C3CD0B5F90C302A692A6002
:102EF00023F400630022AB81DB046A6047D4296BB2
:102F0000C8F8006011B305F14003994202D0404671
:102F100000F0DEF900202863BDE8F0812E69AEB133
:102F20002C682E6091070CBF6B690023A41BAB605B
:102F30000AE0234632466F6AE9694046B8470028EE
:102F4000A4EB0004064404DD002CF2DC0020BDE804
:102F5000F081AB8943F04003AB814FF0FF30BDE817
:102F6000F081D8F800401D2CF3D8194BE340DB4327
:102F700013F00103EDD1B5F90C206B6022F400636E
:102F80002969AB81DA042960B9D5002CB7D128654D
:102F9000B5E7EA6B002A8CDCD8E70123E9694046F3
:102FA000A047431C024602D0AB89AC6A8EE7D8F832
:102FB0000030002BF8D01D2B01D0162B02D1C8F801
:102FC0000060C3E7AB8943F04003AB81BDE8F0810B
:102FD0000100402038B50D46044608B1836BBBB1F3
:102FE000B5F90C0088B16B6EDB0701D4810517D5EC
:102FF00020462946FFF74EFF6B6EDA07044602D4DF
:10300000AB899B0507D5204638BD0446204638BD10
:1030100000F038F8E4E7A86D00F0F6FB204638BD74
:10302000A86D00F0EFFBE3E7014900F0AFBB00BF84
:10303000B93F410010B5002304468181C28103607D
:1030400043608360436603614361836119460822DC
:103050005C30FEF703FE07480749084A084B206228
:10306000E4616162A262E36204F15800BDE81040CD
:1030700000F0C4BBFD3C4100213D41005D3D4100ED
:103080007D3D410010B50446124800F0BBFBA26B29
:10309000D2B904F53B731048C4F8E8320321C4F8F0
:1030A000E022E063C4F8E41260680421FFF7C2FF85
:1030B00001220921A068FFF7BDFF02221221E0686A
:1030C000FFF7B8FF0123A3630248BDE8104000F0FA
:1030D0009BBB00BF0024002029304100014800F0C4
:1030E00091BB00BF14240020014800F08DBB00BF3D
:1030F0001424002038B50A4C0A4D641BA4100AD0D1
:1031000004F18043013B05EB8305013C55F804398C
:103110009847002CF9D1BDE8384002F0FFB800BF55
:103120002C534100285341002DE9F04782B08046DE
:103130008946144600F054FB012836D04A4604F173
:103140005C0301A9404600F075FE421C064625D0EE
:10315000A8B39DF804E000250DF1040A09E02368F6
:103160005A1C226083F800E00135B54227D215F8D9
:103170000AE0A368013B002BA360F0DAA769BB4219
:1031800071462246404602DBBEF10A0FE7D100F04D
:10319000F9FD431CE8D102B0BDE8F087A38943F0F4
:1031A0004003A38102B0BDE8F08709F1FF33FE2B95
:1031B000C4D85FFA89FE06468DF804E0CBE748469E
:1031C00002B0BDE8F08700BF30B5536E13F0010FB9
:1031D000B2F90C30144683B005469AB201D190057D
:1031E0001CD5900406D4626E43F4005342F400529E
:1031F000A381626628462246FFF796FF636EDA07D0
:10320000054602D4A3899B0502D5284603B030BDEC
:10321000A06D00F0F9FA284603B030BDA06D019111
:1032200000F0F0FAB4F90C3001999AB2D9E700BF76
:10323000F8B5244F0C460646FEF75EFDBB685D6898
:10324000C4F57E610F3125F00305294421F47F6127
:1032500021F00F01A1F58054B4F5805F07DB002158
:103260003046FEF75FFDBB682B44984204D03046E1
:10327000FEF748FD0020F8BD61423046FEF752FDE2
:1032800001300DD0104BBA6819682D1B45F00105AF
:103290003046091B55601960FEF734FD0120F8BD6A
:1032A00000213046FEF73EFDBA68831A0F2BDEDDA3
:1032B000064C0549246843F00103001B5360086075
:1032C000D5E700BF6807002038100020700B0020F1
:1032D000002944D02DE9F0410D468046FEF70CFD53
:1032E00055F8047C694927F00103A5F10804E218A8
:1032F0008E685068B24220F003005ED0FE07506036
:103300000BD455F8087CE41B01F1080EA56875453F
:103310003B446DD0E768EF60BD6015186D68ED0740
:103320003ED543F001026260E350B3F5007F17D24F
:10333000DB08581C9A104D6851F83070A7600123C3
:10334000934001EBC0022B43083AE2604B6041F826
:103350003040FC604046BDE8F041FEF7D3BC70470A
:103360005A0A042A52D89A0902F13907FF0002F1D9
:103370003805C819CA59083890424FD0516821F011
:1033800003018B4232D292689042F7D1C368A060A9
:10339000E3609C60C4604046BDE8F041FEF7B2BC0B
:1033A00095683B4FBD42034440D0D068E86043F08D
:1033B000010285606260E350B7E7FF07034407D46A
:1033C00055F8082CA41A1344A068E268C260906003
:1033D000304A126843F00100934260608C60B9D3B8
:1033E0002D4B40461968FFF723FFB3E71046CDE7A2
:1033F00011184968C90744D49168D268CA60034467
:1034000043F0010091606060E350A3E7142A16D8EE
:1034100002F15C07FF0002F15B05AAE7AA10012395
:103420004D6893402B434B600346B0E743F00102E5
:103430004C610C61E560A5606260E3508AE7542A44
:1034400006D81A0B02F16F07FF0002F16E0590E734
:10345000B2F5AA7F06D8DA0B02F17807FF0002F175
:10346000770586E740F25450824206D89A0C02F162
:103470007D07FF0002F17C057BE74FF47E777E2518
:1034800077E743F001016160136063E7680700209C
:1034900070070020740B0020681000209368002B38
:1034A00073D02DE9F04F8B8983B00C46190700903B
:1034B000164626D5226922B313F0020035682CD0B7
:1034C0004FF00009B04FC846B246B84543464A4699
:1034D00028BF3B460098B8F1000F50D0E169666AFA
:1034E000B047002858DDDAF808301B1A8144A8EBF1
:1034F0000008CAF80830002BE7D1002003B0BDE86F
:10350000F08F21460098FFF751FC002840F03381EE
:10351000A389356813F00200D2D113F0010945D117
:103520004F46019637B39A05D4F8088040F183805E
:103530004745C346C0F0AB8013F4906F40F0AC80B9
:103540002068BA465A464946FEF724FBA26823681B
:10355000A2EB08025B44A2602360019A9368A3EB8C
:103560000A03D144A7EB0A079360002BC5D0A389B7
:10357000002FD8D1D5F800906F680835D2E7D5F87C
:103580000090D5F8048008359FE700207047214659
:103590000098FFF71FFD70B3B4F90C3043F04003FF
:1035A0004FF0FF30A38103B0BDE8F08F8146334672
:1035B0004E46A8469A464D464EB380B320682369CE
:1035C0006269B145CB4628BFB34698425F4604D9ED
:1035D000A36813449B4500F3A68093454BDB134639
:1035E000676AE16900982A46B847071ED4DDB9EB3F
:1035F0000709CCD00120DAF80830DB1B3D44F61B6C
:10360000CAF80830002B3FF478AF002ED5D108F16E
:10361000080313E9600098460833002EF9D03246BB
:103620000A212846FEF79CF9002800F0A18001300D
:10363000A0EB0509C2E720682369984202D86369B4
:103640009F425DD2B84528BFB84642464946FEF77C
:10365000A1FAA3682268A3EB08034244A360226096
:103660000BB1C24679E721460098FFF7B3FC00286A
:1036700092D1C24671E75A462946FEF78BFAA268F4
:103680002368A2EB0B025B44A2602360AFE72068D3
:10369000B846BA46BB4655E762692068216902EB25
:1036A0004208A0EB010A08EBD8780AF101004FEAC2
:1036B000680838444045424684BF804642465B0520
:1036C00044D511460098FDF799FE8346002855D051
:1036D00052462169FEF7C4F9A38923F4906343F0AD
:1036E0008003A3810BEB0A00A8EB0A03C4F810B017
:1036F000C4F814802060A360B846BA46BB4621E7F0
:103700006FF00041B94228BF39464A4691FBF3F1B8
:103710000098666A03FB01F3E169B047B0F1000A63
:103720003FF71BAF38E71A4629460193FEF732FAF6
:103730002268019B00981A4422602146FFF74AFC48
:10374000019B00287FF428AF1F4650E7009800F047
:103750002FF983460028C5D1009D21692846FFF72F
:10376000B7FDB4F90C300C2223F080032A6015E772
:1037700006F1010922E74FF0FF30BFE6009A0C2363
:103780001360B4F90C3009E700FCFF7F2DE9F84322
:1037900010F538771FD0884606464FF000097D683F
:1037A000BC68013D11D4A389012B05F1FF3508D96F
:1037B000B4F90E3001332146304602D0C04749EA01
:1037C00000096B1C04F16804EDD13F68002FE6D1BD
:1037D0004846BDE8F883B9464846BDE8F88300BFCF
:1037E000044B054A1B685B6B002B08BF134693F81C
:1037F000280170473C0300207C0B0020704700BF6D
:10380000704700BF704700BF704700BF70B50C46DF
:10381000B1F90E10002990B015461E4614DB01AA1E
:1038200000F02CFC00280FDB029A02F47042A2F593
:103830000052B2FA82F252094FF480634FF40060F2
:1038400032602B6010B070BDA289002312F080009E
:10385000336004D0402218462A6010B070BD4FF487
:1038600080632B6010B070BD8A8992070B4606D525
:1038700001F1430201211A601A6159617047F0B5E4
:1038800083B001AB6A460C460646FFF7BFFF0099BE
:1038900005463046FDF7B2FDB4F90C30D8B1019AB7
:1038A000154F0099F76343F08003A38120602061E6
:1038B00061611AB92B43A38103B0F0BD3046B4F95E
:1038C0000E1000F0EFFBA0B1A38923F0030343F037
:1038D00001031BB2EEE79A05EED423F0030304F1D3
:1038E000430243F002030121A3812260226161614E
:1038F000E2E7B4F90C30DDE72930410070B4124C36
:1039000004F5806554F8083F5E6826F003060F2E24
:103910003146D4BF00200120E3689C4208D05A6899
:10392000DB6822F003029C4200F101001144F6D151
:103930000834A542F0D1054B1A685E62521A5860ED
:103940001962DA6170BC70476807002038100020E7
:10395000F8B50B4D064608460F46FEF7CDF9FFF7C2
:10396000CDFF0FCD34460FC40FCD0FC495E8030033
:1039700084E803003846FEF7C5F93046F8BD00BFBD
:103980003810002082B049B15AB16BB113780B6086
:103990001278101C18BF012002B0704701A9002A3C
:1039A000F3D1104602B070476FF00100F4E700BF9A
:1039B000002900F095802DE9F04F0D46164683B0A2
:1039C000804606F10B07FEF797F955F804EC162F21
:1039D0002EF00304A5F108093CD810221746BE4278
:1039E0003DD8944243DAC44B996809EB04008842FD
:1039F00000F0B480436823F0010101444968C9071D
:103A00004CD51EF0010F00F09B8031464046FDF77B
:103A1000F5FC064600283AD055F8043C23F0010393
:103A20004B44A0F108029A4200F02181221F242A6F
:103A300000F20781132A00F2DB8003462A46116850
:103A400019605168596092689A6029464046FFF7AC
:103A50003FFC1CE027F00707002F3A46BFDA00269C
:103A60000C233046C8F8003003B0BDE8F08F2E4676
:103A7000E31B0F2B1ED8D9F8043003F001032343B6
:103A80004C44C9F80430636843F001036360404666
:103A9000FEF738F9304603B0BDE8F08F23F003039A
:103AA000E11891421FDBC36882682E46D3600C4642
:103AB0009A60DDE7D9F8042009EB070102F0010262
:103AC0004C4443F001031743C9F804704B6063682A
:103AD00043F00103083163604046FFF7F9FBD6E786
:103AE0001146FDF78BBC1EF0010F8ED155F8081C56
:103AF000A9EB010ADAF8041021F003010B44234476
:103B0000934225DBC26881685646CA609160DAF844
:103B10000C1056F8080F221F242AC160886000F29A
:103B20009480132A6FD92968CAF808106968CAF8FE
:103B30000C101B2A00F2A28008350AF1100263E083
:103B400055F8083CA9EB030ADAF8041021F0030148
:103B500063189342FFF659AF5646D8E7416821F003
:103B6000030BA34407F11000834556DA1EF0010F42
:103B70007FF44BAF55F8081CA9EB010ADAF80410E2
:103B800021F003018B445845E2DC5646DAF80C106C
:103B900056F8080F221F242AC160886000F28F8027
:103BA000132A40F28A802968CAF808106968CAF89E
:103BB0000C101B2A00F28A8008350AF110022968CD
:103BC000116069685160A96891600AEB0701ABEB6D
:103BD000070242F0010299604A60DAF8043003F00B
:103BE00001031F434046CAF80470FEF78BF851E703
:103BF0002B6803606B6843601B2A2DD800F1080313
:103C000005F108021BE732462968116069685160B6
:103C1000A96891601C46D1462AE709EB0701ABEB86
:103C2000070B4BF0010299604A6055F8043C03F021
:103C300001031F43404645F8047CFEF763F82E4617
:103C400028E72946FDF7A6FFFFE6294630461C4631
:103C5000D146FDF79FFF0BE7AB688360EB68C3605D
:103C6000242A17D000F1100305F11002E7E650F8FE
:103C7000043C23F003031C442E46F9E6A968CAF865
:103C80001010E968CAF81410242A0CD010350AF173
:103C90001802B9E72B6903616B69436105F11802EA
:103CA00000F11803CBE62A69CAF818206A69CAF835
:103CB0001C2018350AF12002A6E732467FE7294684
:103CC00030460193FDF766FF019B7EE7A968CAF8BD
:103CD0001010E968CAF81410242A03D010350AF12C
:103CE00018026CE72A69CAF818206A69CAF81C2009
:103CF00018350AF1200262E76807002010B50C466B
:103D0000B1F90E1000F0F6F9002803DB236D03442F
:103D1000236510BDA38923F48053A38110BD00BF88
:103D20002DE9F0411646B1F90C201F46D3050C468B
:103D3000054607D500220223B1F90E1000F0C4F9A0
:103D4000B4F90C20B4F90E1022F48052A2813B4643
:103D500032462846BDE8F04100F0A4B810B50C4644
:103D6000B1F90E1000F0B0F9A389421C0EBF23F484
:103D7000805343F480532065A38110BDB1F90E1028
:103D800000F008B9F8B50D461446064610B1836B2D
:103D9000002B4BD0B4F90C20A369A36091B20807A3
:103DA00039D52369002B36D0EDB289042F4615D5BD
:103DB00022686169D31A8B421CDA0133A168501C56
:103DC0000139A1602060157062699A421AD0A389F6
:103DD000DB0701D50A2D15D03846F8BD616E42F4D7
:103DE000005221F40051A281226861666169D31AF0
:103DF0008B42E2DB21463046FFF7ECF840B92268FF
:103E00000123DBE721463046FFF7E4F80028E3D042
:103E10004FF0FF37E0E721463046FEF7C7FF0028A6
:103E2000F6D1B4F90C20236991B2BDE7FFF72AF966
:103E3000B0E700BFF0B5064685B01F4689B1104C0B
:103E4000104D2468646B002C08BF2C46D4F8E04069
:103E5000A047431C03D100228A233A60336005B097
:103E6000F0BD0C460649074A0968496B002908BF9E
:103E700011462246D1F8E04001A9A047E9E700BF7A
:103E80003C0300207C0B002021B1FF2A04D80A70DB
:103E900001207047084670478A2303604FF0FF30C7
:103EA000704700BF70B50D46084C114606461A46CD
:103EB000284600232360F9F7ABFD431C00D070BDFA
:103EC0002368002BFBD0336070BD00BF1824002096
:103ED0002DE9F8432C4D0646286898460F46914632
:103EE000FFF790FC294B1C68D4F84831002B3ED0DA
:103EF0005A681F2A1CDC02F1010E76B103EB820125
:103F00000124C1F88890D3F8880194402043022E00
:103F1000C3F88801C1F8088123D00232C3F804E055
:103F2000286843F82270FFF76FFC0020BDE8F88393
:103F3000174B0BB34FF4C870FDF750FA0346D8B1D6
:103F4000D4F848210260002141600A46C4F84801C3
:103F50004FF0010EC0F88811C0F88C11002EDCD093
:103F6000CCE7D3F88C110C43C3F88C41D5E704F5AA
:103F7000A673C4F84831BBE72868FFF745FC4FF04B
:103F8000FF30BDE8F88300BF780B0020A05141004E
:103F9000DD13410038B5074C002305460846236071
:103FA000FAF744F9431C00D038BD2368002BFBD03E
:103FB0002B6038BD1824002070B559B105460C4659
:103FC00010B1836B002B3CD0636ED80705D5B4F9D4
:103FD0000C302BB90026304670BDA38999053CD51D
:103FE00021462846FEF756FFE36A064633B1E169EB
:103FF000284698470028B8BF4FF0FF36A3891A0615
:1040000022D4216B41B104F14003994202D02846E9
:10401000FFF75EF900232363616C21B12846FFF7A7
:1040200057F900236364FFF759F8636E0022DB073A
:10403000A2810ED5A06DFFF7E3FBFFF755F83046E0
:1040400070BDFFF71FF8BFE721692846FFF740F969
:10405000D7E7A06DFFF7D8FBECE7A06DFFF7D2FB29
:10406000B4F90C30002BBBD1666E16F00106B1D14D
:10407000A06DFFF7C9FB304670BD00BF38B50B46D9
:10408000074C05461146184600232360FAF7D1F87D
:10409000431C00D038BD2368002BFBD02B6038BDFB
:1040A0001824002038B5074C002305460846236035
:1040B000FAF7C4F8431C00D038BD2368002BFBD0AE
:1040C0002B6038BD1824002070B50D46084C1146F1
:1040D00006461A46284600232360FAF7B1F8431C27
:1040E00000D070BD2368002BFBD0336070BD00BFD3
:1040F0001824002070B50D46084C114606461A4695
:10410000284600232360F9F769FC431C00D070BDEA
:104110002368002BFBD0336070BD00BF1824002043
:1041200053B94AB9002908BF00281CBF4FF0FF311E
:104130004FF0FF3000F07AB9ADF1080C6DE904CE14
:1041400000F006F8DDF804E0DDE9022304B0704772
:104150002DE9F0478C460D460446089E002B51D1B0
:104160008A4217466DD9B2FA82FEBEF1000F0BD01B
:10417000CEF1200C01FA0EF520FA0CFC02FA0EF733
:104180004CEA050C00FA0EF44FEA174A250CBCFB6A
:10419000FAF81FFA87F90AFB18CC45EA0C4508FB28
:1041A00009F3AB420AD9ED1908F1FF3280F02381FF
:1041B000AB4240F22081A8F102083D44ED1AA4B2BE
:1041C000B5FBFAF00AFB105544EA054400FB09F977
:1041D000A14509D9E41900F1FF3380F00A81A14516
:1041E00040F2078102383C44A4EB090440EA08404D
:1041F0000021002E61D024FA0EF400233460736095
:10420000BDE8F0878B4207D9002E54D0002186E804
:1042100021000846BDE8F087B3FA83F1002940F099
:104220008E80AB4202D3824200F2FA80841A65EBA0
:1042300003050120AC46002E3FD086E81010BDE8F3
:10424000F08712B90127B7FBF2F7B7FA87FEBEF184
:10425000000F34D1EB1B3A0C1FFA87FC0121B3FB92
:10426000F2F8250C02FB183345EA03450CFB08F372
:10427000AB4207D9ED1908F1FF3002D2AB4200F290
:10428000D1808046ED1AA3B2B5FBF2F002FB1055C7
:1042900043EA05440CFB00FCA44507D9E41900F1EE
:1042A000FF3302D2A44500F2B8801846A4EB0C04F8
:1042B00040EA08409DE731463046BDE8F087CEF140
:1042C000200405FA0EF307FA0EF720FA04F83A0C68
:1042D00025FA04F448EA0308B4FBF2F14FEA184562
:1042E00002FB11441FFA87FC45EA044501FB0CF36D
:1042F000AB4200FA0EF409D9ED1901F1FF3080F05C
:104300008A80AB4240F2878002393D44EB1A1FFAA3
:1043100088F5B3FBF2F002FB103345EA034500FBDE
:104320000CF3AB4207D9ED1900F1FF386FD2AB4265
:104330006DD902383D44EB1A40EA01418FE7C1F1E3
:10434000200722FA07F88B4005FA01F448EA030334
:1043500020FA07FE4FEA134CFD404EEA040EB5FB6F
:10436000FCF94FEA1E440CFB19551FFA83F844EA86
:10437000054509FB08F4AC4202FA01F200FA01FA21
:1043800008D9ED1809F1FF3043D2AC4241D9A9F167
:1043900002091D442D1B1FFA8EFEB5FBFCF00CFB21
:1043A00010554EEA054400FB08F8A04507D9E4186B
:1043B00000F1FF3529D2A04527D902381C4440EA34
:1043C0000940A4EB0804A0FB02894C45C6464D46B3
:1043D00015D312D056B1BAEB0E0364EB050404FA00
:1043E00007F7CB401F43CC40376074600021BDE825
:1043F000F0871846F8E69046E0E6C245EAD2B8EB08
:10440000020E69EB03050138E4E72846D7E740468A
:1044100091E78146BEE7014678E702383C4445E72C
:10442000084608E7A8F102083D442BE7704700BFA3
:10443000010000000200000004000000080000006D
:10444000100000002000000040000000800000007C
:1044500000008000000000010000000200000004D5
:104460000000000800000010000000000000000034
:10447000000000000000000000000000000000003C
:10448000000000000000000000000000000000002C
:10449000302E322E3235000064617461000000005D
:1044A000737461636B000000686561700000000058
:1044B0005A81000001280110020380025329035190
:1044C000FF01026902026B10058000404011088163
:1044D00002560009000F00088202560009000F0072
:1044E00002250103F0AA1104C00040000AC2010A1B
:1044F000010A010A00900203F0AA1202D32003BFAE
:1045000037BE000001280110020381025329035124
:10451000FF01026902026B102D70110000891080EA
:10452000078003C0078003C003C0020003580020B7
:10453000C637000D000F00110008180010F0030C22
:104540002000060B0B330580014040110881025604
:104550000009000F00088202560009000F00022522
:104560000103F0AA1002D10203F0AA1104C0004016
:10457000000AC2010A010A010A00900203F0AA120D
:1045800002D32003BF37BE000128011002038002BE
:1045900053290351FF01026900026B10058000409E
:1045A0004011088104AC0010001000088204AC0027
:1045B0001000100002250103F0AA1104C000400001
:1045C0000AC2010A010A010A00908203F0AA12023B
:1045D000D32003BF37BE000001010203800253292C
:1045E0000351FF01026900026B1005800040401179
:1045F00008810256000A00100008820256000A00D4
:10460000100002350002250103F0AA110AC2010AB6
:10461000010A010A00900203F0AA1202D32003BF8C
:1046200037BE03F0AA1105C4AA55018004C5001FB6
:10463000FF000000012801100203810253290351E9
:10464000FF01026900026B102D70110000891080BB
:1046500009F004F804F804F804F80200041B002030
:1046600091BF0011000F00190009180010F0030C91
:104670002000060B0B330580013E3E11088101E14D
:104680000006001000088201E1000600100002256B
:104690000103F0AA1002D10203F0AA110AC2010A12
:1046A000010A010A00908203F0AA1202D32003BF7C
:1046B00037BE000001280110020381025329035173
:1046C000FF01026900026B102D701100008910803B
:1046D00009F004F804F804F804F80200041B0020B0
:1046E00091BF0011000F00190009180010F0030C11
:1046F0002000060B0B330580013E3E11088101E1CD
:104700000006001000088201E100060010000225EA
:104710000103F0AA1002D10203F0AA110AC2010A91
:10472000010A010A00900203F0AA1202D32003BF7B
:1047300037BE0000012801100203810253290351F2
:10474000FF01026900026B102D70110000891080BA
:1047500009F004F804F804F804F80200041B00202F
:1047600091BF0011000F00190009180010F0030C90
:104770002000060B0B330580013E3E11088101E14C
:104780000010001000088201E10010001000022556
:104790000103F0AA1002D10203F0AA1104C00040E4
:1047A000000AC2010A010A010A00900203F0AA12DB
:1047B00002D32003BF37BE00585F666D747B8289C9
:1047C00090979EA5AC000000565852303000000073
:1047D000302E322E32350000555341525400000025
:1047E0004661696C656420746F20637265617465ED
:1047F000207573617274207461736B0D0A00000080
:1048000048494420436F6D6D616E64730000000081
:104810004661696C656420746F20637265617465BC
:104820002048494420636F6D6D616E642070726F23
:10483000636573736F72207461736B0D0A000000FF
:10484000484944205265706F727400004661696C7B
:10485000656420746F206372656174652048494403
:1048600020706572696F646963207265706F72741D
:10487000207461736B0D0A0056585244454C4554E0
:104880004500000043524153484E4F57000000007E
:1048900000FFFFFFFFFFFF0009279550D204000033
:1048A000021E0104A5000078E700000000000000DF
:1048B00000000000000001010101010101010101EE
:1048C000010101010101CAB40080F080187040208C
:1048D0009200FFFF0000001EA5510080A00020A054
:1048E00040200204FFFF0000001E00000000000046
:1048F00000000000000000000000000000000010A8
:104900000000000000000000000000000000017531
:10491000701279000000000000000000000000009C
:104920000000000000000000000000000000000087
:104930000000000000000000000000000000000077
:104940000000000000000000000000000000000067
:104950000000000000000000000000000000000057
:104960000000000000000000000000000000000047
:104970000000000000000000000000000000000037
:104980000000000000000000000000000000759022
:1049900000FFFFFFFFFFFF0009273412D2040000D1
:1049A000FF200104A5000078007875AA553BB229C4
:1049B0001050540000000101010101010101010139
:1049C00001010101010100000010000000000000D1
:1049D00000000000000000000000001000000000C7
:1049E00000000000000000000000000000100000B7
:1049F000000000000000000000000000000000FCBB
:104A0000004265796F6E640A202020202020015B1F
:104A1000702079070022091461430C88DF137F009E
:104A20003F801F00EF0917000E8001007E00073A4B
:104A30000292810008000000000000000000000059
:104A40000000000000000000000000000000000066
:104A50000000000000000000000000000000000056
:104A60000000000000000000000000000000000046
:104A70000000000000000000000000000000000036
:104A80000000000000000000000000000000209076
:104A900000FFFFFFFFFFFF0009279550D204000031
:104AA000021E0104A5000078E700000000000000DD
:104AB00000000000000001010101010101010101EC
:104AC000010101010101CAB40080F080187040208A
:104AD0009200FFFF0000001EA5510080A00020A052
:104AE00040200204FFFF0000001E00000000000044
:104AF00000000000000000000000000000000010A6
:104B0000000000000000000000000000000001752F
:104B10007012790000030014689F0080FF137F006B
:104B20003F801F00FF091F000F80010000000000F0
:104B30000000000000000000000000000000000075
:104B40000000000000000000000000000000000065
:104B50000000000000000000000000000000000055
:104B60000000000000000000000000000000000045
:104B70000000000000000000000000000000000035
:104B80000000000000000000000000000000B190E4
:104B900000FFFFFFFFFFFF0009273412D2040000CF
:104BA000FF200104A5000078007875AA553BB229C2
:104BB0001050540000000101010101010101010137
:104BC00001010101010100000010000000000000CF
:104BD00000000000000000000000001000000000C5
:104BE00000000000000000000000000000100000B5
:104BF000000000000000000000000000000000FCB9
:104C0000004265796F6E640A202020202020015B1D
:104C1000702079070022091441B70E88DF137F0046
:104C20003F801F00EF0917000E8001007E00073A49
:104C30000292810008000000000000000000000057
:104C40000000000000000000000000000000000064
:104C50000000000000000000000000000000000054
:104C60000000000000000000000000000000000044
:104C70000000000000000000000000000000000034
:104C80000000000000000000000000000000CA90CA
:104C900000FFFFFFFFFFFF0009273412D2040000CE
:104CA000FF200104A5000078007875AA553BB229C1
:104CB0001050540000000101010101010101010136
:104CC00001010101010100000010000000000000CE
:104CD00000000000000000000000001000000000C4
:104CE00000000000000000000000000000100000B4
:104CF000000000000000000000000000000000FCB8
:104D0000004265796F6E640A202020202020015B1C
:104D1000702079070022091439540F88DF137F00AF
:104D20003F801F00EF0917000E8001007E00073A48
:104D30000292810008000000000000000000000056
:104D40000000000000000000000000000000000063
:104D50000000000000000000000000000000000053
:104D60000000000000000000000000000000000043
:104D70000000000000000000000000000000000033
:104D8000000000000000000000000000000034905F
:104D900000FFFFFFFFFFFF0009273412D2040000CD
:104DA000FF200104A5000078007875AA553BB229C0
:104DB0001050540000000101010101010101010135
:104DC00001010101010100000010000000000000CD
:104DD00000000000000000000000001000000000C3
:104DE00000000000000000000000000000100000B3
:104DF000000000000000000000000000000000FCB7
:104E0000004265796F6E640A202020202020015B1B
:104E100070207907002209141EF50A88FF0EFF0092
:104E20003F801F007F071B000E8001007E00073AB5
:104E30000292810008000000000000000000000055
:104E40000000000000000000000000000000000062
:104E50000000000000000000000000000000000052
:104E60000000000000000000000000000000000042
:104E70000000000000000000000000000000000032
:104E8000000000000000000000000000000086900C
:104E900000FFFFFFFFFFFF0009273412D2040000CC
:104EA000FF200104A5000078007875AA553BB229BF
:104EB0001050540000000101010101010101010134
:104EC00001010101010100000010000000000000CC
:104ED00000000000000000000000001000000000C2
:104EE00000000000000000000000000000100000B2
:104EF000000000000000000000000000000000FCB6
:104F0000004265796F6E640A202020202020015B1A
:104F1000702079070022092839540F88DF137F0099
:104F20003F801F00EF0917000E8001001EF50A08E0
:104F3000FF0EFF003F801F007F071B000E80010057
:104F40007E00073A02928100080000000000000085
:104F50000000000000000000000000000000000051
:104F60000000000000000000000000000000000041
:104F70000000000000000000000000000000000031
:104F80000000000000000000000000000000E190B0
:104F9000766964656F5F70726F6300004661696C6B
:104FA000656420746F20637265617465207669643E
:104FB000656F2070726F636573736F7220746173B5
:104FC0006B0D0A0070726F785F74696D656F757430
:104FD0005F74696D65720000FF00FF004932430095
:104FE0004661696C656420746F20637265617465E5
:104FF00020493243207461736B0D0A0054494D45BA
:10500000445F5354415254004661696C6564207496
:105010006F206372656174652074696D65642073C7
:10502000746172747570207461736B0D0A000000F6
:10503000414443004661696C656420746F2063726B
:105040006561746520414443207461736B0D0A00EF
:105050004C4544004661696C656420746F2063723E
:1050600065617465204C4544207461736B0D0A00C2
:1050700046414E004661696C656420746F2063721E
:10508000656174652046616E207461736B0D0A0062
:1050900031323334202020202020202020202020C6
:1050A0000000000049444C4500000000546D72515E
:1050B00000000000546D72205376630000C20100AE
:1050C000C000000000080000000000002D2D20425C
:1050D000696773637265656E204265796F6E6420DF
:1050E0002D2D0A00444953504C4159424F415244DE
:1050F0002056302E342E32002D2D202573202D2DBC
:105100000A0000002D2D2056657273696F6E2025F0
:1051100073202D2D0A00000030383A34363A3330EF
:10512000000000004A616E203137203230323400F6
:105130002D2D20436F6D70696C65643A20257320B6
:105140002573202D2D0A00005553424C6F616400D9
:105150004661696C656420746F2063726561746573
:1051600020555342204C6F61646572207461736BEB
:105170000D0A000048494420436F6D6D616E640064
:10518000737461636B206F766572666C6F77202530
:10519000782025730D0A00006C6F67660000000020
:1051A000400300203031323334353637383941420C
:1051B0004344454600000000303132333435363741
:1051C000383961626364656600000000286E756CA2
:1051D0006C290000202020202020202020202020BA
:1051E00020202020303030303030303030303030FF
:1051F0003030303043000000504F53495800000019
:105200002E00000000202020202020202020282800
:105210002828282020202020202020202020202076
:1052200020202020208810101010101010101010B6
:1052300010101010100404040404040404040410E6
:105240001010101010104141414141410101010174
:10525000010101010101010101010101010101013E
:10526000101010101010424242424242020202024A
:10527000020202020202020202020202020202020E
:1052800010101010200000000000000000000000BE
:10529000000000000000000000000000000000000E
:1052A00000000000000000000000000000000000FE
:1052B00000000000000000000000000000000000EE
:1052C00000000000000000000000000000000000DE
:1052D00000000000000000000000000000000000CE
:1052E00000000000000000000000000000000000BE
:1052F00000000000000000000000000000000000AE
:105300000000000000000000F8B500BFF8BC08BCB9
:105310009E467047752E410029444000F8B500BFF5
:10532000F8BC08BC9E4670470544400024EEFF7F51
:105330000100000030B482B0049C5BB31D460368DA
:1053400043F480330360C9B241F0B44141608368E3
:105350000193019B13F0010FF9D1002306E099009E
:1053600001F58001096845F823100133A342F6D303
:10537000D2B242F0B442426083680193019B13F0C1
:10538000010FF9D0036823F480330360002002B0DA
:1053900030BC70470220FAE70160704782B041607C
:1053A00083680193019B13F0010FF9D0019800F07D
:1053B0000E0002B070470000714440007544400088
:1053C000774440007B4440007F444000B9444000A3
:1053D000094540008144400085444000914440001C
:1053E00009022200010100C032090400000103008B
:1053F0000000092111010001222600070581034058
:10540000000400001201000200000040BD35011040
:105410000001010203010000B8020020BC000020CE
:10542000F40000200180FFFFFFFF00000110FFFFDC
:105430000210FFFF0310FFFF0410FFFF0120FFFF1A
:105440000220FFFF0500000001000000904E410017
:105450000A010100807C797673706D6A6764615F10
:105460005C595754524F4D4B48464442403E3B3A9C
:1054700038363432302F2D2B2A282725242221207C
:105480001E1D1C1B1A181716151413121111100FBC
:105490000E0D0D0C0B0B0A09090808070706060577
:1054A00005040404030303030202020201010101D3
:1054B00001010000000000000000000101020202E2
:1054C00002020303030303030304040404040505A5
:1054D0000505050606060707070808080909090A59
:1054E0000A0B0B0C0C0D0D0E0F0F101111121314D3
:1054F0001515161718191B1C1D1E202122242527DF
:10550000292A2C2E30323437393C3E4144474A4D0B
:105510005054575B5F63676C70757A804747000033
:105520009802002008020020000000001002002065
:10553000AC02002009028500030100C032080B0004
:105540000201010002090400000001010002092417
:105550000100011E0001010C2402010102000203EE
:1055600000000009240302010100010009040100F8
:1055700000010200020904010101010200020724E6
:1055800001020101000B2402010202100180BB0094
:105590000905840500010100000725010000000045
:1055A0000904020001030000000921110100012289
:1055B00026000705810340000400000012010002DC
:1055C00000000040BD35010100010102030100009F
:1055D00094000020A8000020B802002005B0400080
:1055E00025B040007DB0400027B040000000000022
:1055F00006FFFF0901A10109020903150026FF00AA
:1056000075089540810209060907150026FF0075F7
:10561000089540B102C00000000300000000000037
:10562000000000000000000000000000000000007A
:105630000000000000000000000000000403090456
:1056400042696773637265656E0000004265796F39
:105650006E64000100127A00AAAAAAAA0100000042
:1056600040030020000000002C06002094060020CB
:10567000FC06002000000000000000000000000008
:10568000000000000000000000000000000000001A
:10569000000000000000000000000000000000000A
:1056A00000000000000000000000000000000000FA
:1056B00000000000000000000000000000000000EA
:1056C00000000000000000000000000000000000DA
:1056D00000000000000000000000000000000000CA
:1056E00000000000000000000000000000000000BA
:1056F00000000000000000000000000000000000AA
:105700000000000000000000000000000100000098
:10571000000000000E33CDAB34126DE6ECDE050068
:105720000B0000000000000000000000000000006E
:105730000000000000000000000000000000000069
:105740000000000000000000000000000000000059
:105750000000000000000000000000000000000049
:105760000000000000000000000000000000000039
:105A90000000000068070020680700207007002051
:105AA000700700207807002078070020800700207A
:105AB000800700208807002088070020900700202A
:105AC000900700209807002098070020A0070020DA
:105AD000A0070020A8070020A8070020B00700208A
:105AE000B0070020B8070020B8070020C00700203A
:105AF000C0070020C8070020C8070020D0070020EA
:105B0000D0070020D8070020D8070020E007002099
:105B1000E0070020E8070020E8070020F007002049
:105B2000F0070020F8070020F807002000080020F8
:105B300000080020080800200808002010080020A5
:105B40001008002018080020180800202008002055
:105B50002008002028080020280800203008002005
:105B600030080020380800203808002040080020B5
:105B70004008002048080020480800205008002065
:105B80005008002058080020580800206008002015
:105B900060080020680800206808002070080020C5
:105BA0007008002078080020780800208008002075
:105BB0008008002088080020880800209008002025
:105BC000900800209808002098080020A0080020D5
:105BD000A0080020A8080020A8080020B008002085
:105BE000B0080020B8080020B8080020C008002035
:105BF000C0080020C8080020C8080020D0080020E5
:105C0000D0080020D8080020D8080020E008002094
:105C1000E0080020E8080020E8080020F008002044
:105C2000F0080020F8080020F808002000090020F3
:105C300000090020080900200809002010090020A0
:105C40001009002018090020180900202009002050
:105C50002009002028090020280900203009002000
:105C600030090020380900203809002040090020B0
:105C70004009002048090020480900205009002060
:105C80005009002058090020580900206009002010
:105C900060090020680900206809002070090020C0
:105CA0007009002078090020780900208009002070
:105CB0008009002088090020880900209009002020
:105CC000900900209809002098090020A0090020D0
:105CD000A0090020A8090020A8090020B009002080
:105CE000B0090020B8090020B8090020C009002030
:105CF000C0090020C8090020C8090020D0090020E0
:105D0000D0090020D8090020D8090020E00900208F
:105D1000E0090020E8090020E8090020F00900203F
:105D2000F0090020F8090020F8090020000A0020EE
:105D3000000A0020080A0020080A0020100A00209B
:105D4000100A0020180A0020180A0020200A00204B
:105D5000200A0020280A0020280A0020300A0020FB
:105D6000300A0020380A0020380A0020400A0020AB
:105D7000400A0020480A0020480A0020500A00205B
:105D8000500A0020580A0020580A0020600A00200B
:105D9000600A0020680A0020680A0020700A0020BB
:105DA000700A0020780A0020780A0020800A00206B
:105DB000800A0020880A0020880A0020900A00201B
:105DC000900A0020980A0020980A0020A00A0020CB
:105DD000A00A0020A80A0020A80A0020B00A00207B
:105DE000B00A0020B80A0020B80A0020C00A00202B
:105DF000C00A0020C80A0020C80A0020D00A0020DB
:105E0000D00A0020D80A0020D80A0020E00A00208A
:105E1000E00A0020E80A0020E80A0020F00A00203A
:105E2000F00A0020F80A0020F80A0020000B0020E9
:105E3000000B0020080B0020080B0020100B002096
:105E4000100B0020180B0020180B0020200B002046
:105E5000200B0020280B0020280B0020300B0020F6
:105E6000300B0020380B0020380B0020400B0020A6
:105E7000400B0020480B0020480B0020500B002056
:105E8000500B0020580B0020580B0020600B002006
:105E9000600B0020FFFFFFFF00000200F423002042
:105EA00043000000000000000000000000000000AF
:105EB00000000000000000000000000000000000E2
:105EC000430000000000000000000000000000008F
:105ED00000000000000000000000000000000000C2
:105EE000430000000000000000000000000000006F
:105EF00000000000000000000000000000000000A2
:105F0000430000000000000000000000000000004E
:105F10000000000000000000000000000000000081
:105F2000430000000000000000000000000000002E
:105F30000000000000000000000000000000000061
:105F4000430000000000000000000000000000000E
:105F50000000000000000000000000000000000041
:105F600043000000000000000000000000000000EE
:105F70000000000000000000000000000000000021
:105F8000893E410085394100000000000452410073
:105F900000524100A0504100A0504100A0504100DB
:105FA000A0504100A0504100A0504100A05041002D
:105FB000A0504100A0504100FFFFFFFFFFFFFFFF87
:105FC000FFFFFFFFFFFF000001004153434949006D
:105FD00000000000000000000000000000000000C1
:105FE0000000000000000000000041534349490048
:105FF00000000000000000000000000000000000A1
:10600000000000000000000000000000FFFFFFFF94
:10601000FFFFFFFFFFFFFFFFFFFFFFFF1477534767
:00000001FF
